:100000000C945A060C94A0060C94A0060C94A0061E
:100010000C94A0060C94A0060C94A0060C94A006C8
:100020000C94A0060C94DE180C94A0060C94A00668
:100030000C945D320C94A0060C94A0060C94A006BF
:100040000C94A0060C94A0060C94B2150C94A00677
:100050000C94E00B0C94A0060C94AA0B0C94A00634
:100060000C949A1B0C94A0060C94E32D0C94A006FF
:100070000C9473750C94A0060C94D86FC11BC61B0E
:10008000CB1BD41BEB1B021C121C221C3F1C2B1E67
:10009000021CED1CFE1C2D1D4B1D681DC21D1D1ECE
:1000A0002420CE205D21DD211522B822BF24292560
:1000B000A325EC25362664269126F4263E2788279C
:1000C0008128022E362E792EE92E012F422FF92F6C
:1000D000C030C030C030C030C030C030C030C030A0
:1000E000C030C030C030753077307C3094309630BE
:1000F0000A0D426174743A002025642043656C6CDB
:10010000732000204C6F77207761726E696E6720D4
:100110006C6576656C3A2025642E2564000A0D46D0
:100120006F756E6420424C2D4374726C3A2000252A
:1001300064000A0D0A0D2121204D495353494E47B1
:1001400020424C2D4354524C3A202564202121005A
:100150000A0D3D3D3D3D3D3D3D3D3D3D3D3D3D3D32
:100160003D3D3D3D3D3D3D3D3D3D3D3D3D3D3D3DBF
:100170003D3D3D3D3D000A0D43616C696272617415
:10018000696E672070726573737572652073656E32
:10019000736F722E2E004F4B0A0D000A0D466C69CC
:1001A0006768742D74696D65202575206D696E20F2
:1001B00020546F74616C3A2575206D696E000A0DCC
:1001C000436F6E74726F6C3A200048656164696EAB
:1001D00067486F6C64004E6F726D616C20284143FC
:1001E000432D4D6F646529000A0D3D3D3D3D3D3D6C
:1001F0003D3D3D3D3D3D3D3D3D3D3D3D3D3D3D3D2F
:100200003D3D3D3D3D3D3D3D3D3D3D3D3D0A0D00BE
:10021000416E676C654E69636B2020202020202092
:10022000416E676C65526F6C6C202020202020206E
:100230004163634E69636B20202020202020202012
:10024000416363526F6C6C202020202020202020EE
:100250005961774779726F202020202020202020AC
:100260004865696768742056616C75652020202098
:100270004163635A2020202020202020202020209D
:1002800047617320202020202020202020202020B3
:10029000436F6D706173732056616C75652020200B
:1002A000566F6C74616765205B302E31565D20207F
:1002B0005265636569766572204C6576656C2020B1
:1002C0004779726F20436F6D706173732020202017
:1002D0004D6F746F7220312020202020202020209C
:1002E0004D6F746F7220322020202020202020208B
:1002F0004D6F746F7220332020202020202020207A
:100300004D6F746F72203420202020202020202068
:1003100031362020202020202020202020202020B6
:1003200031372020202020202020202020202020A5
:100330003138202020202020202020202020202094
:100340003139202020202020202020202020202083
:10035000536572766F20202020202020202020202E
:10036000486F76657267617320202020202020204E
:1003700043757272656E74205B302E31415D2020B2
:100380004361706163697479205B6D41685D202011
:1003900048656967687420536574706F696E74206E
:1003A0003235202020202020202020202020202026
:1003B0003236202020202020202020202020202015
:1003C000436F6D7061737320536574706F696E74E1
:1003D0004932432D4572726F722020202020202048
:1003E000424C204C696D6974202020202020202060
:1003F0004750535F4E69636B20202020202020202F
:100400004750535F526F6C6C20202020202020200A
:1004100021212120494E434F4D50415449424C45E2
:1004200020212121002E000A0D20444143206F721B
:1004300020493243204552524F5221204368656380
:100440006B204932432C2033567265662C20444180
:100450004320616E6420424C2D4374726C005B2516
:10046000695D005B25695D002B204D696B726F4BE8
:100470006F70746572202B0048573A5625642E25FC
:10048000642053573A25642E256425630053657410
:1004900074696E673A2564202573004D697865722A
:1004A000204572726F7221004861726477617265D3
:1004B000204572726F7220313A2564202121004D4F
:1004C000697373696E6720424C2D4374726C3A25D0
:1004D0006421210021204E432D4552523A202532DD
:1004E0006420212000493243204552524F5221219D
:1004F00021004865696768743A20202535690053F2
:100500006574706F696E743A253569005072657351
:10051000737572653A253569004F66667365743A7E
:1005200020202535690048656967687420636F6E0F
:1005300074726F6C0044495341424C4544006163FE
:10054000742E2062656172696E67004E69636B3A52
:1005500020202020202025356900526F6C6C3A2025
:10056000202020202025356900436F6D7061737352
:100570003A202020253569004B25693A2534692029
:10058000204B25693A25346920004E693A253469A3
:100590002020526F3A253469200047733A25346988
:1005A000202047693A253469200050313A253469C2
:1005B000202050323A253469200050333A253469DE
:1005C000202050343A25346920004779726F202D5D
:1005D0002053656E736F72004E69636B253469201A
:1005E000282533692E25692900526F6C6C253469E2
:1005F00020282533692E256929004769657225342D
:1006000069202825336929004E69636B20253469E8
:1006100020282533692E25782900526F6C6C2025FF
:10062000346920282533692E2578290059617720DF
:1006300020253469202825336929004E69636B2001
:100640002534692028253369292825336929005252
:100650006F6C6C20253469202825336929282533BF
:1006600069290059617720202534692028253369BC
:1006700029282533692900414343202D2053656EE5
:10068000736F72004E69636B20253469202825330F
:10069000692900526F6C6C20253469202825336944
:1006A00029005A2020202025346920282533692953
:1006B00000566F6C746167653A2020202533692EDF
:1006C000253169560043757272656E743A20202098
:1006D0002533692E2531694100506F7765723A20C4
:1006E00020202020253469570044697363686172B3
:1006F00067653A202535696D416800526563656913
:100700007665720052432D525353493A20202020DF
:100710002534690052432D5175616C6974793A2012
:100720002534690052432D4368616E6E656C733ADF
:1007300025346900436F6D70617373004D61676E9E
:1007400065743A202020253569004779726F3A2078
:100750002020202025356900536574706F696E7400
:100760003A2025356900506F746925693A202025A3
:10077000336900506F746925693A20202533690078
:10078000536572766F202000536574706F696E74C4
:10079000202025336900506F736974696F6E3A20A9
:1007A0002533690052616E67653A2533692D25331B
:1007B0006900424C2D4374726C204572726F7273E3
:1007C000200025336420253364202533642025331D
:1007D000642000424C2054656D70657261747572BE
:1007E00065002533642025336420253364202533B8
:1007F000642000424C2D4374726C20666F756E64E9
:100800002000202563202020256320202025632030
:100810002020256320002025632020202563202020
:100820002025632020202563200020256320202010
:100830002D2020202D2020202D200031300031318E
:1008400000313200466C696768742D54696D65200B
:100850002000546F74616C3A2535756D696E0041E6
:1008600063743A20202535756D696E0028726573B2
:10087000657429000A0D47656E65726174696E675B
:100880002064656661756C7420506172616D657479
:10089000657220536574202564000A0D5573696ED6
:1008A0006720506172616D657465722053657420B4
:1008B0002564000A0D47656E65726174696E672074
:1008C00064656661756C74204D6978657220546149
:1008D000626C65000A0D4D697865722D436F6E6616
:1008E00069673A202725732720282575204D6F74C6
:1008F0006F727329000A0D3D3D3D3D3D3D3D3D3D3F
:100900003D3D3D3D3D3D3D3D3D3D3D3D3D3D3D3D17
:100910003D3D3D3D3D000A0D414343206E6F742037
:1009200063616C69627261746564210D0A00000084
:100930008F001E01AD013B02CA025803E603740496
:1009400002058F051B06A7063307BE074808D20815
:100950005B09E3096B0AF20A780BFD0B810C040DAD
:10096000860D070E870E060F840F00107B10F51002
:100970006E11E5115B12CF124213B31323149214BC
:10098000FE146A15D3153B16A11605176717C8176D
:1009900027188318DE1837198E19E319361A871AA3
:1009A000D61A231B6E1BB61BFD1B411C831CC31CCC
:1009B000001D3C1D751DAB1DE01D121E421E6F1E4D
:1009C0009A1EC31EE91E0D1F2E1F4D1F691F841F77
:1009D0009B1FB01FC31FD31FE11FEC1FF51FFB1F81
:1009E000FF1F0020040100005D69000201014C6A44
:1009F00001030202E06A02040303886B030004049B
:100A00003D6B2532692E25316956002533642563F7
:100A100020253033646D2563005374617475730051
:100A20004552524F523A2025326420002534692025
:100A30002532693A25303269002534696D25630015
:100A40002533692025336920253369202533690042
:100A50002533692025336920253369202533690032
:100A600054656D7065726174757265732020202005
:100A7000002563432020202020002532692E2531C7
:100A80006956202533692E2531694100253469577F
:100A9000202536696D4168004D61676E65743A25A1
:100AA0003369252520253369256300496E636C6908
:100AB0002E3A25336925632028256929200025320F
:100AC000756D2F73205361743A2564200020203304
:100AD00044004E6F4678004447505300486F6D65A0
:100AE0003A2533646D202533642563202563004E49
:100AF0006F204E6176694374726C21000A0D77771E
:100B0000772E4D696B726F4B6F707465722E6465D2
:100B10002028632920486953797374656D732047D1
:100B20006D6248000A0D74686520757365206F66F4
:100B3000207468697320736F6674776172652069C9
:100B400073206F6E6C79207065726D697474656462
:100B5000200A0D6F6E206F726967696E616C204D9F
:100B6000696B726F4B6F707465722D486172647738
:100B70006172650047726175706E657220486F54CE
:100B800054004143542044534C004A657469207317
:100B90006174656C6C6974005370656B7472756D0B
:100BA00020736174656C6C697420284C6F772072B7
:100BB00065736F6C7574696F6E29005370656B7423
:100BC00072756D20736174656C6C697420283230A5
:100BD000343829005370656B7472756D20736174BD
:100BE000656C6C6974004D756C74697369676E61CE
:100BF0006C2050504D000A0D526563656976657230
:100C00003A2000756E6B6E6F776E2E205573696E8D
:100C1000672050504D2E2E2E006E6F74207375700D
:100C2000706F7274656420627920686172647761A4
:100C3000726521000A0D3D3D3D3D3D3D3D3D3D3D43
:100C40003D3D3D3D3D3D3D3D3D3D3D3D3D3D3D3DD4
:100C50003D3D3D3D3D3D3D3D3D000A0D466C6967D6
:100C60006874436F6E74726F6C0A0D4861726477BA
:100C70006172653A25642E25640A0D536F66747798
:100C80006172653A5625642E2564256320000A0D9D
:100C90003D3D3D3D3D3D3D3D3D3D3D3D3D3D3D3D84
:100CA0003D3D3D3D3D3D3D3D3D3D3D3D3D3D3D3D74
:100CB0003D3D3D0011241FBECFEFD0E1DEBFCDBFD3
:100CC00011E0A0E0B1E0E0E8F1EF02C005900D9284
:100CD000A63AB107D9F718E0A6EAB1E001C01D9223
:100CE000A636B107E1F76AEAE2E0F0E081E280933C
:100CF00057007491AE014F5F5F4F20EF37EFDA017D
:100D00009FE0F9012F5F3F4F84918D93915097FFA2
:100D1000F8CF773911F40000FECFFA019EE08191FF
:100D200068276095915097FFFACF8889681721F05E
:100D3000773911F40000FECF0E9461070C94BF7850
:100D40000C9400008091B605E82FFF27EE0FFF1FDF
:100D5000EC51F94F808191818D5E9F4F14F010927C
:100D60000301808191818A5B9F4FCCF480910301C4
:100D70008823A9F481E0809303018091A9038F5F08
:100D80008093A903853038F088EE93E09093DB01DF
:100D90008093DA0104C066E970E00E944B348091D0
:100DA000A9039927909337058093360508951F93DB
:100DB000CF93DF93182F882389F080EF90E09F93E3
:100DC0008F9386E992E19F938F93E0917503F09161
:100DD000760309950F900F900F900F908091D90591
:100DE000823308F044C084EF91E00E94A516EC0124
:100DF000112329F0CE010E94AE168823D9F3C2E058
:100E0000D0E026E530E080911E0190911F0182170D
:100E1000930730F02196255D3F4FC730D10598F3F9
:100E20008091D9059927C89F9001C99F300DD89FFF
:100E3000300D1124209300011123D9F068EC70E0EB
:100E40008C2F0E944B34DF93CF9388EF90E09F93D9
:100E50008F9386E992E19F938F93E0917503F091D0
:100E6000760309958DB79EB706968DBF02C0809315
:100E70000001112311F1809100016AE00E941278B3
:100E8000892F99279F938F93809100010E94127858
:100E900099279F938F9383E091E09F938F9386E9A7
:100EA00092E19F938F93E0917503F09176030995FA
:100EB0002DB73EB7285F3F4F2DBFDF91CF911F91D8
:100EC0000895CFEFD0E1DEBFCDBF8824992414B8B8
:100ED00015B807EE13E00253104017FFFCCF189B24
:100EE00006C0199B02C08DE007C08BE005C0199BAE
:100EF00002C084E101C08AE08093020181E887B9E1
:100F00003E9A8FEF88B98BE184B981E085B98EE391
:100F10008AB987E48BB9469A84B7877F84BF80916A
:100F200060008861809360001092600084EC99E01A
:100F30009093DB018093DA0110927702109276028F
:100F40001092E9061092E806109279021092780247
:100F500010927B0210927A0220910201243128F033
:100F600084EC94E0A0E0B0E004C08BE095E0A0E069
:100F7000B0E08093430190934401A0934501B09366
:100F800046012A3011F0243110F0289801C0289A27
:100F90000E940E170E94DF160E949E120E94343299
:100FA0000E94521A81E00E94972D0E9467610E9460
:100FB000776C0E942B74809102018C3010F4299A76
:100FC00001C0299878940E94A92C80912202826005
:100FD00080932202109225020E947E3F84EF91E0CE
:100FE0000E94A5168C018091220280FD05C0C801D7
:100FF0000E94AE168823B9F38DE191E09F938F9301
:10100000C6E9AC2EC2E1BC2EBF92AF92E09175034F
:10101000F0917603099580EA9FE00E94A5168C0165
:10102000C0E0D0E00F900F900F900F90B6E8EB2E3D
:10103000B6E0FB2EAAE3CA2EA6E0DA2E0E947E3F7F
:101040008091220280FD05C0C8010E94AE1688234F
:10105000B9F3F60180811816ACF40BC00E947E3FF4
:101060008091220280FD05C0C8010E94AE1688232F
:10107000B9F3C8010E94AE16882321F4F7018081DC
:10108000882364F7F701808187FF18C02196DF93DA
:10109000CF9321978FE291E09F938F93BF92AF926E
:1010A000E0917503F091760309958091A7018F5F18
:1010B0008093A7018DB79EB706968DBF2196E4E079
:1010C000F0E0CE0EDF1E88E090E0E80EF91ECC3096
:1010D000D10508F4B3CFC0E0D0E003E816E0FAE3AE
:1010E000EF2EF6E0FF2EF801838187FD1CC0F7018B
:1010F00080811816C4F42196DF93CF93219782E361
:1011000091E09F938F9386E992E19F938F93E09173
:101110007503F0917603099582E08093D8018DB72D
:101120009EB706968DBFF8018381807883832196D0
:1011300084E090E0E80EF91E085F1F4FCC30D10527
:1011400090F280E591E09F938F93C6E9D2E1DF931F
:10115000CF93E0917503F091760309959091B405D2
:101160008091A7010F900F900F900F90981728F47F
:1011700080918F03806180938F0386E791E09F9336
:101180008F93DF93CF93E0917503F09176030995E8
:1011900088EE93E00E94A5168C010E94581A0F90C9
:1011A0000F900F900F90C8010E94AE168823D9F3BC
:1011B00086E991E09F938F93DF93CF93E09175033E
:1011C000F0917603099580E00E941A358091020122
:1011D0000F900F900F900F908A3011F0843110F023
:1011E000289801C0289A80ED97E09093DB018093C6
:1011F000DA0185E58093AB038EE090E00E94DC2A63
:101200009927182F00278FE090E00E94DC2A080F12
:10121000111D1093AD010093AC018AE090E00E9493
:10122000DC2A9927182F00278BE090E00E94DC2A07
:10123000080F111D1093AB010093AA010F5F1F4F00
:1012400039F08091AC019091AD018F5F9F4F41F4D7
:101250001092AD011092AC011092AB011092AA0154
:101260008091AA019091AB019F938F938091AC01E3
:101270009091AD019F938F938BE991E09F938F9312
:10128000DF93CF93E0917503F091760309958DB7C5
:101290009EB708968DBF8EEB91E09F938F93DF935F
:1012A000CF93E0917503F091760309958091C20583
:1012B0000F900F900F900F90E0917503F0917603CF
:1012C00082FF07C08AEC91E09F938F93DF93CF93C7
:1012D00008C086ED91E09F938F9386E992E19F93FA
:1012E0008F9309950F900F900F900F900E94961F6B
:1012F00088E893E190933E0180933D0161E0F62EF2
:10130000F092AA038F2D0E94D7068091DC050E94DF
:10131000757388EE91E09F938F93DF93CF93E09165
:101320007503F0917603099580ED97E00E94A5166C
:101330008C018AEF90E00E94A51683E080930E0551
:101340001092A60180911F060F900F900F900F90A2
:1013500084FF02C0F092AE018091B001882311F0A9
:101360004798FECF8091DE01882309F4EBC180917C
:101370001001882309F4E6C11092DE018091A903CF
:10138000882319F00E94A20602C00E9483420E9494
:101390007E3F209102012A3011F0243110F028986C
:1013A00001C0289A80916A02882331F080916A02F4
:1013B000815080936A020EC080916F00806280939A
:1013C0006F001092E5061092E40680918F0388600A
:1013D00080938F0380913D0190913E0101979093FE
:1013E0003E0180933D0180913D0190913E01892B0A
:1013F00021F0809123028823C9F180913D019091D1
:101400003E01892BD9F40E94C12D85E090E0909394
:101410003E0180933D0180914805909149050196D8
:10142000909349058093480580918F038160809354
:101430008F0380910F05826080930F0580910801D2
:10144000909109018F5F9F4FC1F4809169028823B9
:10145000A1F088EA91E69093DB018093DA0180E8BD
:1014600090E0909309018093080107C02A3011F0A1
:10147000243110F0289801C0289A0E94FD748091B0
:10148000DE01882309F05EC180910E01882311F0EE
:101490000E9425170E94E2120E94300EC8010E948D
:1014A000AE16882309F44AC10C5E1F4F80912302B7
:1014B000882349F080918F03826080938F0380910D
:1014C0000F0582600FC08091DA019091DB01892BBA
:1014D00059F480913D0190913E01079728F0809149
:1014E0000F058D7F80930F0580916A02882361F03C
:1014F0008091AE01882341F01092AE0188E893E11B
:101500009093DB018093DA0180910501882321F01B
:101510008150809305012EC08093B5031092400244
:1015200010923F0210923E0210923D0210923C0235
:1015300010923B0280916A028823E1F480910801B5
:10154000909109018F5F9F4FA9F42091AE01223045
:1015500089F088E99AE39093DB018093DA0180E0D7
:101560009CE09093090180930801222319F082E006
:101570008093AE0180919C01893C48F0815080931A
:101580009C0180918F038B7F80938F033FC080915C
:10159000C5078823F9F080918F03846080938F03BF
:1015A00089E08093440380910801909109018F5F45
:1015B0009F4F81F480916902882361F088E99AE362
:1015C0009093DB018093DA0180E098EA909309011F
:1015D000809308011092380310923703109236035B
:1015E00010923503109234031092B8071092F70747
:1015F0001092F6071092F9071092F8078FEF9FEFFD
:101600009093F5078093F40710929C01809100015C
:10161000282F332780911E0190911F018217930775
:10162000CCF480913402806280933402809108016E
:10163000909109018F5F9F4FC1F480E797E19093EC
:10164000DB018093DA0180E093E0909309018093BD
:1016500008010BC08091DA019091DB01892B29F4FC
:10166000809134028F7D809334020E94126684E060
:101670008093D9018091340281FD05C05AEA852EFC
:1016800055E0952E12C08091AF018F5F8093AF011E
:10169000813359F41092AF018091A8019091A90172
:1016A00001969093A9018093A8010894811C911C34
:1016B000F2E78F16FBE09F0609F040C088249924CA
:1016C0002091AC013091AD012F5F3F4F3093AD01C0
:1016D0002093AC018091AA019091AB010196909367
:1016E000AB018093AA01832F9927682F8EE090E0A9
:1016F0000E94E42A8091AC019091AD019070682F16
:101700008FE090E00E94E42A8091AA019091AB01C1
:10171000892F9927682F8AE090E00E94E42A80911F
:10172000AA019091AB019070682F8BE090E00E942D
:10173000E42A84E190E00E94A5168C010E94626672
:101740000E948E6C8091D901882309F005CE0E94F9
:10175000886102CE1F920F920FB60F9211248F93C1
:101760009F93EF93FF93809107018823E1F4809189
:10177000CA019091CB0101969093CB018093CA014D
:10178000FC01EC59FB4FE081ED3019F08A3A9105EC
:1017900039F41092CB011092CA0181E080930701C5
:1017A000E093C60004C01092CB011092CA01FF91D1
:1017B000EF919F918F910F900FBE0F901F901895F2
:1017C0001F920F920FB60F9211242F933F934F93B6
:1017D0005F936F937F938F939F93AF93BF93CF93B9
:1017E000EF93FF9390E08091B001813029F48091D4
:1017F000C6008093CE00CCC08091B001823029F425
:101800008091C6008093B803C3C08091C6008093C6
:10181000C2015091D0015A3A10F09093D1018091B9
:10182000C2018D3009F065C08091D101823009F08C
:1018300060C09093D101852F992788549C4FFC015B
:10184000329740812091CC013091CD01241B310988
:10185000DC0111978C91281B3109C9019F7090936D
:10186000CD018093CC0146E0969587954A95E1F7A6
:10187000982F935C9093CE012F733070235C20934C
:10188000CF018081981729F48C91281711F491E0E9
:1018900006C090E08091BF018F5F8093BF01C0912F
:1018A000C101CC2309F074C0992309F471C081E00F
:1018B0008093C101580F5093BE015150E52FFF276F
:1018C000E854FC4F8DE080838091BA03823509F0A3
:1018D0005FC00E94961F88E190E02CE00FB6F8945C
:1018E000A895809360000FBE20936000C093D8013C
:1018F0004FC02091D101822F992781309105F9F0B5
:10190000823091051CF4892B21F040C0029711F11F
:101910003DC08091C201833239F48091C101882396
:1019200019F481E08093D1018091C2018093B803C2
:1019300081E08093D0018091C201992722C02F5F5E
:101940002093D101E52FFF27E854FC4F8091C2017D
:10195000808309C0E52FFF27E854FC4F8091C20126
:1019600080835A3A20F45F5F5093D00102C01092F6
:10197000D1012091C2018091CC019091CD01820FC3
:10198000911D9093CD018093CC0102C01092D101A2
:10199000FF91EF91CF91BF91AF919F918F917F91E7
:1019A0006F915F914F913F912F910F900FBE0F90CC
:1019B0001F901895AC01A0E0B0E09D01A817B907F1
:1019C00048F4E4E6F4E08191280F311D1196A41744
:1019D000B507C8F33F70FD01EC59FB4FC90156E054
:1019E000969587955A95E1F7835C80831196FD0162
:1019F000EC59FB4F2F733070822F835C8083AB597F
:101A0000BB4F8DE08C93109207018091640480930A
:101A1000C6000895A0E0B0E0E0E1FDE00C948B7812
:101A20002C859D850E85BB2483E2809364049F5999
:101A3000909365042093660433E0E32EF12C002399
:101A400009F49EC0CF84D888BE016D5E7F4FA989FE
:101A5000BA890150109709F493C01097B9F0F601B4
:101A6000EB0DF11DB3949081119791F4002349F18E
:101A7000FB016E5F7F4FDB01C080D1806E5F7F4FC7
:101A80000D90BC91A02DBB24015002C090E019C064
:101A90001097B9F0F601EB0DF11DB3944081119749
:101AA00091F4002341F1FB016E5F7F4FDB01C080A9
:101AB000D1806E5F7F4F0D90BC91A02DBB24015053
:101AC00002C040E018C01097B1F0F601EB0DF11D17
:101AD000B3941081119781F4002371F0FB013296C9
:101AE000DB01CD90DC90BF016E5F7F4FA081B181A3
:101AF000BB24015001C010E0F701EC59FB4F892FC6
:101B000086958695835C80830894E11CF11CF7011F
:101B1000EC59FB4F892F99278370907024E0880F30
:101B2000991F2A95E1F755279A0194E03695279554
:101B30009A95E1F7822B835C80830894E11CF11C69
:101B4000F701EC59FB4F4F705070440F551F440F75
:101B5000551F812F992726E0969587952A95E1F7BD
:101B6000842B835C80830894E11CF11CF701EC5901
:101B7000FB4F1F73135C10830894E11CF11C6ACFA8
:101B8000C7010E94DA0CE9E00C94A778A3E07A2F51
:101B90004091BE014650442309F458C0E72FFF2767
:101BA000E854FC4F80818D537F5FE72FFF27E85477
:101BB000FC4F20812D537F5FE72FFF27E854FC4F18
:101BC00030813D537F5FE72FFF27E854FC4F608152
:101BD0006D537F5F9927880F991F880F991F522F88
:101BE00052955F70582B822F99278F709070F4E078
:101BF000880F991FFA95E1F7232F26952695282B14
:101C0000832F992783709070E6E0880F991FEA95DB
:101C1000E1F7682B41504F3FC9F0EA2FFF27E85406
:101C2000FC4F5083AF5F41504F3F81F0EA2FFF27B9
:101C3000E854FC4F2083AF5F41504F3F39F0EA2F0B
:101C4000FF27E854FC4F6083AF5FA5CF8BEB93E099
:101C50009093BD018093BC01A350A093BB01089554
:101C6000A2E0B0E0E6E3FEE00C9491788091C1013F
:101C7000882309F457C40E94C60D8091B9038236A7
:101C800009F023C38091BA0399278037910509F49D
:101C9000AFC081379105C4F48A36910509F480C23A
:101CA0008B36910544F48B34910571F1863691059C
:101CB00009F45FC10AC38D36910509F469C08E36F7
:101CC000910509F44DC001C38437910541F1853771
:101CD00091054CF48137910509F491C08337910542
:101CE00009F4DFC0F2C28737910509F41BC28837B7
:101CF00091052CF48537910509F4D7C1E6C28937DF
:101D0000910509F46DC1E1C2E091BC01F091BD0102
:101D1000808191819093900180938F01D6C28091B0
:101D2000BE01A091BC01B091BD01853140F080E1C0
:101D3000E3E9F3E00D9001928A95E1F70DC08D91F2
:101D40009D910D90BC91A02D80939303909394034B
:101D5000A0939503B093960380EF8093B9014BC095
:101D6000809107018823E1F38DE490E09F938F93A6
:101D70008DE296E09F938F9381E08F938F938EE413
:101D80008F930E940A0D8DB79EB707968DBF9DC297
:101D9000A091BC01B091BD011C91113081F48DE482
:101DA000EDE2F6E00D9001928A95E1F70E94E62BB4
:101DB000198380918F038F7E80938F0301C01982D6
:101DC000809107018823E1F381E090E09F938F9356
:101DD000CE0101969F938F9381E08F938F938DE433
:101DE0008F930E940A0DADB7BEB71796ADBF6DC2F7
:101DF00081E08093C4018FEF8093050166C2E0917A
:101E0000BC01F091BD01E0818E2F8A508A3058F4D8
:101E10008983882311F481E003C0863010F085E0C7
:101E2000898361E00EC08E2F84518A3070F48983DB
:101E3000882311F481E003C0863010F085E08983A7
:101E400060E089810E94662C12C0E983EF3F19F49B
:101E50000E94492C89838981882311F481E003C081
:101E6000863010F085E0898389810E94FA2A80916A
:101E700007018823E1F387E790E09F938F9385EB39
:101E800095E09F938F9381E090E09F938F93CE0195
:101E900001969F938F9382E08F9381E08F9381E5EA
:101EA00077C12091BC013091BD01D9018C91815045
:101EB000853008F045C0F9018181883509F040C0BE
:101EC000809169028823E1F52F5F3F4F87E7E5EBBB
:101ED000F5E0D9010D9001928A95E1F7F90182911F
:101EE0000E94632B8091F6059927AA27BB27BC0186
:101EF000CD0124EC39E040E050E00E94F377DC01B2
:101F0000CB018093870190938801A0938901B093BE
:101F10008A018091F7059927AA27BB27BC01CD012B
:101F20000E94F377DC01CB018093830190938401BD
:101F3000A0938501B09386010E94492C898301C03A
:101F40001982809107018823E1F381E090E09F935B
:101F50008F93CE0101969F938F9381E08F938F9300
:101F600083E58F930E940A0D8DB79EB707968DBFAC
:101F700026C0E091BC01F091BD01E0818E2F81501F
:101F8000853018F48E2F0E94FA2A0E94492C8983EA
:101F9000809107018823E1F381E090E09F938F9384
:101FA000CE0101969F938F9381E08F938F9386E468
:101FB0008F930E940A0DADB7BEB71796ADBF809143
:101FC0006902882329F46EE670E089810E944B340F
:101FD00080E00E94D7068091DC050E94757375C170
:101FE000E091BC01F091BD018081992787FD90951A
:101FF0009093FF068093FE068181992787FD909537
:1020000090930107809300078281992787FD90951F
:1020100090930307809302078381992787FD90950A
:1020200090930507809304078481992787FD9095F5
:1020300090930707809306078581992787FD9095E0
:1020400090930907809308078681992787FD9095CB
:1020500090930B0780930A078781992787FD9095B6
:1020600090930D0780930C078085992787FD9095A5
:1020700090930F0780930E078185992787FD909590
:1020800090931107809310078285992787FD90957B
:1020900090931307809312078385992787FD909566
:1020A000909315078093140710C1E091BC01F09143
:1020B000BD0180810E948D318A83882319F481E0DB
:1020C000898301C01982809107018823E1F388E0A8
:1020D00090E09F938F938BE796E09F938F9321E0FF
:1020E00030E03F932F938091BC019091BD019F936D
:1020F0008F933F932F93CE0102969F938F933F939D
:102100002F93CE01820F931F9F938F9384E08F9321
:1021100081E08F9385E58F930E940A0DEDB7FEB79E
:1021200073963CC08091BB01893008F4CEC02091E9
:10213000BC013091BD012F5F3F4F88E0ABE7B6E0B7
:10214000F90101900D928A95E1F7D9018E910E94D3
:10215000E3308A83882319F481E0898301C01982DE
:10216000809107018823E1F321E030E03F932F9332
:10217000CE0102969F938F933F932F93CE01820FB0
:10218000931F9F938F9382E08F9381E08F9387E5D6
:102190008F930E940A0DEDB7FEB73B96EDBF95C039
:1021A00080916902882309F090C00E942873898376
:1021B000823019F0843009F088C020E430E0F894CF
:1021C0008091C1008F738093C1008091C9008F738B
:1021D0008093C9008091C100877E8093C100809167
:1021E000C900877E8093C9008091C80087FF03C023
:1021F0008091CE00F9CF8091C00087FF03C080910D
:10220000C600F9CFE091BC01F091BD01E081E13061
:1022100021F482E08093B0012EC0E43611F421E86D
:1022200030E081E08093B001832F99278093CD0027
:102230002093CC008091CD008093C5008091CC008C
:102240008093C4008091CA008F7D8093CA008091E2
:10225000CA008F7E8093CA008091C9008B7F8093D3
:10226000C9008091CA0084608093CA008091CA002E
:1022700082608093CA008091CA00877F8093CA00E1
:102280008091C200877F8093C2008091C9008E7FB9
:102290008093C9008091C10088618093C1008091C2
:1022A000C90088618093C9008091C10080688093D3
:1022B000C1008091C90080688093C90010926E00AF
:1022C00010926F001092700078948091BA03992751
:1022D0008436910509F4BBC085369105ACF481368E
:1022E000910509F46FC0823691052CF48B34910569
:1022F00009F45DC00FC18236910509F470C08336C0
:10230000910509F47FC006C18C36910509F4EDC032
:102310008D3691054CF48736910509F4F8C088365E
:10232000910509F4B2C0F6C08437910529F08637CB
:10233000910509F4E8C0EEC08091BE01A091BC01F6
:10234000B091BD01803140F080E1E3E9F3E00D9010
:1023500001928A95E1F70DC08D919D910D90BC91F0
:10236000A02D8093930390939403A0939503B0932F
:102370009603809107018823E1F31F928091040165
:102380008F9384E58F930E940A0D8AEF8093B901A1
:102390008FEF8093050180EA9FE00E94A51690933D
:1023A000B2018093B1010F900F900F90B3C0E091F4
:1023B000BC01F091BD018081918190939001809347
:1023C0008F01A8C0E091BC01F091BD018081809394
:1023D0000601803298F08FE1809306010FC0A09132
:1023E000BC01B091BD018BE0EBEAF3E00D900192EE
:1023F0008A95E1F78091B403809350058FEF809325
:10240000050188C08091B5019091B601892B89F4AE
:10241000E091BC01F091BD01E081EE2351F08AE032
:10242000E89FC00111240E94A51690938603809313
:102430008503E091BC01F091BD0190818AE0989FF5
:10244000C00111249093B6018093B50115C08FEFA0
:1024500080930501E091BC01F091BD0190818AE07B
:10246000989FC00111249093B8018093B701892BE4
:1024700019F081E08093C60180EA9FE00E94A516D2
:102480009093B2018093B10145C08FEF8093050115
:10249000E091BC01F091BD01908197FD08C082E000
:1024A0008093C3011092B4011092B3011AC09095A9
:1024B00080911B02892B80931B0291818AE0989F57
:1024C000C00111249093B4018093B30184E0809300
:1024D000C30180EA9FE00E94A5169093B201809309
:1024E000B10181E08093C70115C08FEF8093050192
:1024F000E091BC01F091BD01808180931C0281E0DC
:102500008093C80107C081E08093C50103C081E0CA
:102510008093C9011092C1011092BD011092BC01BB
:102520001092BB01E3E0CE5F0C94AD78982F8091C0
:10253000C00085FFFCCF9093C60008950F931F93B2
:1025400088E18093C1008091C00082608093C000C8
:102550008091C10080688093C1008091C100806437
:102560008093C10000E010E00093C5008AE290E093
:102570008093C4008091B7019091B8010E94A51684
:1025800090938803809387038CED90E00E94A516BA
:102590009093B7038093B6031092890386E58093E6
:1025A0008A0382E080938D038BE080938B031092EB
:1025B0008C031093BD010093BC011092BB011F91CD
:1025C0000F910895A0E1B0E0E8EEF2E10C948E786E
:1025D00080910701882309F4C1C28091B1019091D3
:1025E000B2010E94AE16882361F01092B4011092DD
:1025F000B3011092B8011092B7011092B601109277
:10260000B5018091B3019091B401892B41F0809183
:102610006204909163040E94AE16882329F480918D
:10262000C701882309F460C080910701882309F459
:102630005BC08091C30104E615E08430A8F00E94DD
:10264000AC1F80E590E09F938F931F930F9381E0E1
:102650008F938F9388E48F930E940A0D2DB73EB716
:10266000295F3F4F2DBF34C010921D0280E194E0DE
:102670009F938F938FE99FE19F938F93E0917503D1
:10268000F0917603099584E190E09F938F931F93D7
:102690000F9381E090E09F938F9383EC91E09F9361
:1026A0008F9382E08F9381E08F9388E48F930E94D1
:1026B0000A0D8091C301982F8F5F8093C3012DB7BE
:1026C0003EB7215F3F4F2DBF943010F01092C301F1
:1026D0008091B3019091B4010E94A5169093630478
:1026E000809362041092C7018091C801882351F140
:1026F00080910701882331F10E94AC1F80E590E0B2
:102700009F938F9384E695E09F938F9321E030E031
:102710003F932F9380E291E09F938F933F932F936A
:102720008CE192E09F938F9383E08F9381E08F936E
:102730008CE48F930E940A0D1092C8018DB79EB74A
:102740000F968DBF8091C5018823D1F0809107013C
:102750008823B1F08AE090E09F938F9389E893E01B
:102760009F938F9381E08F938F9386E58F930E9441
:102770000A0D1092C5012DB73EB7295F3F4F2DBFFF
:102780008091C9018823D9F0809107018823B9F08D
:102790008BE090E09F938F938BEA93E09F938F93CE
:1027A00081E08F93809104018F9387E48F930E943F
:1027B0000A0D1092C9018DB79EB707968DBF809103
:1027C000B6039091B7030E94AE16882309F461C046
:1027D00080910701882309F45CC08091D105992775
:1027E000880F991F880F991F7C010027F7FC00951F
:1027F000102F8091C4029091C502A091C602B091A1
:10280000C702BC01CD01A80197010E9467783093EF
:10281000A4032093A3038091BC029091BD02A091D8
:10282000BE02B091BF02BC01CD01A80197010E9478
:1028300067783093A6032093A50380914902809383
:10284000A703809148028093A80388E090E09F93BB
:102850008F9383EA93E09F938F9381E08F9383E03C
:102860008F938BE68F930E940A0D8091A9032DB759
:102870003EB7295F3F4F2DBF853018F086E080932B
:10288000A90383E690E00E94A5169093B703809376
:10289000B6038091B7019091B801892B41F08091E6
:1028A0008703909188030E94AE16882321F48091BB
:1028B000C601882339F180910701882319F10E940C
:1028C000353382E490E09F938F938EE095E09F9361
:1028D0008F9381E08F938F9384E48F930E940A0DEE
:1028E0001092C6018DB79EB707968DBF8091B70134
:1028F0009091B801009731F00E94A516909388033B
:10290000809387038091B5019091B601892B09F4DA
:10291000B8C080918503909186030E94AE168823EB
:1029200009F4AFC080910701882309F4AAC08091FF
:10293000D1059927880F991F880F991F7C010027BF
:10294000F7FC0095102F8091C4029091C502A091D0
:10295000C602B091C702BC01CD01A80197010E9437
:10296000677830937803209377038091BC0290912D
:10297000BD02A091BE02B091BF02BC01CD01A80171
:1029800097010E94677830937A032093790320910E
:10299000AD073091AE074091AF075091B007DA0113
:1029A000C90163E0880F991FAA1FBB1F6A95D1F761
:1029B000820F931FA41FB51F820F931FA41FB51F63
:1029C00020914301309144014091450150914601CD
:1029D000BC01CD010E94677830937C0320937B0378
:1029E00080918C0290918D02A0918E02B0918F0205
:1029F00049E0B595A795979587954A95D1F7809326
:102A00007D038091880290918902A0918A02B09101
:102A10008B0239E0B595A795979587953A95D1F7AB
:102A200080937E038091940290919502A0919602EA
:102A3000B091970229E0B595A795979587952A9526
:102A4000D1F780937F038EE090E09F938F9387E789
:102A500093E09F938F9381E08F938F9383E48F9381
:102A60000E940A0D8091B5019091B6010E94A516B1
:102A700090938603809385032DB73EB7295F3F4F20
:102A80002DBF809106018F3F71F1992704E0880FD7
:102A9000991F0A95E1F7805F9D4F40E150E0BC012E
:102AA000CE0101960E94467680E190E09F938F933D
:102AB000CE0101969F938F9381E090E09F938F9337
:102AC00086E091E09F938F9382E08F9381E08F93D4
:102AD00081E48F930E940A0D8FEF809306018DB7DA
:102AE0009EB70B968DBF809150058823D1F08091C1
:102AF00007018823B1F081E090E09F938F9380E5F8
:102B000095E09F938F9381E08F938F9382E48F93CF
:102B10000E940A0D109250052DB73EB7295F3F4F16
:102B20002DBF8091C4018823C9F0809107018823BB
:102B3000A9F084E390E09F938F9384EE96E09F93B7
:102B40008F9381E08F938F9380E58F930E940A0D7E
:102B50001092C4018DB79EB707968DBFE6E0C05FA7
:102B60000C94AA781F920F920FB60F9211242F93F4
:102B70003F935F936F937F938F939F93AF93BF9395
:102B8000EF93FF9320E08091D901882329F0809171
:102B9000D90181508093D90180915503882319F080
:102BA0008150809355038091E10181508093E10130
:102BB0008F3F09F05BC089E08093E1018091DF01E4
:102BC0009091E00101969093E0018093DF01809164
:102BD0000F018F5F817080930F01882319F481E0CA
:102BE0008093DE01349903C081E08093E2018091FB
:102BF000DA019091DB01892B21F18091DA0190912A
:102C0000DB010B9750F08091DA019091DB010A977C
:102C10009093DB018093DA0104C01092DB011092E3
:102C2000DA018091DA019091DB0120910801309165
:102C3000090182239323892B11F021E008C020E0B1
:102C400006C08FEF9FEF9093090180930801809158
:102C50000201222331F08A3011F45A9A07C0479AB0
:102C600005C08A3011F45A9801C047988091E2015A
:102C7000882309F45AC020919C01222309F055C0F1
:102C800080919D0783FF51C086B19927FC01E071B7
:102C9000F07084FF13C08091DC019091DD010196FA
:102CA0009093DD018093DC018091DC019091DD0146
:102CB000895E9340D0F12093E20137C08091DC011E
:102CC0009091DD01892B69F18091DC019091DD010A
:102CD0008A56914030F58091DC019091DD0169E2E6
:102CE00070E00E941E788091DC019091DD01860FDA
:102CF000971F9093DD018093DC018091DC0190911E
:102D0000DD010B9750F08091DC019091DD010A9775
:102D10009093900180938F0104C0F0939001E09311
:102D20008F011092DD011092DC01FF91EF91BF91B4
:102D3000AF919F918F917F916F915F913F912F9173
:102D40000F900FBE0F901F9018952091DF013091CA
:102D5000E001280F391FC901019608952091DF0174
:102D60003091E001821B930B892F992786958074FF
:102D700090700895CF93DF930E94A516EC01CE01C9
:102D80000E94AE168823D9F3DF91CF910895CF9397
:102D9000DF930E94A516EC0109C0809110018823E1
:102DA00029F0909310018FEC80937A00CE010E945D
:102DB000AE16982F882389F3DF91CF9108959FB79E
:102DC000F8945F983E9A469A8091B0008F708093F5
:102DD000B0008091B00083608093B0008091B1001A
:102DE0008B738093B1008091B1008B608093B100B0
:102DF0001092B2008FEF8093B3008091B000806892
:102E00008093B000809170008A7F809370008091E1
:102E100070008260809370009FBF08958AE090E008
:102E20000E94A5169093E8018093E70182E085BD9A
:102E300083EA84BD17BC84EB88BD86E086BD8091A3
:102E40006E00816080936E000895A0E0B0E0EBE238
:102E5000F7E10C948D788091EC05E82FFF27E75B74
:102E6000FE4F9681D08080910E01A92FBB27A7FD30
:102E7000B095CB2FDB2F813009F0DDC02091C4024B
:102E80003091C5024091C6025091C702BD01CE01EA
:102E90000E94F37797FF04C061587F4F8F4F9F4F79
:102EA0007B018C01F7E015950795F794E794FA9567
:102EB000D1F78D2D992787FD9095A92FB92F2091B6
:102EC000BC023091BD024091BE025091BF02BC01D4
:102ED000CD010E94F37797FF04C061587F4F8F4F59
:102EE0009F4FE7E09595879577956795EA95D1F798
:102EF000F801E701C61BD70BE80BF90B20913F0344
:102F000030914003C90153E0880F991F5A95E1F7AA
:102F1000821B930BAA2797FDA095BA2FC81BD90B2C
:102F2000EA0BFB0B8091E3059927AA27BB27BC017D
:102F3000CD019E01AF010E94F37797FF04C061505D
:102F40007E4F8F4F9F4FFC01EB0149E0F595E795D0
:102F5000D795C7954A95D1F780916E01992736E0AC
:102F6000880F991F3A95E1F740910C0150910D019E
:102F70002091EB053327841B950BB9010E94327811
:102F800080910C0190910D01860F971F90930D0178
:102F900080930C0180910C0190910D0197FD0F968B
:102FA00024E0959587952A95E1F79093D501809334
:102FB000D40180911E0680FF07C08091D4019091BA
:102FC000D5018C0F9D1F06C08091D4019091D50131
:102FD0008C1B9D0B9093D5018093D4018091E405C7
:102FE000282F3327220F331F220F331F8091D40144
:102FF0009091D501821793077CF08091E505282FE9
:103000003327220F331F220F331F8091D401909159
:10301000D5012817390724F43093D5012093D40122
:1030200080910201843108F4C2C080910E018F5F4B
:1030300080930E01BEC02091BC023091BD02409130
:10304000BE025091BF02BD01CE010E94F37797FFEF
:1030500004C061587F4F8F4F9F4F7B018C01C7E0A9
:1030600015950795F794E794CA95D1F78D2D992773
:1030700087FD9095A92FB92F2091C4023091C502E8
:103080004091C6025091C702BC01CD010E94F37766
:103090009B01AC0197FF04C021583F4F4F4F5F4F3A
:1030A000B7E05595479537952795BA95D1F72E0DE9
:1030B0003F1D401F511F8091E7059927AA27BB2775
:1030C000BC01CD010E94F37797FF04C061507E4F91
:1030D0008F4F9F4FFC01EB01A9E0F595E795D79540
:1030E000C795AA95D1F780916D01992776E0880F51
:1030F000991F7A95E1F740910A0150910B012091B7
:10310000EB053327841B950BB9010E94327880911F
:103110000A0190910B01860F971F90930B018093EA
:103120000A0180910A0190910B0197FD0F9664E0CE
:10313000959587956A95E1F79093D3018093D20195
:1031400080911E0681FF07C08091D2019091D3012A
:103150008C0F9D1F06C08091D2019091D3018C1BD2
:103160009D0B9093D3018093D2018091E805282F85
:103170003327220F331F220F331F8091D2019091EA
:10318000D301821793077CF08091E905282F33271C
:10319000220F331F220F331F8091D2019091D30150
:1031A0002817390724F43093D3012093D2011092C9
:1031B0000E01E7E0CDB7DEB70C94A9781F920F920D
:1031C0000FB60F9211242F933F934F935F938F93DA
:1031D0009F93EF93FF93809102019091E3018431DB
:1031E00008F04CC0992309F01CC18091B00086FF03
:1031F00024C08091B0008F7B8093B0008091D40177
:103200009091D50187559E4F9093D7018093D60119
:1032100025E08D3D920718F08CED95E005C08757AD
:10322000914030F487E791E09093D7018093D601E5
:103230008091D6019091D701BAC08091B00080648E
:103240008093B0008091EA05282F33278DED96E01A
:10325000289FA001299F500D389F500D1124CA01AD
:103260002091E4013091E501821B930B9093D701EB
:103270008093D60181E080930E01D0C0992309F09C
:10328000D0C08091B00086FF97C08091B0008F7B46
:103290008093B000E091E601EE23F1F48091EA051D
:1032A000282F33278DED96E0289FA001299F500DF0
:1032B000389F500D1124CA012091E4013091E5019D
:1032C000821B930B9093D7018093D6011092E50156
:1032D0001092E401469AA2C089EA93E09093D70144
:1032E0008093D6018E2F992783309105D9F08430B1
:1032F000910534F48130910549F0029761F020C0C6
:103300008430910591F0059799F01AC08091D4010D
:103310009091D50104C08091D2019091D30187553D
:103320009E4F1DC08091790705C08091520702C051
:10333000809182079927880F991F880F991FEFCFD7
:10334000FF27EE0FFF1FEC51F94F20813181220F33
:10335000331F8091D6019091D701820F931F9093D4
:10336000D7018093D6018091D6019091D70155E085
:103370008D3D950718F08CED95E005C0875791407D
:1033800030F487E791E09093D7018093D6012091A4
:10339000D6013091D7012C5B30403093D701209378
:1033A000D6018091E4019091E501820F931F9093E3
:1033B000E5018093E40132C08091B0008064809385
:1033C000B0008CEB90E09093D7018093D601809170
:1033D000E4019091E50184549F4F9093E50180931F
:1033E000E4018091D801882321F080916A0288232A
:1033F00021F48091D801823011F4469801C0469A98
:103400008091E6018F5F8093E6019091EA0598171D
:1034100028F481E080930E011092E60181E0809310
:10342000E3012091D6013091D70141E02F373407D5
:1034300030F08FEF8093B3002F5F30400FC02F3FED
:103440003105C9F0C0F0A9014F5F50404F37510519
:1034500050F480E88093B300205830403093D70177
:103460002093D60112C08FEF8093B3005093D70101
:103470004093D6010AC08091D6018093B300109288
:10348000D7011092D6011092E301FF91EF919F9125
:103490008F915F914F913F912F910F900FBE0F90A1
:1034A0001F90189510927C008FEC80937A000895FD
:1034B000CF93DF931092ED0183E090E00E94DC2A2D
:1034C000C82FDD27C531D10508F02A97C7BD84E68E
:1034D00090E00E94C71680911401909115018052CE
:1034E000934010F4C0E0D0E0CA3FD105F8F4C7BD66
:1034F00082E390E00E94C71685E294E09F938F9349
:1035000086E992E19F938F93E0917503F0917603A2
:10351000099580911401909115010F900F900F90D3
:103520000F908052934010F02196DECFC09361053A
:103530006C2F83E090E00E94E42A8091C20580FF16
:103540000AC0809161058A508B3E28F080918E03DD
:10355000806480938E03C7BD8CE291E00E94C71601
:10356000DF91CF910895EF92FF921F93CF9310E0D8
:1035700080ED97E00E94A5167C01CCE8133019F489
:10358000CB3008F0C9E010E08091FD019091FE0180
:103590008C5F934024F48091130181500AC0809184
:1035A000FD019091FE018750944034F08091130109
:1035B0008F5F8093130101C011E08091FB01909116
:1035C000FC018C5F934024F48091120181500AC069
:1035D0008091FB019091FC018750944034F08091E0
:1035E00012018F5F8093120101C01F5F8091F9016A
:1035F0009091FA018C5F934024F4809111018150E5
:103600000AC08091F9019091FA0187509440C4F06A
:10361000809111018F5F8093110113C087E294E0C4
:103620009F938F9386E992E19F938F93E091750327
:10363000F091760309950F900F900F900F905FC057
:103640001F5F82E180932802809122028E7F809307
:10365000220285EA8093BC00809113018A3040F4F5
:1036600080918E03816080938E038AE080931301A2
:1036700080911301863F40F080918E03816080939A
:103680008E0385EF80931301809112018A3040F4FC
:1036900080918E03826080938E038AE08093120172
:1036A00080911201863F40F080918E03826080936A
:1036B0008E0385EF80931201809111018A3040F4CE
:1036C00080918E03846080938E038AE08093110141
:1036D00080911101863F40F080918E038460809339
:1036E0008E0385EF8093110180912802882339F0A1
:1036F000C7010E94AE16882309F090CFF5CF109233
:1037000010018FEC80937A00809110018823E1F3FF
:10371000CA3020F48AE090E00E94C716C15009F038
:103720002DCF86E490E00E94C716CF911F91FF90A5
:10373000EF9008951F920F920FB60F921124EF92FF
:10374000FF920F931F932F933F934F935F936F932A
:103750007F938F939F93AF93BF93EF93FF9380914A
:103760000602282F3327442755278F5F80930602B0
:10377000F9012231310508F0B4C3E25CFF4F0C942B
:10378000B978809178009091790046C08091780056
:10379000909179002CC1809178009091790090935C
:1037A00009028093080257C18091CD029091CE0208
:1037B0002091780030917900821B930B90935205F1
:1037C0008093510580915105909152059093130279
:1037D000809312025EC180917800909179002091CF
:1037E000CF023091D002821B930B9093600580939F
:1037F0005F0580915F05909160059093150280931D
:10380000140271C380910C0290910D0220917800F6
:1038100030917900820F931F90930D0280930C02D8
:1038200081E062C380910A0290910B02209178009E
:1038300030917900820F931F90930B0280930A02BC
:1038400084E052C380911E0190911F019C01220FC0
:10385000331F280F391F809178009091790063E021
:1038600070E00E941E78260F371F369527953695F3
:10387000279530931F0120931E0185E035C3809169
:103880007800909179004091C9025091CA02841B3E
:10389000950B9093F4018093F3018091F301909143
:1038A000F401029704F122E04E3E520784F4209185
:1038B00007022B5F209307022550809135029091DB
:1038C0003602845F914018F4215F209307028091B3
:1038D0000702853684F14F5F5F4F5093CA024093D1
:1038E000C902845626C08091F3019091F4018F5F44
:1038F0009F4F0CF532E047325307ECF0209107025E
:103900002550209307022B5F80913502909136025B
:10391000845F914018F42F50209307028091070292
:103920008C394CF4415050405093CA024093C90224
:103930008C598093070281E08093F2018091780096
:103940009091790090935805809357058091F301E9
:103950009091F4019C01442737FD4095542F8091AC
:10396000840290918502A0918602B0918702820F15
:10397000931FA41FB51F8093840290938502A09388
:103980008602B09387022091840230918502409193
:1039900086025091870257FF04C021503C4F4F4F81
:1039A0005F4F6AE055954795379527956A95D1F70A
:1039B0008091840290918502A0918602B091870245
:1039C000821B930BA40BB50B80938402909385020A
:1039D000A0938602B09387022EC180910A02909133
:1039E0000B022091780030917900820F931F909301
:1039F0000B0280930A021092050278C280910201A4
:103A00008A3071F4809178009091790020910802B9
:103A100030910902820F931F01969695879517C0E2
:103A20004091080250910902843158F020917800A9
:103A300030917900240F351F8FEF97E0821B930B95
:103A400006C08091780090917900840F951F909323
:103A5000FA018093F90186E047C28091CD029091EE
:103A6000CE022091780030917900821B930B9093C5
:103A700052058093510580915105909152052091F6
:103A8000120230911302820F931F9093F8018093DA
:103A9000F70187E029C28091780090917900209108
:103AA000CF023091D002821B930B909360058093DC
:103AB0005F0580915F05909160052091140230911F
:103AC0001502820F931F9093F6018093F5010BC2AC
:103AD00020910C0230910D02809178009091790034
:103AE000280F391F30930D0220930C0280910201A0
:103AF0008A3019F4220F331F04C0220F331F220F04
:103B0000331F30930D0220930C0220910C02309150
:103B10000D02C90137FD079603E0959587950A9533
:103B2000E1F79093FE018093FD0180910E02909148
:103B30000F02820F931F97FD01969595879590939D
:103B40000F0280930E022091D9023091DA02821B7B
:103B5000930B90931D0180931C01209103023091DF
:103B6000040280911C0190911D01280F391F37FF1D
:103B700002C02F5F3F4F3595279530930402209365
:103B800003024ECE20910A0230910B028091780000
:103B900090917900280F391F30930B0220930A026D
:103BA000809102018A3019F4220F331F04C0220FC2
:103BB000331F220F331F30930B0220930A022091F0
:103BC0000A0230910B02C90137FD0796F3E0959583
:103BD0008795FA95E1F79093FC018093FB01809122
:103BE000100290911102820F931F97FD01969595F7
:103BF000879590931102809310022091D702309103
:103C0000D802821B930B90931B0180931A01209181
:103C100001023091020280911A0190911B01280F3C
:103C2000391F37FF02C02F5F3F4F359527953093DF
:103C300002022093010283E057C11092060281E044
:103C4000809310018091E9019091EA01019690938F
:103C5000EA018093E9018091780090917900909336
:103C60001501809314018091140190911501AA27E8
:103C7000BB272091160230911702409118025091F3
:103C80001902280F391F4A1F5B1F20931602309319
:103C90001702409318025093190280911A028F5F05
:103CA00080931A02823108F41EC18091160190910E
:103CB0001701A0911801B09119017C018D0163E0F9
:103CC000EE0CFF1C001F111F6A95D1F7E81AF90AC4
:103CD0000A0B1B0BE20EF31E041F151F8091ED0152
:103CE000992787FD9095A92FB92FBC01CD0126EC0E
:103CF00034E240E050E00E94F377DC01CB01E81AA7
:103D0000F90A0A0B1B0BD801C7010496A11DB11DAE
:103D1000B7FF05C0D801C7010B96A11DB11D23E057
:103D2000B595A795979587952A95D1F78093160114
:103D300090931701A0931801B09319018091590530
:103D400090915A057C010027F7FC0095102F809177
:103D5000160190911701A0911801B0911901E81A6C
:103D6000F90A0A0B1B0BE0926402F09265020093C1
:103D70006602109367022091EE013091EF014091AD
:103D8000F0015091F10157FF04C0215F3F4F4F4FA9
:103D90005F4F84E055954795379527958A95D1F7DC
:103DA0008091EE019091EF01A091F001B091F101AD
:103DB000821B930BA40BB50B8093EE019093EF0144
:103DC000A093F001B093F1018091EE019091EF0189
:103DD000A091F001B091F1018E0D9F1DA01FB11FA8
:103DE0008093EE019093EF01A093F001B093F10165
:103DF0008091EE019091EF01A091F001B091F1015D
:103E0000B7FF03C00F96A11DB11D14E0B595A7958E
:103E1000979587951A95D1F72091640230916502A4
:103E2000281B390BC90137FF03C0309521953F4F3F
:103E3000AC01F3E0440F551FFA95E1F72138310545
:103E4000C4F08091EB019091EC019C01E3E0220F22
:103E5000331FEA95E1F7281B390B240F351F37FF75
:103E600002C0295F3F4F73E0359527957A95E1F7BA
:103E700017C08091EB019091EC019C0165E0220F4D
:103E8000331F6A95E1F7281B390B240F351F37FFC5
:103E900002C0215E3F4F45E0359527954A95E1F7F1
:103EA0003093EC012093EB01809116029091170260
:103EB000A0911802B0911902B7FF03C00196A11D8D
:103EC000B11DB595A7959795879580931602909308
:103ED0001702A0931802B093190289E080931A0286
:103EE00002C01092060282E08093050280910502D2
:103EF00080937C0080910602882319F08FEC8093D8
:103F00007A00FF91EF91BF91AF919F918F917F9137
:103F10006F915F914F913F912F911F910F91FF9062
:103F2000EF900F900FBE0F901F90189590E2E4E66F
:103F3000F5E08FE49193815087FFFCCF0895909135
:103F40001D02903540F4E92FFF27EC59FA4F80838A
:103F50009F5F90931D020895AF92BF92CF92DF9220
:103F6000FF920F931F93CF93DF9320911B0220FFAB
:103F70000AC080911C02882311F0815002C08091F8
:103F8000200180931C0221FF0CC090911C028091A3
:103F90002001981719F410921C0203C09F5F9093A0
:103FA0001C02822F992780FF04C081FF02C010925B
:103FB0001C020E94961F80911C02282F33279FE924
:103FC000C92E9FE1D92EC0917503D09176038A3016
:103FD00098F481E180931D023F932F938EE594E046
:103FE0009F938F93DF92CF92FE0109952DB73EB735
:103FF0002A5F3F4F2DBF11C080E180931D023F9388
:104000002F9383E694E09F938F93DF92CF92FE01EC
:1040100009958DB79EB706968DBF20911C02822F01
:104020009927AA27BB27FC01419710F00C94E1289F
:10403000E05BFF4F0FE9C02E0FE1D02EC09175035A
:10404000D09176030C94B97810921D0288E694E022
:104050009F938F930FE91FE1DF92CF92FE010995A5
:1040600084E180931D020F900F900F900F9083E6D4
:1040700090E09F938F9386E590E09F938F931F929C
:104080001F92809102016AE00E941278892F99277D
:104090009F938F93809102010E94127899279F939A
:1040A0008F9388E794E09F938F93DF92CF92E09174
:1040B0007503F0917603099588E280931D02EDB7B0
:1040C000FEB73E96EDBF8EE296E09F938F930E94DF
:1040D000492C99279F938F938DE894E09F938F931A
:1040E000DF92CF92E0917503F0917603099580916C
:1040F0008F032DB73EB7285F3F4F2DBF84FF06C00B
:104100008CE380931D028BE994E0D2C090918E03E2
:10411000992351F08CE380931D02892F99279F9357
:104120008F9388EA94E03BC1909123029923B1F0E8
:104130008CE380931D02892F99279F938F938FEB98
:1041400094E09F938F931F930F93E0917503F091E9
:1041500076030995EDB7FEB7369679C4909144037E
:10416000992371F08CE380931D02892F99279F93E7
:104170008F9384ED94E09F938F931F930F93D9C4F3
:1041800080913D0190913E01069710F00C94EA2831
:104190008CE380931D0285EE94E0A5C780919D0776
:1041A0001FE9C12E1FE1D12EC0917503D091760376
:1041B00080FF6BC010921D02809164029091650295
:1041C000A0916602B0916702BC01CD0125E030E00C
:1041D00040E050E00E9467783F932F9382EF94E095
:1041E0009F938F93DF92CF92FE01099584E1809394
:1041F0001D028DB79EB706968DBF8091600290918B
:104200006102A0916202B0916302BC01CD0125E080
:1042100030E040E050E00E9467783F932F938FEFAB
:1042200094E09F938F93DF92CF92E0917503F0918A
:104230007603099588E280931D02EDB7FEB73696A6
:10424000EDBF80911401909115019F938F938CE0A5
:1042500095E09F938F93DF92CF92E0917503F09159
:10426000760309958CE380931D022DB73EB72A5F34
:104270003F4F2DBF87B599279F938F9389E195E095
:104280009F938F93DF92CF928EC010921D0286E291
:1042900095E09F938F93DF92CF92FE01099584E181
:1042A00080931D020F900F900F900F9085E395E083
:1042B0009F938F93DF92CF921AC710921D028EE3C5
:1042C00095E09F938F930FE91FE1DF92CF92FE015C
:1042D000099584E180931D020F900F900F900F902D
:1042E0008091C4029091C502A091C602B091C7020C
:1042F000B7FF04C081509C4FAF4FBF4FCAE0B59588
:10430000A79597958795CA95D1F7BF93AF939F933C
:104310008F938BE495E09F938F931F930F93E0917E
:104320007503F0917603099588E280931D02EDB73D
:10433000FEB73896EDBF8091BC029091BD02A0916E
:10434000BE02B091BF02B7FF04C081509C4FAF4F77
:10435000BF4FFAE0B595A79597958795FA95D1F750
:10436000BF93AF939F938F938AE595E09F938F932D
:104370001F930F93E0917503F091760309958CE3F9
:1043800080931D022DB73EB7285F3F4F2DBF809110
:104390005A0790915B079F938F9389E695E09F93CF
:1043A0008F931F930F93E0917503F0917603099516
:1043B0008DB79EB706968DBF0DC7E1E0FE2EC1E01A
:1043C000D0E006EE16E09F2D969584E1989FC001FF
:1043D000112480931D02F801828193819F938F9312
:1043E0002196DF93CF932197808191819F938F9323
:1043F000DF93CF9388E795E09F938F938FE99FE1B9
:104400009F938F93E0917503F091760309952DB7F3
:104410003EB7245F3F4F2DBF32E0F30E22960C5F74
:104420001F4F88E08F1578F6D5C610921D02809137
:10443000B705E82FFF27EE0FFF1FEC51F94F8081E2
:1044400091819F938F938091B605E82FFF27EE0F00
:10445000FF1FEC51F94F808191819F938F938AE8E0
:1044600095E09F938F93DF92CF92FE01099584E1AF
:1044700080931D02EDB7FEB73896EDBF8091B90568
:10448000E82FFF27EE0FFF1FEC51F94F808191813C
:104490009F938F938091B805E82FFF27EE0FFF1FA2
:1044A000EC51F94F8081918181589F4F9F938F9359
:1044B0008AE995E09F938F93DF92CF92E091750305
:1044C000F0917603099588E280931D022DB73EB7DF
:1044D000285F3F4F2DBF8091BB05E82FFF27EE0FD0
:1044E000FF1FEC51F94F8081918181589F4F9F931D
:1044F0008F938091BA05E82FFF27EE0FFF1FEC5135
:10450000F94F8081918181589F4F9F938F938AEAC1
:1045100095E09F938F93DF92CF92E0917503F09196
:10452000760309958CE380931D028DB79EB708969C
:104530008DBF8091BD05E82FFF27EE0FFF1FEC51C7
:10454000F94F8081918181589F4F9F938F938091E4
:10455000BC05E82FFF27EE0FFF1FEC51F94F8081BC
:10456000918181589F4F9F938F938AEB95E063C20F
:1045700010921D028AEC95E09F938F930FE91FE143
:10458000DF92CF92FE010995809102010F900F906A
:104590000F900F908A3009F09DC084E180931D0236
:1045A0008091D9029091DA029C0197FF02C0295FA5
:1045B0003F4F287F821B930B9F938F938091D9024B
:1045C0009091DA0297FD079673E0959587957A9515
:1045D000E1F79F938F932091D9023091DA0237FF50
:1045E00002C0295F3F4F63E0359527956A95E1F753
:1045F0008091FD019091FE01821B930B9F938F93FD
:1046000088ED95E09F938F931F930F93E09175032F
:10461000F0917603099588E280931D022DB73EB78D
:10462000265F3F4F2DBF8091D7029091D8029C0109
:1046300097FF02C0295F3F4F287F821B930B9F93F8
:104640008F938091D7029091D80297FD079653E0FF
:10465000959587955A95E1F79F938F932091D7026F
:104660003091D80237FF02C0295F3F4F43E03595B4
:1046700027954A95E1F78091FB019091FC01821BFF
:10468000930B9F938F9389EE95E09F938F931F9346
:104690000F93E0917503F091760309958CE3809375
:1046A0001D028DB79EB70A968DBF8091D50290915D
:1046B000D6029F938F938091D5029091D60220913C
:1046C000F9013091FA01821B930B9F938F938AEF2C
:1046D00095E0ADC08B3019F0843108F4ADC084E1B1
:1046E00080931D028091D9029091DA029C0197FF7C
:1046F00002C0215F3F4F207F821B930B97FD0196E5
:10470000959587959F938F938091D9029091DA0226
:1047100097FD0F9624E0959587952A95E1F79F934D
:104720008F932091D9023091DA0237FF02C0295FBE
:104730003F4FC3E035952795CA95E1F78091FD017C
:104740009091FE01821B930B9F938F9388E096E0DC
:104750009F938F931F930F93E0917503F0917603CE
:10476000099588E280931D022DB73EB7265F3F4F23
:104770002DBF8091D7029091D8029C0197FF02C073
:10478000215F3F4F207F821B930B97FD01969595EC
:1047900087959F938F938091D7029091D80297FD30
:1047A0000F96A4E095958795AA95E1F79F938F932F
:1047B0002091D7023091D80237FF02C0295F3F4FC6
:1047C000F3E035952795FA95E1F78091FB019091FB
:1047D000FC01821B930B9F938F938AE196E09F933A
:1047E0008F931F930F93E0917503F09176030995D2
:1047F0008CE380931D028DB79EB70A968DBF809182
:10480000D5029091D60297FD0196959587959F9335
:104810008F938091D5029091D6022091F901309129
:10482000FA01821B930B9F938F938CE296E09F93E8
:104830008F931F930F9303C18D3009F0CBC484E194
:1048400080931D028091130199279F938F938091EC
:10485000D9029091DA0297FD0F9674E095958795AD
:104860007A95E1F79F938F932091D9023091DA02E4
:1048700037FF02C0295F3F4F63E0359527956A9562
:10488000E1F78091FD019091FE01821B930B9F93B4
:104890008F938BE396E09F938F931F930F93E091F9
:1048A0007503F0917603099588E280931D022DB778
:1048B0003EB7265F3F4F2DBF8091120199279F93EE
:1048C0008F938091D7029091D80297FD0F9654E074
:1048D000959587955A95E1F79F938F932091D702ED
:1048E0003091D80237FF02C0295F3F4F43E0359532
:1048F00027954A95E1F78091FB019091FC01821B7D
:10490000930B9F938F938FE496E09F938F931F93C6
:104910000F93E0917503F091760309958CE38093F2
:104920001D028DB79EB70A968DBF80911101992700
:104930009F938F938091D5029091D60297FD019617
:10494000959587959F938F938091D5029091D602EC
:104950002091F9013091FA01821B930B9F938F9361
:1049600083E696E09F938F931F930F93E0917503D7
:10497000F09176030995EDB7FEB73A9668C01092AC
:104980001D0287E796E09F938F93DF92CF92FE01FF
:10499000099584E180931D020F900F900F900F9066
:1049A0008091CF029091D0029F938F938091F501D7
:1049B0009091F6019F938F9384E896E09F938F9355
:1049C000DF92CF92E0917503F0917603099588E22A
:1049D00080931D022DB73EB7285F3F4F2DBF8091BA
:1049E000CD029091CE029F938F938091F701909189
:1049F000F8019F938F9383E996E09F938F93DF92C3
:104A0000CF92E0917503F091760309958CE3809342
:104A10001D028DB79EB708968DBF8091C9029091F7
:104A2000CA029F938F938091F3019091F4019F9319
:104A30008F9382EA96E09F938F93DF92CF92E091DB
:104A40007503F09176030995EDB7FEB73896EDBF83
:104A5000C1C310921D0280911E0190911F016AE056
:104A600070E00E9432789F938F9380911E01909105
:104A70001F016AE070E00E9432787F936F9381EBB0
:104A800096E09F938F93DF92CF92FE01099584E188
:104A900080931D022DB73EB7285F3F4F2DBF8091F9
:104AA0003208909133086AE070E00E941E789F936C
:104AB0008F9380913208909133086AE070E00E94F1
:104AC0001E787F936F9385EC96E09F938F93DF9290
:104AD000CF92E0917503F0917603099588E2809377
:104AE0001D028DB79EB708968DBF809134089091B6
:104AF00035089F938F9389ED96E09F938F93DF9274
:104B0000CF92E0917503F091760309958CE3809341
:104B10001D02EDB7FEB73696EDBF80913608909135
:104B200037089F938F9389EE96E09F938F93DF9240
:104B3000CF92E0917503F091760309952DB73EB7BA
:104B40002A5F3F4F4FC110921D028BEF96E09F935B
:104B50008F93DF92CF92FE01099584E180931D022D
:104B60000F900F900F900F908091E4069091E506C2
:104B70009F938F9384E097E09F938F93DF92CF92E0
:104B8000E0917503F0917603099588E280931D0208
:104B90008DB79EB706968DBF80916A0299279F9325
:104BA0008F9384E197E09F938F93DF92CF92E09170
:104BB0007503F091760309958CE380931D02EDB7A0
:104BC000FEB73696EDBF8091E306992701979F9334
:104BD0008F9384E297E0A9CF10921D0284E397E0BF
:104BE0009F938F93DF92CF92FE01099584E180938A
:104BF0001D020F900F900F900F9080918F01909158
:104C000090019F938F938CE397E09F938F93DF9214
:104C1000CF92E0917503F0917603099588E2809335
:104C20001D028DB79EB706968DBF80915A07909151
:104C30005B079F938F938AE497E09F938F93DF9214
:104C4000CF92E0917503F091760309958CE3809300
:104C50001D02EDB7FEB73696EDBF809182029091AE
:104C600083029F938F9388E597E05FCFCBE6CC2EAE
:104C7000C2E0DC2E20E030E0E901B3E0FB2EC0937F
:104C80001D02F60181916F0199279F938F938901EE
:104C90000F5F1F4F1F930F9386E697E09F938F93AD
:104CA0008FE99FE19F938F93E0917503F0917603D5
:104CB00009952DB73EB7285F3F4F2DBFFA946496F4
:104CC0009801F7FEDCCF86C2AFE6CA2EA2E0DA2E4C
:104CD000C0E0D0E08E01F3E0FF2E00931D02F6014C
:104CE00081916F0199279F938F932596DF93CF939F
:104CF00083E797E09F938F938FE99FE19F938F9333
:104D0000E0917503F091760309952DB73EB7285FC2
:104D10003F4F2DBFFA940C5E1F4F2497F7FEDDCF57
:104D200059C210921D0280E897E09F938F930FE97C
:104D30001FE1DF92CF92FE01099584E180931D026D
:104D40000F900F900F900F9080916E0199279F9375
:104D50008F9388E897E09F938F93DF92CF92E091B3
:104D60007503F0917603099588E280931D028DB753
:104D70009EB706968DBF8091D4019091D50197FD85
:104D8000039695958795959587959F938F9386E93B
:104D900097E09F938F931F930F93E0917503F0918A
:104DA000760309958CE380931D02EDB7FEB7369626
:104DB000EDBF8091E50599279F938F938091E4053E
:104DC00099279F938F9384EA97E09F938F931F93E4
:104DD0000F93E0917503F091760309952DB73EB7D7
:104DE000285F3F4F2DBFF6C110921D0282EB97E066
:104DF0009F938F937FE9A72E7FE1B72EDF92CF920B
:104E0000FE0109950F900F900F900F90C3E8D6E028
:104E100000E010E062E0F62E802F8C5E80931D0291
:104E20008B8D99278F7790709F938F938B8999277C
:104E30008F7790709F938F938B8599278F77907042
:104E40009F938F938B8199278F7790709F938F93E8
:104E500082EC97E09F938F93BF92AF92E09175039E
:104E6000F091760309958DB79EB70C968DBFFA9495
:104E70000C5E1F4FA096F7FECFCFACC110921D0263
:104E800083ED97E09F938F935FE9A52E5FE1B52EA9
:104E9000DF92CF92FE0109950F900F900F900F9027
:104EA000C3E8D6E000E010E042E0F42E802F8C5EF4
:104EB00080931D028F8D992787FD90959F938F93E7
:104EC0008F89992787FD90959F938F938F85992739
:104ED00087FD90959F938F938F81992787FD90955C
:104EE0009F938F9382EE97E09F938F93BF92AF92A1
:104EF000E0917503F09176030995EDB7FEB73C9606
:104F0000EDBFFA940C5E1F4FA096F7FECFCF62C1A3
:104F100010921D0283EF97E09F938F930FE91FE19B
:104F2000DF92CF92FE01099584E180931D020F90DC
:104F30000F900F900F9080919E06881F8827881FE2
:104F400097E0899FC00111248D969F938F93809144
:104F50009606881F8827881F96E0899FC001112424
:104F60008D969F938F9380918E06881F8827881F28
:104F700095E0899FC00111248D969F938F93809116
:104F80008606881F8827881F9927880F991F880FF2
:104F9000991F8D969F938F9382E098E09F938F93B4
:104FA000DF92CF92E0917503F0917603099588E244
:104FB00080931D022DB73EB7245F3F4F2DBF8091D8
:104FC000BE06881F8827881F9BE0899FC001112487
:104FD0008D969F938F938091B606881F8827881F90
:104FE0009AE0899FC00111248D969F938F938091A1
:104FF000AE06881F8827881F99E0899FC001112469
:105000008D969F938F938091A606881F8827881F6F
:10501000992723E0880F991F2A95E1F78D969F9392
:105020008F9386E198E09F938F93DF92CF92E091E8
:105030007503F091760309958CE380931D028DB77B
:105040009EB70C968DBF8091C606881F8827881F43
:105050009CE0899FC00111248D969F938F938AE2D3
:1050600098E09F938F93DF92CF92E0917503F09138
:10507000760309958091CE06EDB7FEB73696EDBF63
:1050800087FF12C080E480931D028BE398E09F931A
:105090008F93DF92CF92E0917503F091760309959B
:1050A0000F900F900F900F908091D60687FF12C03F
:1050B00084E480931D028EE398E09F938F931F9367
:1050C0000F93E0917503F091760309950F900F907F
:1050D0000F900F908091DE0687FF7CC088E480935C
:1050E0001D0281E498E09F938F931F930F93E091AB
:1050F0007503F091760309950F900F900F900F9024
:1051000069C010921D0284E498E09F938F93DF9210
:10511000CF92FE01099584E180931D020F900F90BC
:105120000F900F908091AA019091AB019F938F9364
:1051300082E598E09F938F93DF92CF92E091750381
:10514000F0917603099588E280931D022DB73EB752
:105150002A5F3F4F2DBF8091AC019091AD019F938D
:105160008F938FE598E09F938F93DF92CF92E0919A
:105170007503F0917603099589E480931D028DB73C
:105180009EB706968DBF8CE698E09F938F93DF9233
:10519000CF92E0917503F0917603099580911B02FF
:1051A0000F900F900F900F9083FF14C01092AD01DD
:1051B0001092AC0160E070E08EE090E00E94F52A71
:1051C00009C080912001281719F421502093200153
:1051D00010921C0210921B02DF91CF911F910F9130
:1051E000FF90DF90CF90BF90AF900895F999FECFD8
:1051F00092BD81BDF89A80B599270895F999FECF9F
:105200001FBA92BD81BD60BD0FB6F894FA9AF99AA3
:105210000FBE08954AEA20E030E02617370740F431
:10522000FC018191480F2F5F3F4F26173707C8F3C6
:10523000842F99270895EAEA40E050E0461757077F
:1052400078F49C01F999FECF32BD21BDF89A80B562
:10525000E80F4F5F5F4F2F5F3F4F4617570790F3A1
:105260008E2F9927089581E08093B80582E080937E
:10527000B70583E08093B60584E08093B90585E0A7
:105280008093BA0586E08093BB0587E08093BC05D8
:1052900088E08093BD0589E08093BE058AE0809315
:1052A000BF058BE08093C0058CE08093C105089515
:1052B00088E58093B50580910201843150F08AE041
:1052C0008093D5051092F9058BE18093D1058EE48A
:1052D0000AC083E08093D50580E28093F9058EE1D2
:1052E0008093D10585E58093F6058093F70580E2EC
:1052F0008093F8058AE68093C20582E280931F06B8
:1053000064E06093DC05109218061092150648E0E0
:105310004093CF0556EE5093D00530E43093D2053C
:105320009EE19093C3058FEF8093C5052FE02093F6
:10533000C6059093C4051092C8054093C9053093E3
:10534000CA051092CB052093C7051092DE05109276
:10535000DF051092E0051092E1051092FB05109216
:10536000FC051092FD051092FE0590E89093E20571
:1053700032E33093E30582E080931E062093E40538
:105380005093E5056093EA058DE78093ED058093E2
:10539000EE058093EF059093E60525E52093E7055C
:1053A00086E48093E8058CED8093E9058CE3809397
:1053B000EB051092EC058FE58093FF0583EF80935A
:1053C00001068AEA809303068093040684E18093B1
:1053D0000006809302063093F0059AE59093F1055C
:1053E0003093F20510921D068EEF8093050684E639
:1053F00080930606909307069093080690930906FB
:105400008BE480930A0620930B0680930C0610927F
:105410000D0686E080930E0640930F0690931006CB
:105420008AE28093110685EF809312068CE88093C0
:10543000130685E080931406109216061092170644
:1054400081E28093D9058DE28093DA059093DB05A4
:105450001092190610921A0610921B0686E9809384
:105460001C069093F30587E38093F4050895CF938A
:10547000DF930E9458298AE08093CC0580E18093D5
:10548000CD0526E02093CE059AE59093D30588E7D5
:105490008093D4059093D6058093D7052093D805A3
:1054A00080E28093DD058CE38093F5058BE48093A7
:1054B000FA05A0E2B6E08CE0E1E2F1E0ED01019056
:1054C00009928A95E1F767E770E0CD018B5690402D
:1054D0000E940A2980932C06DF91CF910895CF93E3
:1054E000DF930E94582988E08093CC0530E1309307
:1054F000CD0526E02093CE0594E69093D30588E76A
:105500008093D4059093D6058093D7052093D80532
:105510003093DD0586E48093F5058093FA05A0E2DB
:10552000B6E08CE0E7E2F1E0ED01019009928A95A6
:10553000E1F767E770E0CD018B5690400E940A29A1
:1055400080932C06DF91CF910895CF93DF930E9433
:10555000582926E02093CC058AE08093CD0584E08D
:105560008093CE0594E69093D30588E78093D40585
:105570009093D6058093D7052093D80580E180933A
:10558000DD0586E48093F5058093FA05A0E2B6E098
:105590008CE0EFE2F1E0ED01019009928A95E1F7EC
:1055A00067E770E0CD018B5690400E940A298093F6
:1055B0002C06DF91CF910895F999FECF92BD81BD60
:1055C000F89A80B599270895F999FECF1FBA92BD30
:1055D00081BD60BD0FB6F894FA9AF99A0FBE08958E
:1055E00066EF78E20E94817608954EEF58E20E94BD
:1055F000BB760895EF92FF920F931F93CF93C82F1E
:105600008150853008F0C3E088E7C89F80011124ED
:105610008CEEE82E8FEFF82EE00EF11E67E770E0BB
:10562000C7010E941B29682F98012D593F4F8FB346
:105630009927AC014270507081FDF9CF32BD21BD78
:10564000F89A80B5861711F0CA0121C08FB3992747
:105650009C012270307081FDF9CFF2BCE1BCF89A58
:1056600080B5883511F0C90112C088E7C89FC00114
:105670001124449726EF38E248E750E0BC0185EB5F
:1056800095E00E945C760E94536681E090E0CF91A5
:105690001F910F91FF90EF900895282F863010F002
:1056A00025E003C0882309F421E0F999FECF1FBA51
:1056B00082E090E092BD81BD20BD0FB6F894FA9AC9
:1056C000F99A0FBE0895CF93C82F8091B5058835FC
:1056D00009F044C0C63010F0C5E003C0CC2309F483
:1056E0003DC00E94E77467E770E085EB95E00E949B
:1056F0000A2980932C0688E7C89FC00111242EEF49
:1057000038E248E750E065EB75E044970E949976EF
:105710002EEF38E24CE050E066EB75E080E590E07B
:105720000E9499766CE070E086EB95E00E940A2971
:10573000282FF999FECF1FBA8CE590E092BD81BD6C
:1057400020BD0FB6F894FA9AF99A0FBE8C2F0E94DA
:105750004D2B0E94536681E090E002C080E090E013
:10576000CF9108956DE470E088EE93E00E941B29CC
:10577000482F8FB399279C012270307081FDF9CF9B
:1057800085E394E092BD81BDF89A80B5841779F4E1
:105790008FB399279C012270307081FDF9CF88EE7C
:1057A00093E092BD81BDF89A80B5813011F0C901B6
:1057B000089526EF38E24EE450E068EE73E08DE2A3
:1057C00096E00E945C7681E090E0089580912D063D
:1057D0008130A9F46DE470E08DE296E00E940A2920
:1057E00080937A062EEF38E24EE450E06DE276E0E8
:1057F00088EE93E00E94997681E090E0089580E041
:1058000090E00895CF93DF9381E080932D06EDE241
:10581000F6E08FE0158616861786108A815034963A
:1058200087FFF8CF80E480933A0680933B0610927E
:105830003C0680933D0680933E0690EC90933F0695
:1058400010924006809341068093420610924306D0
:10585000909344069093450680934606109247061F
:105860008093480690934906AEE2B6E087E0E5E310
:10587000F1E0ED01019009928A95E1F76DE470E0A5
:10588000CD0101970E940A2980937A06DF91CF917A
:105890000895F999FECF82E090E092BD81BDF89A1B
:1058A00080B5282F863078F023E0322FF999FECF8B
:1058B0001FBA82E090E092BD81BD30BD0FB6F89472
:1058C000FA9AF99A0FBE822F992708951F93CF93C2
:1058D000C82F162F863010F0C5E003C0882309F4C6
:1058E000C1E08C2F99278230910541F083309105DA
:1058F00044F4019731F40E94372A05C00E946F2AB0
:1059000002C00E94A52A1123E1F06CE070E080E55E
:1059100090E00E941B29282FF999FECF8CE590E09A
:1059200092BD81BDF89A80B5821759F426EF38E20E
:105930004CE050E060E570E086EB95E00E945C761C
:1059400002C00E9433298C2F0E94632BCF911F919C
:105950000895DF92EF92FF920F931F93CF93FF244E
:10596000DF2CEF2C81E090E00E94DC2A883511F0DA
:1059700031E0E32E6CE070E080E590E00E941B29AE
:10598000C82FF999FECF8CE590E092BD81BDF89AC1
:1059900080B58C1711F421E0D22EC1E001E010E0B7
:1059A000EE2029F48C2F0E94FA2A8823C9F591E071
:1059B000F92E1F930F9384E798E09F938F9386E9C6
:1059C00092E19F938F93E0917503F091760309958F
:1059D0002DB73EB72A5F3F4F2DBF0230110549F06A
:1059E000033011054CF40130110531F40E94372ABF
:1059F00005C00E946F2A02C00E94A52ADD2059F02E
:105A000026EF38E24CE050E060E570E086EB95E090
:105A10000E945C7602C00E9433298C2F0E94632B67
:105A2000CF5F0F5F1F4FC63008F4BACFFF2019F0C9
:105A300083E00E944D2B0E94492CC82F0E94FA2A15
:105A40008C2F99279F938F938AE998E09F938F9348
:105A500006E912E11F930F93E0917503F09176032D
:105A6000099581E090E00E94DC2A2DB73EB72A5FBD
:105A70003F4F2DBF8F3F21F00E94B22B882399F416
:105A800083EB98E09F938F931F930F93E09175039F
:105A9000F091760309950E94022C0E94E62B0F904C
:105AA0000F900F900F90EE2029F068E581E090E0D4
:105AB0000E94E42A1092B40590E0EAE3F6E0CFE019
:105AC0008081349618160CF49F5FC150C7FFF8CF41
:105AD0009093B405892F99279F938F938EE296E038
:105AE0009F938F9384ED98E09F938F931F930F93D1
:105AF000E0917503F091760309958DB79EB70896EE
:105B00008DBF85EF98E09F938F931F930F93E09144
:105B10007503F091760309950F900F900F900F90F9
:105B2000CF911F910F91FF90EF90DF900895982FE4
:105B30002FB7F8943998389A88B1836088B98091E2
:105B4000B9008C7F8093B9008AE28093B8001092EC
:105B500028021092260210922502992379F0E3E898
:105B6000F6E08BE010821182128213821482158279
:105B7000168217828150389687FFF4CF78942FBF12
:105B800008951092280284E98093BC0080E88093F5
:105B9000BC001092BD001092BA001092BB0010928F
:105BA000B9001092B8001092240280E00E94972D54
:105BB0001092BB0085E88093BC0080912202826035
:105BC0008093220208951F920F920FB60F92112414
:105BD0002F933F934F935F938F939F93EF93FF93F5
:105BE00080912802282F3327442755278F5F8093E1
:105BF0002802F9012731310508F0C2C2EF59FF4FE1
:105C00000C94B97881E08093240209C08091260227
:105C10008C3090F4809126028F5F809326028091D1
:105C20002602E82FFF27EE0FFF1FEE0FFF1FE35D99
:105C3000F94F8585181654F7809126028C3070F044
:105C400010922102109220021092260285E0809389
:105C5000280280912502880F8D5A04C08091260267
:105C6000880F8E5A8093BB0085E87FC28091260200
:105C7000E82FFF2783E0EE0FFF1F8A95E1F7ED572E
:105C8000F94F81818093BB0085E88093BC008091AF
:105C90002602E82FFF27EE0FFF1FEE0FFF1FEE0F6C
:105CA000FF1FED57F94F808180FF91C08091260240
:105CB000E82FFF27EE0FFF1FEE0FFF1FEE0FFF1F56
:105CC000ED57F94F8281882329F08091B405873000
:105CD00008F46CC28091200290912102892B09F076
:105CE00065C280911E0290911F02892B09F05EC24D
:105CF0006EC08091260221E030E002C0220F331FE7
:105D00008A95E2F780911E0290911F022823392381
:105D1000232B79F080912602E82FFF27EE0FFF1F3B
:105D2000EE0FFF1FEE0FFF1FED57F94F80E1848349
:105D30000DC080912602E82FFF27EE0FFF1FEE0F08
:105D4000FF1FEE0FFF1FED57F94F148280912602BF
:105D5000E82FFF2753E0EE0FFF1F5A95E1F7ED57AD
:105D6000F94F8481282F332743E0220F331F4A95B0
:105D7000E1F780912602E82FFF2793E0EE0FFF1F47
:105D80009A95E1F7ED57F94F82818770822B8093C6
:105D9000BB0085E88093BC002091260281E090E062
:105DA00002C0880F991F2A95E2F7209120023091B6
:105DB000210282239323892B51F08BE796E0909365
:105DC0002C0280932B0288E080932D02EFC184E0A7
:105DD00089C1E0912B02F0912C0281918093BB004C
:105DE00085E88093BC00F0932C02E0932B02809115
:105DF0002D02815080932D02882309F4D7C183E0BE
:105E000071C18091B900803351F5809129028823B6
:105E100029F4809126028F5F8093290280912602C7
:105E2000E82FFF2783E0EE0FFF1F8A95E1F7ED577C
:105E3000F94F838199278F7790708F3791057CF484
:105E400080912602E82FFF27EE0FFF1FEE0FFF1FA6
:105E5000EE0FFF1FED57F94F83818F5F8383109201
:105E6000280284E98093BC008AE090E090933E0190
:105E700080933D01809126028F5F809326021092CD
:105E800028026DC18091B9008034C9F1809125024A
:105E9000E82FFF27EE0FFF1FEE0FFF1FEE0FFF1F74
:105EA000ED57F94F83818F778383809125028F5F30
:105EB00080932502809125028C30A0F0109225025B
:105EC00010921F0210921E0280912A028F5F80930F
:105ED0002A028C3038F010922A02809122028D7FA3
:105EE000809322028091220281608093220210928C
:105EF000280284E98093BC001092240273C0809130
:105F00002502E82FFF27EE0FFF1FEE0FFF1FEE0FFA
:105F1000FF1FED57F94F83818068838380912502AD
:105F2000E82FFF27EE0FFF1FEE0FFF1FEE0FFF1FE3
:105F3000ED57F94F808180FF2FC080912502E82F17
:105F4000FF2753E0EE0FFF1F5A95E1F7ED57F94F8A
:105F500084819927009751F04097D9F58BE796E017
:105F600090932C0280932B0288E031C0809125020F
:105F7000992743E0880F991F4A95E1F78857994F71
:105F800090932C0280932B029091250280912A02FB
:105F90009817E1F483E01BC080912502992733E034
:105FA000880F991F3A95E1F78857994F90932C02E3
:105FB00080932B028091220281FD06C090912502E0
:105FC00080912A02981711F482E001C081E0809349
:105FD0002D0280912D02813011F485E801C085ECFD
:105FE0008093BC00809129028093230210922902A1
:105FF000DDC0E0912B02F0912C028091BB008083E8
:1060000080912B0290912C02019690932C02809308
:106010002B0280912D02815080932D02823010F04E
:1060200085EC5DC0813011F485E859C08091220271
:1060300081FF2DC08091340280FD1DC0809125021A
:10604000E82FFF2723E0EE0FFF1F2A95E1F7ED571A
:10605000F94F86818A3F79F480912502E82FFF2746
:1060600093E0EE0FFF1F9A95E1F7ED57F94F80810E
:10607000816080830CC080912502E82FFF2783E098
:10608000EE0FFF1F8A95E1F7ED57F94F10828091CF
:1060900025028F5F80932502809125028C30A0F02D
:1060A0001092250210921F0210921E0280912A0265
:1060B0008F5F80932A028C3038F010922A028091F0
:1060C00022028D7F809322021092280284E980931D
:1060D000BC008091220281608093220265C080937F
:1060E000BC0086E08093280261C088E9BBCD809126
:1060F0002702880F805FB6CD8091270299278130D3
:10610000910561F0823091051CF4892B21F04EC07D
:10611000029739F04BC080911301A4CD80911201F8
:10612000A1CD809111019ECD80E89CCD10922802D6
:1061300084E98093BC00109224028AE090E090935E
:106140003E0180933D0180912702823088F4809146
:1061500027028F5F8093270282E18093280280913B
:1061600022028E7F8093220285EA8093BC001EC0AB
:10617000109227028091220281608093220216C031
:106180001092280284E98093BC00809122028160F1
:10619000809322028AE090E090933E0180933D013B
:1061A000109226021092250210922402FF91EF9184
:1061B0009F918F915F914F913F912F910F900FBEC3
:1061C0000F901F9018951F93CF93DF93182F8091F6
:1061D0006902882321F48091B901882319F081E0B4
:1061E00090E097C01D3008F092C01123B1F0E12F6C
:1061F000FF2723E0EE0FFF1F2A95E1F7ED57F94F38
:1062000035978081359688230CF081C0389780813E
:1062100080FD03C083E090E07CC080917B068230EB
:1062200019F084E090E075C067E070E08BE796E0DD
:106230000E940A2990918206891719F085E090E062
:1062400068C080ED97E00E94A516EC0180912202C3
:1062500080FD05C0CE010E94AE168823B9F311233C
:1062600019F48FEF90E00BC0212F332721503040DD
:1062700081E090E002C0880F991F2A95E2F7909381
:10628000210280932002A1E0B0E0E3E8F6E040E0E4
:1062900050E06BE0CD01042E02C0880F991F0A94D4
:1062A000E2F7209120023091210282239323892B4F
:1062B00011F01182128261504F5F5F4F389667FF75
:1062C000E9CF1092260210922802809122028E7F3E
:1062D0008093220285EA8093BC008091220280FD97
:1062E00005C0CE010E94AE168823B9F3809120022A
:1062F00090912102892B29F0CE010E94AE168823AD
:1063000011F38091200290912102009711F082E018
:1063100090E0DF91CF911F9108950F931F93CF933A
:10632000DF93982F80916902882321F48091B9012D
:10633000882319F081E090E092C09D30A0F4992369
:1063400019F486E090E08BC0C92FDD27FE0133E011
:10635000EE0FFF1F3A95E1F7ED57F94F3597808122
:10636000359687FD03C082E090E079C03897808140
:1063700080FD03C083E090E072C080ED97E00E9452
:10638000A5168C018091220280FD05C0C8010E94E3
:10639000AE168823B9F3219721E030E0C90102C08D
:1063A000880F991FCA95E2F790931F0280931E02EF
:1063B000D901E3E8F6E040E050E06BE0CD01042EC7
:1063C00002C0880F991F0A94E2F720911E023091B3
:1063D0001F0282239323892B11F0118212826150B4
:1063E0004F5F5F4F389667FFE9CF109225021092FA
:1063F0007B061092820610922802809122028E7FE4
:106400008093220285EA8093BC008091220280FD65
:1064100005C0C8010E94AE168823B9F380911E0200
:1064200090911F02892B29F0C8010E94AE16882383
:1064300011F380917B06823019F084E090E00FC068
:1064400067E070E08BE796E00E940A29909182064F
:10645000891719F085E090E002C080E090E0DF91BC
:10646000CF911F910F910895CF93DF9380E022E8A1
:106470003FEFC8E1D7E0E4EEF6E0DF01853020F43D
:1064800011961C921E9202C03183208319821882B9
:1064900022968F5F129632968A3180F31092D6023E
:1064A0001092D5021092D8021092D7021092DA02FE
:1064B0001092D902DF91CF9108951F920F920FB6DB
:1064C0000F9211240F931F932F933F934F935F933A
:1064D0006F937F938F939F93AF93BF93CF93DF93EC
:1064E000EF93FF93409186005091870080912F0297
:1064F00090913002481B590BCA0157FD0196AC011F
:106500005595479580918600909187009093300231
:1065100080932F02CA0189599840A0913102B0910D
:106520003202875E954338F4149714F010924101BB
:1065300081E090E081C0AD30B1050CF081C0CA01AE
:106540008B5F90408356944008F071C0425C53408A
:10655000FD01EA0FFB1FEC51F94F80819181FA0197
:10656000E81BF90BCF01F7FF03C0909581959F4F72
:1065700006974CF480916A02883C28F480916A0264
:10658000865F80936A02FD01EA0FFB1FEC51F94F11
:10659000808191819C01220F331F280F391F240F06
:1065A000351F37FF02C02D5F3F4FE901D595C795D5
:1065B000D595C795CA0101968C179D0714F42197AC
:1065C00006C041505040C417D5070CF42196809165
:1065D0006A02833CD8F08D010A0F1B1FF801EC51B1
:1065E000F94F808191819E01281B390BC90163E01D
:1065F00070E00E943278CB01880F991F860F971F99
:10660000085E184FF8019183808307C0AA0FBB1F53
:10661000A85EB84F11961C921E92E0913102F09143
:106620003202EE0FFF1FEC51F94FD183C0838091EE
:10663000310290913202019690933202809331029E
:10664000FF91EF91DF91CF91BF91AF919F918F918A
:106650007F916F915F914F913F912F911F910F917A
:106660000F900FBE0F901F901895EF92FF920F930F
:106670001F938091D1059927880F991F880F991F23
:106680007C010027F7FC0095102F8091C4029091A7
:10669000C502A091C602B091C702BC01CD01A801FC
:1066A00097010E946778309311052093100580911F
:1066B000BC029091BD02A091BE02B091BF02BC018C
:1066C000CD01A80197010E946778309313052093AC
:1066D00012058091A1079091A20797FD03969595C9
:1066E00087959595879590931505809314058091CE
:1066F000B1079091B20797FD03969595879595956B
:10670000879590931705809316058091D5029091F7
:10671000D6022091F9013091FA01821B930B9093DC
:106720001905809318058091640290916502A091EB
:106730006602B0916702BC01CD0125E030E040E087
:1067400050E00E94677830931B0520931A058091D2
:10675000F3019091F40190931D0580931C058091A5
:106760008F01909190019093210580932005809155
:106770001E0190911F019093230580932205809123
:106780006A029927909325058093240580915A07E2
:1067900090915B079093270580932605809184064E
:1067A0009927909329058093280580918C06992735
:1067B00090932B0580932A058091940699279093B6
:1067C0002D0580932C0580919C06992790932F0589
:1067D00080932E058091D4019091D5019093390535
:1067E00080933805809132089091330890933D054D
:1067F00080933C05809136089091370890933F052F
:1068000080933E058091600290916102A0916202A6
:10681000B0916302BC01CD0125E030E040E050E0E2
:106820000E94677830934105209340058091820251
:106830009091830290934705809346058091380894
:10684000992790934B0580934A0580913703909147
:10685000380390934D0580934C05809135039091BA
:10686000360390934F0580934E0580918E038823C5
:1068700021F480918F03882321F080910F0581609E
:1068800003C080910F058E7F80930F051F910F919C
:10689000FF90EF9008951F93CF93DF93182FEB0194
:1068A00080916902882309F5809102018C3010F4EF
:1068B000299801C0299A11501F3F81F0D093DB0124
:1068C000C093DA018091DA019091DB01892BD1F735
:1068D000CE018C0F9D1F0E94BA16EDCF8091020150
:1068E0008C3010F4299A01C02998DF91CF911F9123
:1068F0000895CF93DF93809102018D3011F40E94AF
:10690000B31A10927A008091FD019091FE0190934C
:106910006607809365078091FB019091FC0190933D
:106920005607809355078091F9019091FA01909351
:10693000A7078093A6072091F5013091F601C901C0
:10694000880F991F880F991F820F931F820F931F23
:106950009093A2078093A1072091F7013091F8014D
:10696000C901880F991F880F991F820F931F820FEB
:10697000931F9093B2078093B1078FEC80937A00B6
:10698000ABE6B2E0CAEBD5E097E08991E82FFF27AC
:10699000EE0FFF1FEC51F94F0190F081E02DE1580F
:1069A000FF4F1E161F061CF0E0E0F0E005C0EF3FB1
:1069B000F10514F0EFEFF0E08C91282F3327E21768
:1069C000F30714F4815004C02E173F0714F48F5FAF
:1069D0008C939150119697FFD8CF8091F605992707
:1069E000AA27BB27BC01CD0124EC39E040E050E0F0
:1069F0000E94F377DC01CB0180938701909388019B
:106A0000A0938901B0938A018091F7059927AA275D
:106A1000BB27BC01CD010E94F377DC01CB01809341
:106A2000830190938401A0938501B0938601DF9147
:106A3000CF910895A0E0B0E0E0E2F5E30C9488780F
:106A4000882EC0E0D0E07E016E0110928E03469A3F
:106A5000D093D002C093CF02D093CE02C093CD0288
:106A6000D093CA02C093C902D093DA02C093D9026C
:106A7000D093D802C093D702D093D602C093D50248
:106A800010926B0110926A011092ED010E9479340C
:106A900084E690E00E94C7160E9479348091C20576
:106AA00080FF10C08091140190911501875B934085
:106AB00038F480911401909115018E5E924010F48B
:106AC0000E94581A0FE18AE090E00E94C716809158
:106AD000F9019091FA01C80FD91F8091FD019091A1
:106AE000FE01E80EF91E8091FB019091FC01C80E99
:106AF000D91E015007FFE7CF9701205F3F4F369522
:106B00002795369527953093DA022093D902C6014E
:106B1000409696958795969587959093D802809301
:106B2000D7026096F5E0D695C795FA95E1F7D09330
:106B3000D602C093D5029093D4028093D3023093AF
:106B4000D2022093D102882009F441C08091A1078C
:106B50009091A20797FF03C0909581959F4F6CE09D
:106B600070E00E9432789B017093D0026093CF0254
:106B70008091B1079091B20797FF03C090958195DE
:106B80009F4F6CE070E00E9432787093CE02609369
:106B9000CD0280915705909158059093CA02809339
:106BA000C902B90184E090E00E94F52A6091CD020B
:106BB0007091CE0286E090E00E94F52A6091C902B1
:106BC0007091CA0288E090E00E94F52A65C084E0D6
:106BD00090E00E94F02A9093D0028093CF0286E04A
:106BE00090E00E94F02A9093CE028093CD0288E03C
:106BF00090E00E94F02A9C019093CA028093C902FF
:106C00008091CF029091D0028150984050F48091B1
:106C1000CD029091CE028150984018F4215034401A
:106C2000D8F186E199E09F938F9386E992E19F9353
:106C30008F93E0917503F091760309958091A107F8
:106C40009091A20797FF03C0909581959F4F6CE0AC
:106C500070E00E9432787093D0026093CF028091EE
:106C6000B1079091B20797FF03C0909581959F4F10
:106C70006CE070E00E9432787093CE026093CD0297
:106C800080915705909158059093CA028093C9024C
:106C90000F900F900F900F9010926607109265075B
:106CA00010925607109255071092A7071092A60748
:106CB00084E690E00E94C7168091F5019091F6015C
:106CC0009C01220F331F220F331F280F391F280F5B
:106CD000391F3093A2072093A1078091F70190916B
:106CE000F8018C01000F111F000F111F080F191F51
:106CF000080F191F1093B2070093B1078091D105B7
:106D0000C82EDD24EE24FF24442737FD4095542F60
:106D1000C701B6010E94F3774B015C016093C40286
:106D20007093C5028093C6029093C70298014427CE
:106D300037FD4095542FC701B6010E94F377DC015F
:106D4000CB018093BC029093BD02A093BE02B0938E
:106D5000BF028092A0029092A102A092A202B092E1
:106D6000A3028093980290939902A0939A02B09301
:106D70009B02109294021092950210929602109229
:106D800097028091160190911701A0911801B0917E
:106D9000190190935A05809359051092EC011092B5
:106DA000EB011092840210928502109286021092DA
:106DB000870200918F01109190011093830200933C
:106DC000820284E690E090938C0180938B0182E3B1
:106DD00090E09093DB018093DA018091F60599278A
:106DE000AA27BB27BC01CD0124EC39E040E050E0EC
:106DF0000E94F377DC01CB018856954CAF4FBF4F13
:106E00008093870190938801A0938901B0938A01B0
:106E10008091F7059927AA27BB27BC01CD010E94C5
:106E2000F377DC01CB018856954CAF4FBF4F809371
:106E3000830190938401A0938501B0938601109201
:106E4000480110924701C801AA2797FDA095BA2FC3
:106E500020914301309144014091450150914601F8
:106E6000BC01CD010E94F377DC01CB018093AD071B
:106E70009093AE07A093AF07B093B00710927F0234
:106E800010927E0281E0809301010E9453668091FE
:106E900034028460809334028FEF80932D08109227
:106EA0002E0880E280932F08CBE6D2E0AAEBB5E073
:106EB00007E08D91E82FFF27EE0FFF1FEC51F94FF0
:106EC0008081918181588993015007FFF2CF84E638
:106ED00080936A028091D801882311F0469A579ACC
:106EE0008091D9029091DA0280569940815C9B4250
:106EF00028F080918E03816080938E038091D70269
:106F00009091D80280569940815C9B4228F08091F4
:106F10008E03826080938E038091D5029091D60279
:106F20008C5291408957954028F080918E0384605F
:106F300080938E038091CF029091D0028C52914029
:106F4000835C914028F080918E03886080938E034B
:106F50008091CD029091CE028C529140835C914001
:106F600028F080918E03806180938E038091C90206
:106F70009091CA02805092408355914028F08091B0
:106F80008E03806280938E0386E480937E01ECE022
:106F9000CDB7DEB70C94A478A3E1B0E0E2EDF7E35F
:106FA0000C9482788091D5029091D6022091F901BB
:106FB0003091FA01821B930B9093A7078093A60749
:106FC000809103029091040297FD07969C0113E0C3
:106FD000359527951A95E1F7309366072093650755
:106FE000809101029091020297FD0796B3E095957A
:106FF0008795BA95E1F7909356078093550730939C
:1070000071072093700790936907809368078091B8
:10701000A1079091A207AC01440F551F480F591FBB
:107020002091F5013091F601C901880F991F880F51
:10703000991F820F931F820F931F480F591F57FFED
:1070400002C04D5F5F4F55954795559547955093B5
:10705000A2074093A1078091B1079091B207AC01BC
:10706000440F551F480F591F2091F7013091F80127
:10707000C901880F991F880F991F820F931F820FD4
:10708000931F480F591F57FF02C04D5F5F4F559523
:107090004795559547955093B2074093B107209176
:1070A000F5013091F601C901880F991F880F991FCA
:1070B000820F931F820F931F9C01442737FD409539
:1070C000542F8091B4029091B502A091B602B09174
:1070D000B702820F931FA41FB51F8093B402909331
:1070E000B502A093B602B093B7022091F701309198
:1070F000F801C901880F991F880F991F820F931FEC
:10710000820F931F9C01442737FD4095542F809197
:10711000B0029091B102A091B202B091B302820F7D
:10712000931FA41FB51F8093B0029093B102A09348
:10713000B202B093B30280917A0790917B072091BD
:10714000F5013091F601820F931F90937B07809396
:107150007A078091A9079091AA072091F7013091B1
:10716000F801820F931F9093AA078093A90780913B
:10717000CB029091CC0201969093CC028093CB02EB
:1071800080915705909158052091C9023091CA020B
:10719000821B930B9C01442737FD4095542F80910F
:1071A000AC029091AD02A091AE02B091AF02820FFD
:1071B000931FA41FB51F8093AC029093AD02A093C0
:1071C000AE02B093AF028FEC80937A001092100160
:1071D00020919C0230919D0240919E0250919F020D
:1071E00029873A874B875C8729543B46414050406A
:1071F0002CF028E43BE641E050E00DC089859A85FB
:10720000AB85BC85885B9449AE4FBF4F4CF428EBEF
:1072100034E94EEF5FEF2D833E834F83588708C0DC
:1072200089859A85AB85BC858D839E83AF83B8871E
:107230002091A4023091A5024091A6025091A7028C
:107240002D873E874F87588B29543B4641405040FD
:107250002CF028E43BE641E050E00DC08D859E8592
:10726000AF85B889885B9449AE4FBF4F4CF428EB8B
:1072700034E94EEF5FEF29833A834B835C8308C088
:107280008D859E85AF85B88989839A83AB83BC83BE
:10729000A091A607B091A707BB8BAA8BFD01CF01D8
:1072A000AA2797FDA095BA2FA0909402B0909502BE
:1072B000C0909602D0909702A80EB91ECA1EDB1E7F
:1072C000A0929402B0929502C0929602D092970238
:1072D000E090AD07F090AE070091AF071091B007B6
:1072E000E80EF91E0A1F1B1FE092AD07F092AE07D1
:1072F0000093AF071093B007F0914F02F98BFF2373
:1073000009F098C180914E02882309F093C18091C1
:107310009D0786FF8FC18091550790915607AA2738
:1073200097FDA095BA2FBC01CD0129813A814B81EF
:107330005C810E94F3779B01AC0197FF04C0215050
:10734000384F4F4F5F4FBBE0559547953795279581
:10735000BA95D1F780916A01682E77248824992400
:10736000CA01B901A40193010E94F377DC01CB01AA
:107370008093E5029093E602A093E702B093E802BF
:10738000B7FF04C08150904FAF4FBF4F1C012D017C
:10739000ACE05594479437942794AA95D1F720925E
:1073A000E5023092E6024092E7025092E8028091B4
:1073B000650790916607AA2797FDA095BA2FBC0193
:1073C000CD012D813E814F8158850E94F37797FF33
:1073D00004C06150784F8F4F9F4FFBE09595879584
:1073E00077956795FA95D1F7A40193010E94F377F9
:1073F000DC01CB018093E9029093EA02A093EB02B7
:10740000B093EC02B7FF04C08150904FAF4FBF4F15
:107410009C01AD01ECE05595479537952795EA9588
:10742000D1F72093E9023093EA024093EB025093A4
:10743000EC028091E5029091E60290934D078093D3
:107440004C078091E9029091EA0290935107809352
:10745000500722193309440955092093E902309352
:10746000EA024093EB025093EC02E20EF31E041F7B
:10747000151FE092AD07F092AE070093AF0710938F
:10748000B007809169018823B1F457FF04C02F5FD2
:107490003F4F4F4F5F4F5595479537952795A21A08
:1074A000B30AC40AD50AA0929402B0929502C0927F
:1074B0009602D09297022A893B8979010027F7FC2E
:1074C0000095102F8091E9029091EA02A091EB02C1
:1074D000B091EC02E80EF91E0A1F1B1FC801B7018C
:1074E00029813A814B815C810E94F3779B01AC0139
:1074F00097FF04C02150384F4F4F5F4F6BE05595B9
:107500004795379527956A95D1F780916B01A82EFD
:10751000BB24CC24DD24CA01B901A60195010E9437
:10752000F377DC01CB018093DD029093DE02A09320
:10753000DF02B093E002B7FF04C08150904FAF4F1D
:10754000BF4F3C014D013CE095948794779467943C
:107550003A95D1F76092DD027092DE028092DF02EE
:107560009092E002C801B7012D813E814F8158857C
:107570000E94F37797FF04C06150784F8F4F9F4F61
:107580002BE095958795779567952A95D1F7A60174
:1075900095010E94F377DC01CB018093E102909387
:1075A000E202A093E302B093E402B7FF04C081506B
:1075B000904FAF4FBF4FAC01BD018CE07595679503
:1075C000579547958A95D1F74093E1025093E2028F
:1075D0006093E3027093E4022A893B8937FF03C07A
:1075E000309521953F4F21343105E4F1D401C30199
:1075F00097FE07C0B095A095909581959F4FAF4F8E
:10760000BF4F81389105A105B10584F4DB01CA01A2
:1076100077FF07C0B095A095909581959F4FAF4F8C
:10762000BF4F81389105A105B105E4F081E0809359
:10763000800218C0109251071092500710924D0707
:1076400010924C071092E1021092E2021092E302B3
:107650001092E4021092DD021092DE021092DF021C
:107660001092E0028091E1029091E202A091E30287
:10767000B091E402BC01CD0124E630E040E050E0EE
:107680000E946778E090DD02F090DE02E21AF30AD1
:10769000F0926407E09263078091DD029091DE0230
:1076A000A091DF02B091E002BC01CD0124E630E000
:1076B00040E050E00E946778DA01C9012091E102C0
:1076C0003091E2028C01021B130B109358070093B8
:1076D00057078091430190914401A0914501B091D9
:1076E0004601BC01CD0128E631E040E050E00E94B7
:1076F000F3772091AD073091AE074091AF075091DD
:10770000B007261737074807590764F0261B370BC1
:10771000480B590B2093AD073093AE074093AF074A
:107720005093B0072091AD073091AE074091AF075D
:107730005091B00757FF0CC0260F371F481F591F25
:107740002093AD073093AE074093AF075093B00737
:1077500060915507709156076E0D7F1D9B01442760
:1077600037FD4095542F8091980290919902A091F5
:107770009A02B0919B02820F931FA41FB51F8093A2
:10778000980290939902A0939A02B0939B028091E1
:10779000540290915502681B790BCB01AA2797FDE3
:1077A000A095BA2F29853A854B855C85820F931F5A
:1077B000A41FB51F80939C0290939D02A0939E02EC
:1077C000B0939F02C0908301D0908401E090850126
:1077D000F0908601C816D906EA06FB06C4F488EACA
:1077E00091E6A0E0B0E08C199D09AE09BF09809335
:1077F0009C0290939D02A0939E02B0939F0280935F
:10780000980290939902A0939A02B0939B02222728
:107810003327A9012C193D094E095F0980919C026B
:1078200090919D02A0919E02B0919F0282179307B2
:10783000A407B507B4F4D701C601885A9146A04001
:10784000B04080939C0290939D02A0939E02B093BF
:107850009F028093980290939902A0939A02B0930A
:107860009B026091650770916607600F711F9B0115
:10787000442737FD4095542F8091A0029091A1029A
:10788000A091A202B091A302820F931FA41FB51F63
:107890008093A0029093A102A093A202B093A302AE
:1078A0008091520290915302681B790BCB01AA2759
:1078B00097FDA095BA2F2D853E854F855889820F5B
:1078C000931FA41FB51F8093A4029093A502A093B9
:1078D000A602B093A702E0908701F0908801009182
:1078E000890110918A01E816F9060A071B07C4F4FA
:1078F00088EA91E6A0E0B0E08E199F09A00BB10BD9
:107900008093A4029093A502A093A602B093A7022D
:107910008093A0029093A102A093A202B093A3022D
:1079200022273327A9012E193F09400B510B8091C3
:10793000A4029091A502A091A602B091A70282177D
:107940009307A407B507B4F4D801C701885A914634
:10795000A040B0408093A4029093A502A093A602F9
:10796000B093A7028093A0029093A102A093A202D9
:10797000B093A3028091940290919502A0919602F7
:10798000B09197028093A8029093A902A093AA02B3
:10799000B093AB028091A4029091A502A091A6029F
:1079A000B091A7028093C4029093C502A093C6022F
:1079B000B093C70280919C0290919D02A0919E027B
:1079C000B0919F028093BC029093BD02A093BE022F
:1079D000B093BF028091A0029091A102A091A20257
:1079E000B091A3028093C0029093C102A093C202FF
:1079F000B093C3028091980290919902A0919A024B
:107A0000B0919B028093B8029093B902A093BA02FE
:107A1000B093BB0280911C0190911D0197FD0796C8
:107A200003E0959587950A95E1F790936607809313
:107A3000650780911A0190911B0197FD079613E04D
:107A4000959587951A95E1F790935607809355077A
:107A50008091FD019091FE010F9734F488E19CEF35
:107A600090936607809365078091FD019091FE01D8
:107A7000079734F480E398EF909366078093650747
:107A8000209102012A30A9F48091FD019091FE011C
:107A9000835F934034F088EE93E090936607809381
:107AA00065078091FD019091FE018A5F9340DCF0B3
:107AB00014C08091FD019091FE01815D974034F0EA
:107AC00088EE93E090936607809365078091FD01AF
:107AD0009091FE01805E974034F080ED97E09093A6
:107AE0006607809365078091FB019091FC010F97D9
:107AF00034F488E19CEF909356078093550780916A
:107B0000FB019091FC01079734F480E398EF909388
:107B10005607809355072A30A9F48091FB01909174
:107B2000FC01835F934034F088EE93E09093560716
:107B3000809355078091FB019091FC018A5F9340EF
:107B4000DCF014C08091FB019091FC01815D9740B5
:107B500034F088EE93E09093560780935507809118
:107B6000FB019091FC01805E974034F080ED97E03E
:107B7000909356078093550760917501662309F429
:107B8000AFC040911C0150911D018091ED02909178
:107B9000EE02481B590B5093F4024093F3022091DC
:107BA0001C0130911D01280F391F37FF02C02F5FC4
:107BB0003F4F359527953093EE022093ED024138E3
:107BC00051051CF080E890E005C040585F4F34F448
:107BD00080E89FEF9093F4028093F30240911A01A2
:107BE00050911B018091EF029091F002481B590BBC
:107BF0005093F2024093F10220911A0130911B013F
:107C0000280F391F37FF02C02F5F3F4F359527954B
:107C10003093F0022093EF02413851051CF080E8C8
:107C200090E005C040585F4F34F480E89FEF909398
:107C3000F2028093F102462F55278091F302909132
:107C4000F402849FB001859F700D949F700D1124E4
:107C50009B0177FF02C0215F3F4FF4E035952795E8
:107C6000FA95E1F78091650790916607820F931F5F
:107C700090936607809365078091F1029091F202DC
:107C8000849FD001859FB00D949FB00D1124AD014C
:107C90009D01B7FF02C0215F3F4FE4E03595279576
:107CA000EA95E1F78091550790915607820F931F4F
:107CB000909356078093550780911C0190911D0168
:107CC000860F971F90931D0180931C0180911A01CC
:107CD00090911B01840F951F90931B0180931A01B3
:107CE000009168071091690780914C0790914D07AA
:107CF000101611065CF59C0197FF04C0222733275C
:107D0000281B390BC901AA2797FDA095BA2F2091EE
:107D10006901332744275527BC01CD010E94F37721
:107D20009B01AC0197FF04C0215C3F4F4F4F5F4F59
:107D300076E055954795379527957A95D1F78091B7
:107D4000630790916407820F931F27C097FF03C0BA
:107D5000909581959F4FAA2797FDA095BA2F2091C6
:107D60006901332744275527BC01CD010E94F377D1
:107D70009B01AC0197FF04C0215C3F4F4F4F5F4F09
:107D800066E055954795379527956A95D1F7809187
:107D9000630790916407821B930B90936407809311
:107DA0006307E0907007F090710780915007909101
:107DB00051071E141F045CF59C0197FF04C0222785
:107DC0003327281B390BC901AA2797FDA095BA2F85
:107DD00020916901332744275527BC01CD010E941A
:107DE000F3779B01AC0197FF04C0215C3F4F4F4FDD
:107DF0005F4F96E055954795379527959A95D1F71A
:107E00008091570790915807820F931F27C097FFC3
:107E100003C0909581959F4FAA2797FDA095BA2FF3
:107E200020916901332744275527BC01CD010E94C9
:107E3000F3779B01AC0197FF04C0215C3F4F4F4F8C
:107E40005F4F86E055954795379527958A95D1F7E9
:107E50008091570790915807821B930B9093580776
:107E60008093570780919D0787FF44C0B989BB2342
:107E700009F040C080914E028823E1F5E1E0EE1662
:107E8000E1E0FE064CF080916507909166078E0D4B
:107E90009F1D805091400DC0F0E0EF16FFEFFF06F0
:107EA00064F480916507909166078E0D9F1D805048
:107EB0009F4F909366078093650721E0013012077A
:107EC0004CF08091550790915607800F911F80507C
:107ED00091400CC03FEF0030130764F480915507C8
:107EE00090915607800F911F80509F4F9093560797
:107EF00080935507E2E1CD5E0C949E7880916902F3
:107F0000882301F5809134028C7F80933402A3E9A9
:107F1000B3E0E3E8F6E09BE08091B901882309F43F
:107F20008C938D91818312829150389697FFF4CF74
:107F30008091B901882359F08091B90181508093D3
:107F4000B90105C080913402816080933402809130
:107F50002402882319F010922402089580932602A7
:107F600080932802809122028E7F8093220285EAEC
:107F70008093BC000895CF93DF93ABE6B2E0CAEBE9
:107F8000D5E057E09991E92FFF27EE0FFF1FEC5145
:107F9000F94F0190F081E02DE158FF4FEF3FF105DF
:107FA00021F01CF0EFEFF0E004C0F7FF02C0E0E0CA
:107FB000F0E0993111F4EC931BC04C91242F33273E
:107FC000E217F307A9F0CF01821B930B97FD0396ED
:107FD0009595879595958795242F280F2C93822F1B
:107FE0009927E817F90714F4215001C02F5F2C934B
:107FF0005150119657FFC6CF8091C405883F38F085
:10800000EFEFF0E0E81BF109E559FD4F8081809327
:108010007B0180917B01882329F0843618F084E667
:1080200080937B018091C605883F38F0EFEFF0E048
:10803000E81BF109E559FD4F80818093790180911A
:108040007901882329F0843618F084E68093790139
:108050008091D305883F38F0EFEFF0E0E81BF1099D
:10806000E559FD4F808180937401809174018B30BC
:1080700010F48AE002C08F3F11F480937401809164
:108080000006883F38F0EFEFF0E0E81BF109E55912
:10809000FD4F808180937C0780917C07863010F4AF
:1080A00085E002C08F3F11F480937C078091020627
:1080B000883F38F0EFEFF0E0E81BF109E559FD4F9C
:1080C00080818093A4078091A407863010F485E016
:1080D00002C08F3F11F48093A4078091ED05883F83
:1080E00038F0EFEFF0E0E81BF109E559FD4F808132
:1080F000809379078091EE05883F38F0EFEFF0E04C
:10810000E81BF109E559FD4F80818093520780916A
:10811000EF05883F38F0EFEFF0E0E81BF109E55993
:10812000FD4F8081809382078091C505883F38F09C
:10813000EFEFF0E0E81BF109E559FD4F80818093F6
:108140007A018091C805883F38F0EFEFF0E0E81B36
:10815000F109E559FD4F8081809378018091CA052E
:10816000883F38F0EFEFF0E0E81BF109E559FD4FEB
:108170008081809376018091D205883F38F0EFEFBF
:10818000F0E0E81BF109E559FD4F8081809377010C
:108190008091D405883F38F0EFEFF0E0E81BF1095B
:1081A000E559FD4F8081809373018091D505883F0B
:1081B00038F0EFEFF0E0E81BF109E559FD4F808161
:1081C000809375018091D605883F38F0EFEFF0E09D
:1081D000E81BF109E559FD4F808180937201809180
:1081E000D705883F38F0EFEFF0E0E81BF109E559DB
:1081F000FD4F8081809371018091DD05883F38F0CB
:10820000EFEFF0E0E81BF109E559FD4F8081809325
:108210006F018091DE05883F38F0EFEFF0E0E81B5A
:10822000F109E559FD4F8081809349028091DF0576
:10823000883F38F0EFEFF0E0E81BF109E559FD4F1A
:108240008081809348028091E005883F38F0EFEF0D
:10825000F0E0E81BF109E559FD4F8081809347026A
:108260008091E105883F38F0EFEFF0E0E81BF1097D
:10827000E559FD4F8081809346028091FB05883F40
:1082800038F0EFEFF0E0E81BF109E559FD4F808190
:10829000809345028091FC05883F38F0EFEFF0E0D5
:1082A000E81BF109E559FD4F8081809344028091DC
:1082B000FD05883F38F0EFEFF0E0E81BF109E559E4
:1082C000FD4F8081809343028091FE05883F38F006
:1082D000EFEFF0E0E81BF109E559FD4F8081809355
:1082E00042028091E205883F38F0EFEFF0E0E81BB2
:1082F000F109E559FD4F808180936E018091E6057B
:10830000883F38F0EFEFF0E0E81BF109E559FD4F49
:10831000808180936D018091F005883F38F0EFEF08
:10832000F0E0E81BF109E559FD4F808180936C0175
:108330008091F305883F38F0EFEFF0E0E81BF1099A
:10834000E559FD4F808180936B018091F405883F52
:1083500038F0EFEFF0E0E81BF109E559FD4F8081BF
:1083600080936A018091F505883F38F0EFEFF0E0E7
:10837000E81BF109E559FD4F8081809369018091E7
:108380001C06883F38F0EFEFF0E0E81BF109E559F3
:10839000FD4F8081809361078091C20580939D0786
:1083A00080911F06809381078091FA05883F38F0FD
:1083B000EFEFF0E0E81BF109E559FD4F8081809374
:1083C000680180911506883F38F0EFEFF0E0E81B78
:1083D000F109E559FD4F80818093B40780916F01C9
:1083E000282F33272F5F3F4F8CE398E2B9010E947B
:1083F000327870937D0160937C018091D0058093E9
:10840000A5078091CF0580936A0790911706933353
:10841000C8F181E080934102983F58F0EFEFF0E01F
:10842000E91BF109E559FD4F8081823310F4109268
:10843000410280917E0120914102821799F08330A0
:1084400070F4222319F08CED95E002C088EC90E0E6
:108450009093DB018093DA0120937E0103C0815069
:1084600080937E018091F4079091F50797FF0FC0EC
:1084700080914102882359F080918E038068809317
:108480008E0305C0109241028AE080937E018091A4
:10849000F4079091F50797FF1DC08091690288232A
:1084A000C9F0809141028823A9F080910801909140
:1084B00009018F5F9F4F71F488E99AE39093DB0184
:1084C0008093DA0180E094EA909309018093080197
:1084D0001092410280914102882369F08091330219
:1084E00081608093330280916B01823D48F4825E0B
:1084F00080936B0105C0809133028E7F809333029D
:10850000DF91CF910895A7E1B0E0E9E8F2E40C949F
:1085100082780E94CC37E0907402F0907502FA8263
:10852000E98280916A0799270A96E816F90614F4F9
:108530009A83898380916A02843608F066C08091AC
:10854000330282FD62C08091090390910A03009773
:1085500031F0019790930A03809309030BC01092A6
:1085600069029093360280933502809134028D7EA9
:1085700080933402809102018A3011F0843110F02E
:10858000289A01C028988091350290913602895E20
:108590009340C0F18091DA05282F33273A8329834D
:1085A000809134028061809334028091B605A82FB7
:1085B000BB27AA0FBB1FFD01E85EF84F1182108296
:1085C0008091B705282F3327220F331FC901885EFA
:1085D000984FFC0111821082AC51B94F11961C9238
:1085E0001E922C51394FD90111961C921E928091E6
:1085F000B905E82FFF27EE0FFF1FEC51F94F11824D
:108600001082A9C210926902A6C280916A028D38B6
:1086100008F4A1C2809134028F7E8093340290913D
:10862000DB0582E3989FC001112490930A03809395
:108630000903E981FA81B9978CF080916902882356
:1086400069F08091350290913602FFEF8F3F9F07CE
:1086500029F001969093360280933502809135027D
:10866000909136028F3F910509F008F510928C0227
:1086700010928D0210928E0210928F021092880238
:108680001092890210928A0210928B021092F502C7
:108690001092F6021092F7021092F80210929402D1
:1086A00010929502109296021092970205C0809146
:1086B00034028260809334028091B805E82FFF274E
:1086C000EE0FFF1FEC51F94F8081918181359105AB
:1086D0000CF435C120916902222309F030C1809148
:1086E000B905E82FFF27EE0FFF1FEC51F94F8081EE
:1086F00091818C3491050CF4FFC080910B038F5F46
:1087000080930B03893C08F41AC120930B03109249
:108710003602109235023091B605E32FFF27EE0F97
:10872000FF1FEC51F94F8081918187349105B4F49A
:108730008091B705E82FFF27EE0FFF1FEC51F94F8F
:10874000808191810190F081E02DF7FF03C0F095C9
:10875000E195FF4FE734F1050CF478C041E020913A
:10876000B705A22FBB27AA0FBB1FAC51B94F8D91E4
:108770009C9111978734910544F0E32FFF27EE0F6A
:10878000FF1FEC51F94F808191818D919C9187342D
:10879000910574F08091B605E82FFF27EE0FFF1FBB
:1087A000EC51F94F80819181873491050CF042E0C2
:1087B000E22FFF27EE0FFF1FEC51F94F80819181CF
:1087C0008634910574F48091B605E82FFF27EE0FEB
:1087D000FF1FEC51F94F80819181873491050CF096
:1087E00043E0E22FFF27EE0FFF1FEC51F94F80818E
:1087F00091818A5B9F4F74F48091B605E82FFF2723
:10880000EE0FFF1FEC51F94F808191818734910564
:108810000CF044E0E22FFF27EE0FFF1FEC51F94F61
:10882000808191818A5B9F4F74F48091B605E82F17
:10883000FF27EE0FFF1FEC51F94F808191818634A5
:1088400091050CF445E0842F0E944D2B8091B705D3
:10885000E82FFF27EE0FFF1FEC51F94F8081918128
:108860000190F081E02DF7FF03C0F095E195FF4FF7
:108870007E97BCF48091B605E82FFF27EE0FFF1F0F
:10888000EC51F94F808191818A5B9F4F54F481E0D4
:108890008093A90388EE93E09093DB018093DA0143
:1088A0004EC00E94492C0E94FA2A80E00E94D706FE
:1088B0008091DC050E94757380919D0780FF10C038
:1088C0008091140190911501875B934038F4809159
:1088D0001401909115018E5E924010F40E94581A76
:1088E0001092D80180E00E941A3581E080930E0337
:1088F0008093D801579A1AC080819181855B9F4FE0
:10890000E4F480910B038F5F80930B03893CB8F0F4
:108910002093690220930B031092360210923502C5
:1089200081E00E941A3581E080930E030E94492C59
:1089300068E770E00E944B3402C020930B038091E3
:10894000B805E82FFF27EE0FFF1FEC51F94F80818C
:1089500091818B5A9F4F0CF0FEC030916902E091DB
:10896000B905332309F0CCC0FF27EE0FFF1FEC51F0
:10897000F94F80819181855B9F4F0CF0BEC02091A3
:108980001806E22FFF27EE0FFF1FEC51F94F8081F1
:108990009181855B9F4F1CF0222309F0AEC080912E
:1089A0000C038F5F80930C03893C08F4D4C0309390
:1089B0000C0380918E03882309F098C080910E03E8
:1089C000882309F493C080914403882309F08EC062
:1089D00081E090E0909336028093350281E08093AD
:1089E00069021092F5021092F6021092F7021092AC
:1089F000F802109294021092950210929602109230
:108A0000970210929002109291021092920210928C
:108A100093028091D105E82EFF2400271127809131
:108A2000A1079091A2079C01442737FD4095542F40
:108A3000C801B7010E94F377DC01CB018093A40247
:108A40009093A502A093A602B093A7028091B107CC
:108A50009091B2079C01442737FD4095542FC801DF
:108A6000B7010E94F377DC01CB0180939C029093C5
:108A70009D02A0939E02B0939F028091C4029091A8
:108A8000C502A091C602B091C7028093A002909344
:108A9000A102A093A202B093A3028091BC02909184
:108AA000BD02A091BE02B091BF0280939802909344
:108AB0009902A0939A02B0939B0210928C0210929A
:108AC0008D0210928E0210928F02109288021092E4
:108AD000890210928A0210928B028091340288607F
:108AE0008093340284E680930F0335C08CED95E0CB
:108AF0009093DB018093DA012EC010920C032BC0FF
:108B0000FF27EE0FFF1FEC51F94F808191818C34CC
:108B10009105FCF020911806E22FFF27EE0FFF1FB2
:108B2000EC51F94F80819181855B9F4F14F0222396
:108B300081F480910D038F5F80930D03893C58F081
:108B40001092690210920D031092360210923502B3
:108B500002C010920D038091410181508093410128
:108B6000809141018F3F21F08091340284FFA9C39D
:108B70000E94BB3FB090CC058091180390911903DF
:108B80009C01220F331F280F391FC090B605AC2D52
:108B9000BB27AA0FBB1FFD01EC51F94F4B2D5527E9
:108BA00080819181849FF001859FF00D949FF00D4D
:108BB00011242E0F3F1F37FF02C02D5F3F4FB90119
:108BC0007595679575956795A85EB84F8091CD05A9
:108BD000082F11278D919C91809F7001819FF00C2F
:108BE000909FF00C11246E0D7F1D709319036093FC
:108BF000180380911A0390911B039C01220F331FCD
:108C0000280F391FD090B705AD2DBB27AA0FBB1F6A
:108C1000FD01EC51F94F80819181849FF001859F86
:108C2000F00D949FF00D11242E0F3F1F37FF02C04F
:108C30002D5F3F4FA9015595479555954795A85EDE
:108C4000B84F8D919C91809F7001819FF00C909FF7
:108C5000F00C11244E0D5F1D50931B0340931A031B
:108C600080914102882309F448C0CB0177FD039627
:108C7000DC01B595A795B595A795CA0157FD039653
:108C8000FC01F595E795F595E79580919D01682F95
:108C9000772767FD70956A9F90016B9F300D7A9FD3
:108CA000300D112480914603482F552747FD5095DC
:108CB0004E9FC0014F9F900D5E9F900D1124280F75
:108CC000391F37FF02C0295F3F4F93E03595279545
:108CD0009A95E1F730937B0220937A026E9F900180
:108CE0006F9F300D7E9F300D11244A9FC0014B9F16
:108CF000900D5A9F900D11243FC080911606E82FC9
:108D0000FF27E75BFE4F868180939D0190819093C2
:108D10004603A82FBB27A7FDB095A69F9001A79F4C
:108D2000300DB69F300D1124E92FFF27E7FDF09598
:108D3000E49FC001E59F900DF49F900D1124280F32
:108D4000391F37FF02C0295F3F4F83E035952795D4
:108D50008A95E1F730937B0220937A02A49F9001D9
:108D6000A59F300DB49F300D1124E69FC001E79FF1
:108D7000900DF69F900D1124281B390B37FF02C070
:108D8000295F3F4F03E0359527950A95E1F730932A
:108D90007902209378028091B905E82FFF27EE0F22
:108DA000FF1FEC51F94F80819181909581959F4FE4
:108DB00090937702809376028530910514F00497A2
:108DC00005C00FEF8C3F900734F404969093770220
:108DD0008093760204C010927702109276028091FE
:108DE0003403882309F43EC0282F332780917A0268
:108DF00090917B0297FD079613E0959587951A95BC
:108E0000E1F7289FA001299F500D389F500D112494
:108E1000CA0157FD0F96B4E095958795BA95E1F78D
:108E200090937B0280937A028091780290917902EC
:108E300097FD0796A3E095958795AA95E1F7289F5A
:108E4000B001299F700D389F700D1124CB0177FD63
:108E50000F96F4E095958795FA95E1F7909379024E
:108E60008093780280907A0290907B028091370301
:108E700090913803881A990A90927B0280927A0224
:108E80000091780210917902809135039091360318
:108E9000081B190B10937902009378028091B80592
:108EA000E82FFF27EE0FFF1FEC51F94FE080F18014
:108EB0008FE790E0E80EF91EF0927502E0927402DE
:108EC000809174019927AA2797FDA095BA2FBC011C
:108ED000CD010E946777DC01CB0120E030E040E269
:108EE00051E4BC01CD010E94D576DC01CB01BC016F
:108EF000CD010E943977DC01CB018093AB078091D3
:108F0000730180938307809172019927AA2797FDA7
:108F1000A095BA2FBC01CD010E946777DC01CB017F
:108F200020E030E040E251E4BC01CD010E94D57662
:108F3000DC01CB01BC01CD010E943977DC01CB0102
:108F400080935C0780917101809372078091B503D3
:108F500080FF59C08091B407813808F454C08091D3
:108F6000AE03992787FD90952B2D3327829FD00143
:108F7000839FB00D929FB00D11248A0E9B1E90927C
:108F80007B0280927A028091AF03992787FD9095AA
:108F9000829FF001839FF00D929FF00D11240E0F20
:108FA0001F1F10937902009378028091B003282F3D
:108FB000332727FD30958091760290917702820FBA
:108FC000931F90937702809376028091B203282FAB
:108FD000332727FD30958091C7059927289F800169
:108FE000299F100D389F100D1124109348010093F4
:108FF00047018091B10399278E159F0524F4909322
:10900000750280937402809174029091750297FFAB
:1090100004C0109275021092740280919D0782FF25
:1090200002C01092830740917A0250917B02CA01DC
:1090300057FD03969C01359527953595279537FF64
:1090400003C0309521953F4F8091390290913A02AB
:1090500082179307B4F4CA0157FF03C09095819516
:109060009F4F97FD03969595879595958795909336
:109070003A02809339028536910544F084E690E007
:1090800001C0019790933A0280933902409178028F
:1090900050917902CA0157FD03969C013595279599
:1090A0003595279537FF03C0309521953F4F809127
:1090B00037029091380282179307B4F4CA0157FF20
:1090C00003C0909581959F4F97FD03969595879541
:1090D0009595879590933802809337028536910550
:1090E00044F084E690E001C00197909338028093A9
:1090F00037028091340284FF08C010923A02109225
:1091000039021092380210923702ED2DFF27EE0F30
:10911000FF1FEC51F94F4091F105242F3327808137
:1091200091812817390744F480911D0682FF04C0FD
:1091300081E080934D0213C0ED2DFF27EE0FFF1F3E
:10914000EC51F94F842F99272091F205821B910948
:10915000208131812817390714F410924D02409173
:10916000B705E42FFF27EE0FFF1FEC51F94F509189
:10917000F105852F992722273327281B390B80815A
:1091800091818217930744F480911D0683FF04C0E8
:1091900081E080934C0216C080914C02882391F0AC
:1091A000E42FFF27EE0FFF1FEC51F94F8091F205DE
:1091B0009927851B9109208131818217930714F427
:1091C00010924C02EC2DFF27EE0FFF1FEC51F94FD0
:1091D0004091F105242F3327808191812817390789
:1091E00044F480911D0680FF04C081E080934A0210
:1091F00017C080914A02882399F0EC2DFF27EE0FCB
:10920000FF1FEC51F94F842F99272091F205821B03
:109210009109208131812817390714F410924A02EC
:109220004091B605E42FFF27EE0FFF1FEC51F94FD9
:109230005091F105852F992722273327281B390BB9
:10924000808191818217930744F480911D0681FFEC
:1092500004C081E080934B0216C080914B028823AA
:1092600091F0E42FFF27EE0FFF1FEC51F94F809193
:10927000F2059927851B9109208131818217930777
:1092800014F410924B0280914D02882319F48091BE
:109290004C02811181E080934E0280914A02882322
:1092A00021F480914B02882351F081E080934F029A
:1092B00010924E0210924D0210924C0202C0809306
:1092C0004F0280914E02882321F480914F0288231F
:1092D00069F08091F005992729813A8182179307D7
:1092E00014F49A83898381E0809380028091330211
:1092F00099279C012470307082FF2DC08091370324
:1093000090913803909581959F4F90937B02809325
:109310007A028091350390913603909581959F4F05
:1093200090937902809378028091810190918201DB
:10933000909375028093740280919D078B778B6662
:1093400080939D07809181078C7B8093810788ECB7
:1093500080937A011EC08091340284FF1AC030933A
:1093600077022093760230937B0220937A02309327
:109370007902209378029AE59093AB0788E780936F
:10938000830790935C078093720710924E021092AD
:109390004F028091750790917607A0917707B09161
:1093A00078072091C4023091C5024091C6025091C5
:1093B000C702820F931FA41FB51F80937507909358
:1093C0007607A0937707B093780780917D079091F7
:1093D0007E07A0917F07B0918007E090BC02F090DB
:1093E000BD020091BE021091BF02EB82FC820D8390
:1093F0001E838E0D9F1DA01FB11F80937D0790932C
:109400007E07A0937F07B093800780916C079091AF
:109410006D07A0916E07B0916F07E090C002F090C9
:10942000C1020091C2021091C302EF82F88609873F
:109430001A878E0D9F1DA01FB11F80936C079093FC
:109440006D07A0936E07B0936F0780915D079091B1
:109450005E07A0915F07B0916007E090B802F090BE
:10946000B9020091BA021091BB02EB86FC860D870F
:109470001E878E0D9F1DA01FB11F80935D079093C7
:109480005E07A0935F07B0936007F0904F02FF86DE
:10949000FF2029F480914E02882309F460C01092C5
:1094A000B4021092B5021092B6021092B702109256
:1094B000B0021092B1021092B2021092B302109256
:1094C000750710927607109277071092780710921E
:1094D0007D0710927E0710927F07109280071092EE
:1094E0006C0710926D0710926E0710926F07109222
:1094F0005D0710925E0710925F07109260078091DF
:10950000A4029091A502A091A602B091A702809317
:10951000A0029093A102A093A202B093A302809113
:109520009C0290919D02A0919E02B0919F02809317
:10953000980290939902A0939A02B0939B02109282
:10954000EA011092E9011092530210925202109215
:109550005502109254020F85002309F0F8C1809142
:109560004E02882309F0F3C1809157059091580568
:10957000815092402CF480916902882309F4E7C15C
:1095800090902D08A090D1052090A1073090A207BF
:109590004090B1075090B20719140CF0E3C0BB24FF
:1095A000CC24DD24CA01B901A60195010E94677887
:1095B00079018A018091F6079091F707281A390AF4
:1095C000C101AA2797FDA095BA2FE81AF90A0A0B3C
:1095D0001B0B6B817C818D819E81A60195010E9470
:1095E000677859016A018091F8079091F907481A44
:1095F000590AC201AA2797FDA095BA2FA81AB90A3D
:10960000CA0ADB0A292C332427FC3094432C532C20
:10961000C801B701A20191010E94F37797FF04C02E
:1096200061507E4F8F4F9F4F3B014C0109E0959455
:109630008794779467940A95D1F7C601B501A20182
:1096400091010E94F37797FF04C061507E4F8F4FC6
:109650009F4F5B016C0119E0D594C794B794A79410
:109660001A95D1F78091390290913A02813491058F
:109670003CF4809137029091380281349105D4F006
:10968000D401C30197FE03C00196A11DB11D3C0189
:109690004D019594879477946794D601C501D7FEC0
:1096A00003C00196A11DB11D5C016D01D594C79445
:1096B000B794A7948091B905E82FFF27EE0FFF1FFD
:1096C000EC51F94F808191810190F081E02DF7FFFD
:1096D00003C0F095E195FF4F7A97A4F0C401B30160
:1096E00023E030E040E050E00E94677839014A0111
:1096F000C601B50123E030E040E050E00E94677809
:1097000059016A0180912F08282F332727FD3095B2
:10971000432F532F261537054805590514F43901F1
:109720004A01992787FD9095909581959F4FAA278B
:1097300097FDA095BA2F681679068A069B0614F441
:109740003C014D012A153B054C055D0514F45901FA
:109750006A01A816B906CA06DB060CF0D0C05C0187
:109760006D01CDC0EA2CFF2400271127CA01B901E1
:10977000A80197010E94677839014A01C101AA270F
:1097800097FDA095BA2F681A790A8A0A9B0A6B81FD
:109790007C818D819E81A80197010E946778590183
:1097A0006A01C201AA2797FDA095BA2FA81AB90A83
:1097B000CA0ADB0AD401C30197FE03C00F96A11D9C
:1097C000B11D3C014D01F4E0959487947794679422
:1097D000FA95D1F7D601C501D7FE03C00F96A11D9A
:1097E000B11D5C016D01E4E0D594C794B794A794D2
:1097F000EA95D1F78091390290913A02813491052E
:109800003CF4809137029091380281349105A4F0A4
:10981000C401B30123E030E040E050E00E946778EB
:1098200039014A01C601B50123E030E040E050E0D3
:109830000E94677859016A018091B905E82FFF27D6
:10984000EE0FFF1FEC51F94F808191810190F08163
:10985000E02DF7FF03C0F095E195FF4F7A97A4F054
:10986000C401B30123E030E040E050E00E9467789B
:1098700039014A01C601B50123E030E040E050E083
:109880000E94677859016A0189E180938D0121E284
:1098900062167104810491042CF070E2672E712C21
:1098A000812C912C30EE63163FEF73063FEF830659
:1098B0003FEF930644F460EE662E6FEF762E6FEF67
:1098C000862E6FEF962E41E2A416B104C104D10496
:1098D0002CF050E2A52EB12CC12CD12C50EEA516A7
:1098E0005FEFB5065FEFC5065FEFD50644F440EEC7
:1098F000A42E4FEFB42E4FEFC42E4FEFD42E8091F5
:10990000A4029091A502A091A602B091A702861987
:109910009709A809B9098093A4029093A502A0937E
:10992000A602B093A70280919C0290919D02A09103
:109930009E02B0919F028A199B09AC09BD098093D0
:109940009C0290939D02A0939E02B0939F028091EF
:10995000E9019091EA018F3F910509F008F4C4C52F
:109960006F85662309F04EC580914E02882309F069
:1099700049C580918002882309F044C57091F9059A
:10998000788B772309F43EC580917507909176070F
:10999000A0917707B0917807B7FF04C081509F4F1F
:1099A000AF4FBF4FE92EFA2E0B2F112707FD1A9547
:1099B000E0927507F0927607009377071093780787
:1099C00080917D0790917E07A0917F07B0918007DD
:1099D000B7FF04C081509F4FAF4FBF4F892F9A2FC1
:1099E000AB2FBB27A7FDBA95898B9A8BAB8BBC8B12
:1099F00080937D0790937E07A0937F07B0938007A5
:109A00008091D105A82EBB24CC24DD242091B40262
:109A10003091B5024091B6025091B702C601B5012E
:109A20000E94F37797FF04C061507F4F8F4F9F4F85
:109A3000672E782E892E992487FC9A946092B4021E
:109A40007092B5028092B6029092B7022091B00255
:109A50003091B1024091B2025091B302C601B501FA
:109A60000E94F37797FF04C061507F4F8F4F9F4F45
:109A7000272E382E492E552447FC5A942092B002A6
:109A80003092B1024092B2025092B3028091AC0285
:109A90009091AD02A091AE02B091AF02B7FF04C0A9
:109AA00081509F4FAF4FBF4F892F9A2FAB2FBB27AE
:109AB000A7FDBA958093AC029093AD02A093AE023D
:109AC000B093AF02D801C70186199709A809B9094F
:109AD0008093010390930203A0930303B0930403C4
:109AE0002091F805E22EFF2400271127BC01CD01AB
:109AF000A80197010E94677859016A012093100319
:109B000030931103409312035093130389899A8968
:109B1000AB89BC8982199309A409B509809305030F
:109B200090930603A0930703B0930803BC01CD01F3
:109B3000A80197010E9467782093140330931503BE
:109B40004093160350931703D601C501D7FE04C0F6
:109B500081509F4FAF4FBF4F892F9A2FAB2FBB27FD
:109B6000A7FDBA95909353028093520257FF04C009
:109B700021503F4F4F4F5F4FBB2757FDBA95A52F41
:109B8000942F832F90935502809354028091390231
:109B900090913A0281349105DCF4809137029091E2
:109BA000380281349105A4F48091B905E82FFF278C
:109BB000EE0FFF1FEC51F94F808191810190F081F0
:109BC000E02DF7FF03C0F095E195FF4F7A97E4F0A1
:109BD00080912D088F3FC1F48091520290915302E1
:109BE00097FD019695958795909353028093520225
:109BF000809154029091550297FD01969595879515
:109C0000909355028093540280916C0790916D0758
:109C1000A0916E07B0916F07B7FF04C081509F4FAE
:109C2000AF4FBF4F892F9A2FAB2FBB27A7FDBA95F8
:109C300080936C0790936D07A0936E07B0936F07A6
:109C400080915D0790915E07A0915F07B0916007DA
:109C5000B7FF04C081509F4FAF4FBF4F892F9A2F3E
:109C6000AB2FBB27A7FDBA9580935D0790935E0746
:109C7000A0935F07B09360078091C4029091C502E2
:109C8000A091C602B091C7022F81388549855A85B7
:109C9000281B390B4A0B5B0B2093F9023093FA0215
:109CA0004093FB025093FC028091BC029091BD0254
:109CB000A091BE02B091BF02EB84FC840D851E858D
:109CC000E81AF90A0A0B1B0BE092FD02F092FE0261
:109CD0000093FF02109300032093010330930203CB
:109CE0004093030350930403E0920503F0920603AC
:109CF00000930703109308038091A0029091A102A2
:109D0000A091A202B091A302821B930BA40BB50BEE
:109D10008093A0029093A102A093A202B093A30209
:109D20008091980290919902A0919A02B0919B0221
:109D30008E199F09A00BB10B809398029093990202
:109D4000A0939A02B0939B0288898823E1F0209126
:109D50007E0230917F02213831054CF08091D5028E
:109D60009091D60201969093D6028093D502205806
:109D70003F4F4CF48091D5029091D6020197909379
:109D8000D6028093D50210927F0210927E0281E06B
:109D900090E090931D0380931C03E0900103F090EA
:109DA00002030091030310910403D801C70117FFB8
:109DB00007C088279927DC018E199F09A00BB10BDA
:109DC00081509240A040B04034F084E090E0909305
:109DD0001D0380931C038091220390912303A09183
:109DE0002403B091250320917507309176074091A7
:109DF000770750917807821B930BA40BB50B815EFC
:109E0000914BAF4FBF4F8F539C49A040B04028F0BB
:109E100080912E0889310CF4FFC021E0E21620E188
:109E2000F20620E0020720E012070CF473C08091D4
:109E30001E03882309F46AC0D801C70117FF07C0B1
:109E400088279927DC018E199F09A00BB10B9C0173
:109E5000AD01B7FF04C021503E4F4F4F5F4FF9E0B7
:109E60005595479537952795FA95D1F780911C031D
:109E700090911D03820F931F90931D0380931C03E9
:109E8000D801C70117FF03C00796A11DB11DE3E06C
:109E9000B595A79597958795EA95D1F78093100387
:109EA00090931103A0931203B09313038958934125
:109EB000A040B04064F088E893E1A0E0B0E0809377
:109EC000100390931103A0931203B09313032091F6
:109ED000100330911103409112035091130357FF67
:109EE00004C021503F4F4F4F5F4F232F342F452F3A
:109EF000552747FD5A958091520290915302820F47
:109F0000931F909353028093520206C081E0809386
:109F10001E0302C010921E0340E0E41640EFF40658
:109F20004FEF04074FEF14070CF073C080911F032D
:109F3000882309F46AC0D801C70117FF07C0882722
:109F40009927DC018E199F09A00BB10B9C01AD0173
:109F5000B7FF04C021503E4F4F4F5F4F69E055950A
:109F60004795379527956A95D1F780911C03909175
:109F70001D03820F931F90931D0380931C03D80130
:109F8000C70117FF03C00796A11DB11D23E0B595BA
:109F9000A795979587952A95D1F78093100390936D
:109FA0001103A0931203B093130388579C4EAF4F35
:109FB000BF4F64F488E79CEEAFEFBFEF80931003D0
:109FC00090931103A0931203B093130320911003F5
:109FD00030911103409112035091130357FF04C0B5
:109FE00021503F4F4F4F5F4F232F342F452F552781
:109FF00047FD5A958091520290915302820F931F10
:10A00000909353028093520211C081E080931F030A
:10A010000DC010921F030AC010921D0310921C0362
:10A0200084E690E090938C0180938B016889262FC1
:10A03000332780911C0390911D032817390724F4BE
:10A0400030931D0320931C0310912E08112379F0E7
:10A05000212F332727FD309580911C0390911D03FC
:10A060002817390724F430931D0320931C034091D3
:10A07000010350910203609103037091040341387E
:10A0800051056105710574F08091D9029091DA0251
:10A0900020911C0330911D03820F931F9093DA02CD
:10A0A0008093D90240585F4F6F4F7F4F74F4809177
:10A0B000D9029091DA0220911C0330911D03821B7A
:10A0C000930B9093DA028093D90281E090E0909311
:10A0D0001D0380931C03C0900503D0900603E090FD
:10A0E0000703F0900803D701C601F7FE07C08827D1
:10A0F0009927DC018C199D09AE09BF098150924056
:10A10000A040B04034F084E090E090931D03809331
:10A110001C038091260390912703A0912803B091FE
:10A12000290320917D0730917E0740917F07509150
:10A130008007821B930BA40BB50B815E914BAF4F35
:10A14000BF4F8F539C49A040B04018F019310CF418
:10A15000FFC001E0C01600E1D00600E0E00600E02C
:10A16000F0060CF473C080912003882309F46AC0C0
:10A17000D701C601F7FE07C088279927DC018C1993
:10A180009D09AE09BF099C01AD01B7FF04C0215074
:10A190003E4F4F4F5F4F09E05595479537952795AF
:10A1A0000A95D1F780911C0390911D03820F931F94
:10A1B00090931D0380931C03D701C601F7FE03C0D3
:10A1C0000796A11DB11D13E0B595A79597958795A5
:10A1D0001A95D1F78093140390931503A093160357
:10A1E000B093170389589341A040B04064F088E8C9
:10A1F00093E1A0E0B0E08093140390931503A09343
:10A200001603B09317032091140330911503409166
:10A2100016035091170357FF04C021503F4F4F4F73
:10A220005F4F232F342F452F552747FD5A95809197
:10A23000540290915502820F931F90935502809380
:10A24000540206C081E08093200302C010922003D4
:10A2500020E0C21620EFD2062FEFE2062FEFF20623
:10A260000CF073C080912103882309F46AC0D701E0
:10A27000C601F7FE07C088279927DC018C199D09C4
:10A28000AE09BF099C01AD01B7FF04C021503E4F8C
:10A290004F4F5F4FE9E05595479537952795EA95DC
:10A2A000D1F780911C0390911D03820F931F90930F
:10A2B0001D0380931C03D701C601F7FE03C0079658
:10A2C000A11DB11D73E0B595A795979587957A95D2
:10A2D000D1F78093140390931503A0931603B093C2
:10A2E000170388579C4EAF4FBF4F64F488E79CEE2E
:10A2F000AFEFBFEF8093140390931503A093160361
:10A30000B093170320911403309115034091160365
:10A310005091170357FF04C021503F4F4F4F5F4FDD
:10A32000232F342F452F552747FD5A9580915402EE
:10A3300090915502820F931F90935502809354027F
:10A3400011C081E0809321030DC0109221030AC047
:10A3500010921D0310921C0384E690E090938C01F0
:10A3600080938B014889242F332780911C0390917F
:10A370001D032817390724F430931D0320931C0371
:10A3800080912E08882379F0282F332727FD3095D8
:10A3900080911C0390911D032817390724F43093F2
:10A3A0001D0320931C034091050350910603609107
:10A3B000070370910803413851056105710574F078
:10A3C0008091D7029091D80220911C0330911D03F7
:10A3D000820F931F9093D8028093D70240585F4F0B
:10A3E0006F4F7F4FCCF48091D7029091D80220918B
:10A3F0001C0330911D03821B930B9093D802809312
:10A40000D7020AC0109255021092540210925302C1
:10A41000109252021092800280918307882341F4A7
:10A42000109255021092540210925302109252024E
:10A430008091750790917607A0917707B091780782
:10A440008093220390932303A0932403B0932503C6
:10A4500080917D0790917E07A0917F07B091800742
:10A460008093260390932703A0932803B093290396
:10A470001092B4021092B5021092B6021092B70276
:10A480001092B0021092B1021092B2021092B30276
:10A490001092AC021092AD021092AE021092AF0276
:10A4A000109275071092760710927707109278072E
:10A4B00010927D0710927E0710927F0710928007FE
:10A4C00010926C0710926D0710926E0710926F0732
:10A4D00010925D0710925E0710925F07109260075E
:10A4E0001092EA011092E901E0907602F090770272
:10A4F000C701F7FE04C0882799278E199F09049782
:10A500003CF080919D0784FD03C082E380930F039C
:10A510001091CE05A12EBB24CC24DD24B7018827C1
:10A5200077FD8095982F9701F7FE04C022273327E7
:10A530002E193F09442737FD4095542F0E94F37789
:10A540009B01AC01C601B5010E94F37797FF04C0DF
:10A5500061507E4F8F4F9F4F59E095958795779526
:10A5600067955A95D1F79B01812F99278E9DD00130
:10A570008F9DB00D9E9DB00D1124CD01B7FD0396AA
:10A580009595879595958795280F391F8091560247
:10A5900090915702280F391F442737FD4095542FBB
:10A5A0002093F5023093F6024093F7025093F8029D
:10A5B0008091940290919502A0919602B091970299
:10A5C000821B930BA40BB50B80939402909395027E
:10A5D000A0939602B09397028155934CA040B0404F
:10A5E00064F080E593ECA0E0B0E080939402909357
:10A5F0009502A0939602B093970280919402909155
:10A600009502A0919602B0919702805B9C43AF4F58
:10A61000BF4F64F480EB9CE3AFEFBFEF80939402F5
:10A6200090939502A0939602B093970200918F01A8
:10A630001091900117FDFCC080919D0783FFF8C029
:10A6400080918E01815080938E01882309F0F4C09F
:10A650008DE080938E018091C4029091C502A091FB
:10A66000C602B091C702B7FF04C081509E4FAF4FE2
:10A67000BF4F39E0B595A795979587953A95D1F74E
:10A680007C0197FF04C0F094E194F108F394809169
:10A69000BC029091BD02A091BE02B091BF02B7FF73
:10A6A00004C081509E4FAF4FBF4F29E0B595A7958D
:10A6B000979587952A95D1F79C0197FF03C0309510
:10A6C00021953F4FE216F3060CF47901B701F7FE2E
:10A6D00002C0695F7F4F2B01A3E055944794AA9570
:10A6E000E1F722E030E0420E531E6090AD0770901B
:10A6F000AE078090AF079090B00720914301309152
:10A7000044014091450150914601C401B3010E94AA
:10A71000677859016A0130935B0720935A07021B3F
:10A72000130BC801845E9D4F68E671E00E94327889
:10A730009C01245B304080918B0190918C010097AB
:10A7400031F0019790938C0180938B011BC049E1FC
:10A75000E416F104BCF480917E0290917F02820F96
:10A76000931F90937F0280937E0280910F03882332
:10A7700049F0815080930F03882321F4B092830223
:10A78000A092820280918B0190918C01892BF9F427
:10A7900080918D019927289FB001299F700D389FC6
:10A7A000700D1124CB01B2010E943278CB01AA278F
:10A7B00097FDA095BA2F680E791E8A1E9B1E609287
:10A7C000AD077092AE078092AF079092B00780916C
:10A7D0000F03882369F58091820290918302209172
:10A7E0005A0730915B07821B930B845E9D4F68E68E
:10A7F00071E00E9432789C01245B304080917701A7
:10A8000086959927289FD001299FB00D389FB00DBC
:10A8100011249D01B7FF02C0215F3F4FF4E0359541
:10A820002795FA95E1F7309357022093560204C01A
:10A83000109257021092560280918002882381F074
:10A84000109288021092890210928A0210928B0252
:10A8500010928C0210928D0210928E0210928F0232
:10A86000F0904F02FF20F1F480918307282F3327C7
:10A87000442755278091C4029091C502A091C60239
:10A88000B091C702BC01CD010E94F377DC01CB017E
:10A89000BC01CD0128EF3AE240E050E00E94677829
:10A8A000390102C066247724E0904E02EE20F1F4D4
:10A8B00080918307282F3327442755278091BC0296
:10A8C0009091BD02A091BE02B091BF02BC01CD012A
:10A8D0000E94F377DC01CB01BC01CD0128EF3AE205
:10A8E00040E050E00E946778290102C044245524CA
:10A8F0008091570790915807893C91051CF088EC8E
:10A9000090E005C088539F4F34F488E39FEF909305
:10A910005807809357078091630790916407893C9B
:10A9200091051CF088EC90E005C088539F4F34F4EB
:10A9300088E39FEF90936407809363078091650796
:10A9400090916607AA2797FDA095BA2F2091AB0793
:10A95000A22EBB24CC24DD24BC01CD01A60195018F
:10A960000E94F3779B01AC018091570790915807A3
:10A97000AA2797FDA095BA2FE7E0880F991FAA1F75
:10A98000BB1FEA95D1F7280F391F4A1F5B1F57FFDE
:10A9900004C0215C3F4F4F4F5F4F76E05595479580
:10A9A000379527957A95D1F78301020F131F1093DE
:10A9B0006607009365078091550790915607AA276F
:10A9C00097FDA095BA2FBC01CD01A60195010E946B
:10A9D000F3779B01AC018091630790916407AA27EC
:10A9E00097FDA095BA2F67E0880F991FAA1FBB1F7C
:10A9F0006A95D1F7280F391F4A1F5B1F57FF04C004
:10AA0000215C3F4F4F4F5F4FF6E055954795379587
:10AA10002795FA95D1F74201820E931E9092560720
:10AA2000809255078091A6079091A707880F991FDC
:10AA3000AA2797FDA095BA2F20915C0733274427BA
:10AA40005527BC01CD010E94F3775B016C0197FF94
:10AA500008C02FE330E040E050E0A20EB31EC41E59
:10AA6000D51EE6E0D594C794B794A794EA95D1F79C
:10AA700080917207282F3327442755278091A802F9
:10AA80009091A902A091AA02B091AB02BC01CD01A4
:10AA90000E94F377DC01CB01BC01CD0120EF35E54D
:10AAA00040E050E00E946778B501620F731F709319
:10AAB000A7076093A6070150104134F080E090E1B1
:10AAC000909366078093650780916507909166076C
:10AAD0008050904F34F480E090EF9093660780931D
:10AAE000650751E0851650E1950634F080E090E16D
:10AAF000909356078093550780915507909156077C
:10AB00008050904F34F480E090EF909356078093FC
:10AB100055076150704134F080E090E19093A707B1
:10AB20008093A6078091A6079091A7078050904F29
:10AB300034F480E090EF9093A7078093A60780916C
:10AB40000001482F552780911E0190911F01481741
:10AB5000590794F420911E0130911F0109811A8137
:10AB6000049FC001059F900D149F900D1124B90101
:10AB70000E941E787A83698329813A81220F331FCC
:10AB8000220F331F3A83298340919D0740FD02C065
:10AB90000C94B85DEE2009F0EBC7FF2009F0E8C780
:10ABA00000E010E048018091500290915102909392
:10ABB0003B0580933A052091DB023091DC022115A0
:10ABC000310509F03FC08091140190911501895918
:10ABD000934058F087B5853F20F48091ED01815076
:10ABE00011C081E0809333034EC080911401909195
:10ABF00015018436910508F587B58B30D0F080912A
:10AC0000ED018F5F8093ED019AE08902900111249C
:10AC100080916105821B87BD8CE291E09093DB01FE
:10AC20008093DA018EE591E09093DC028093DB0261
:10AC30002AC081E08093320326C0F0923203F09262
:10AC4000330321C08091640290916502A091660255
:10AC5000B091670264E0880F991FAA1FBB1F6A9515
:10AC6000D1F78093EE019093EF01A093F001B093A0
:10AC7000F1011093EC010093EB012150304030932F
:10AC8000DC022093DB0220917A0141FF24C02233B1
:10AC9000D8F4809191018150809391018F3FD9F533
:10ACA000109281028091640290916502A0916602E7
:10ACB000B09167028093600290936102A093620258
:10ACC000B093630281E004C081E08093810288EC4C
:10ACD0008093910120C08091470190914801820F9B
:10ACE000911D2091C7053327829FA001839F500D9E
:10ACF000929F500D1124CA01AA2797FDA095BA2F43
:10AD00008093600290936102A0936202B093630209
:10AD100081E0809381028091C4029091C502A0914C
:10AD2000C602B091C702E0904301F0904401009147
:10AD3000450110914601BC01CD01A80197010E9477
:10AD4000677859016A018091BC029091BD02A0917F
:10AD5000BE02B091BF02BC01CD01A80197010E94C3
:10AD60006778B901C5010E941C765C01CC971CF084
:10AD70005CE3A52EB12CC5010E9455695C0180E2FF
:10AD80008093420110925F0210925E0280918102D4
:10AD9000882309F45FC58091340299279C012071B2
:10ADA000307084FD57C580913302826080933302F6
:10ADB00070918107872F992741E0C42ED12CC8229A
:10ADC000D92280FD04C080919D0781FD10C0C980FB
:10ADD000DA8030932B0320932A0330935F02209371
:10ADE0005E0280913402806C80933402ABC2809109
:10ADF000340281FF7AC20091810110918201C80161
:10AE00000F962090740230907502821593050CF015
:10AE100058C080913203882309F053C080913402D6
:10AE200087FF15C0809134028F7780933402809120
:10AE3000640290916502A0916602B09167028093CE
:10AE4000600290936102A0936202B09363028091CA
:10AE50003402806480933402E0906107EE20F1F0C8
:10AE60008091600290916102A0916202B0916302B0
:10AE7000BC01CD0124E630E040E050E00E9467785C
:10AE80008E2D9927AA27BB2782179307A407B507FA
:10AE90002CF4D0925F02C0925E0210C0C101801BF0
:10AEA000910B0F9797FF03C0909581959F4F9093BB
:10AEB0005F0280935E028BE28093420110925802FF
:10AEC00016C1C8010F9728163906C4F5209133031F
:10AED0002223A1F58091340286FF15C080913402AF
:10AEE0008F7B809334028091640290916502A091DF
:10AEF0006602B09167028093600290936102A09312
:10AF00006202B093630280913402806880933402BD
:10AF1000C101801B910B0F9697FF03C090958195FF
:10AF20009F4F909581959F4F90935F0280935E0213
:10AF30008DE28093420120935802D9C08DE3809323
:10AF4000420160915902662371F120915A023091B9
:10AF50005B0240915C0250915D0280916002909191
:10AF60006102A0916202B091630282179307A40765
:10AF7000B507CCF480913402806480933402862F2C
:10AF8000992790935F0280935E028AE08093580233
:10AF90008EE5809342018091340287FFA8C08091A2
:10AFA00034028F7733C0662309F443C020915A02DC
:10AFB00030915B0240915C0250915D028091600291
:10AFC00090916102A0916202B09163022817390743
:10AFD0004A075B0774F580913402806880933402DD
:10AFE000862F9927909581959F4F90935F0280932C
:10AFF0005E0286EF8093580286E78093420180913B
:10B00000340286FF74C0809134028F7B80933402B7
:10B010008091640290916502A0916602B0916702EE
:10B020008093600290936102A0936202B0936302E6
:10B030005EC080913402807C09F459C0809158022E
:10B04000882379F5E0906402F09065020091660231
:10B0500010916702D801C70180589040A040B040CD
:10B06000209160023091610240916202509163022E
:10B0700082179307A407B5075CF4D801C70180586D
:10B080009F4FAF4FBF4F281739074A075B075CF048
:10B090008093600290936102A0936202B093630276
:10B0A00002C010925802809134028F738093340250
:10B0B00010922B0310922A0371FF06C084EF91E0D7
:10B0C0009093DB018093DA0180916802882379F400
:10B0D0008091640290916502A0916602B09167022E
:10B0E000C397A105B1051CF081E0809368026091CF
:10B0F0002A0370912B0380915E0290915F02680F8A
:10B10000791F70932B0360932A03CB0177FF04C050
:10B1100088279927861B970B855F91400CF4CEC03A
:10B1200040915802442389F180915A0290915B0228
:10B130002091600230916102821B930B0996439724
:10B1400048F480915A0290915B02A0915C02B09108
:10B150005D0212C0242F332727FD3095432F532F34
:10B160008091600290916102A0916202B0916302AD
:10B17000820F931FA41FB51F8093600290936102FA
:10B18000A0936202B093630224C08091C70520910E
:10B190006002309161024091620250916302161682
:10B1A000170644F463E00E941278280F311D411DF8
:10B1B000511D07C063E00E941278281B3109410924
:10B1C00051092093600230936102409362025093D0
:10B1D000630210922B0310922A03E0906402F09015
:10B1E00065020091660210916702D801C701805084
:10B1F0009440A040B04020916002309161024091A3
:10B2000062025091630282179307A407B5075CF4AA
:10B21000D801C70180509C4FAF4FBF4F2817390747
:10B220004A075B0744F08093600290936102A09309
:10B230006202B09363028091810781FF06C084E6B9
:10B2400090E09093DB018093DA018091CB05882315
:10B25000A9F580915902882389F5409150025091B7
:10B26000510257FF02C04D5F5F4F55954795559569
:10B27000479580911E0190911F0120910001332775
:10B28000489FF001499FF00D589FF00D1124CF0108
:10B29000B9010E9432787093820160938101663413
:10B2A00071051CF486E490E005C06739710534F03F
:10B2B00086E990E090938201809381018091DB0286
:10B2C0009091DC02892BD1F180916402909165020A
:10B2D000A0916602B0916702809360029093610230
:10B2E000A0936202B093630229C08091640290919E
:10B2F0006502A0916602B091670280599140A0401A
:10B30000B0408093600290936102A0936202B09378
:10B3100063028091CB05882311F0992702C088E74A
:10B3200090E09093820180938101E980FA80F0920D
:10B330005102E09250028EE280934201C09050028E
:10B34000D0905102E0906402F09065020091660294
:10B350001091670220916002309161024091620277
:10B36000509163022E153F054007510724F080914C
:10B37000810780FDBBC28091DB029091DC02892BAA
:10B3800039F0C0905002D090510200E010E0D7C0D8
:10B39000D801C701821B930BA40BB50B8093F90254
:10B3A0009093FA02A093FB02B093FC02823000E873
:10B3B00090070FEFA0070FEFB0072CF481E090E8A3
:10B3C000AFEFBFEF09C08F5F9F47A040B04064F070
:10B3D0008FEF9FE7A0E0B0E08093F9029093FA022C
:10B3E000A093FB02B093FC020091F9021091FA02C3
:10B3F00080917901282F3327442755278091F9021E
:10B400009091FA02A091FB02B091FC02BC01CD0127
:10B410000E94F37797FF04C0615E7F4F8F4F9F4F6D
:10B4200025E095958795779567952A95D1F760934F
:10B43000F9027093FA028093FB029093FC0265304C
:10B440002EEF72072FEF82072FEF92072CF484E084
:10B450009EEFAFEFBFEF09C0605074408040904056
:10B4600064F080E094E0A0E0B0E08093F902909373
:10B47000FA02A093FB02B093FC028090F902909034
:10B48000FA022091EB013091EC0137FF02C0295FF5
:10B490003F4F83E0359527958A95E1F74FEF2238A6
:10B4A00034071CF421E83FEF05C02038310514F0C3
:10B4B00020E830E0C901AA2797FDA095BA2F209176
:10B4C0007B01332744275527BC01CD010E94F37728
:10B4D00097FF04C06D5F7F4F8F4F9F4FB2E09595F0
:10B4E000879577956795BA95D1F79B015FEF6130A6
:10B4F00075071CF420E03FEF06C06F3F710519F09F
:10B5000014F020E031E080913402807C49F0C901E0
:10B5100037FD03969C0135952795359527950DC0E8
:10B520008091810780FF09C0C90137FD07969C0102
:10B53000F3E035952795FA95E1F7820E931E209159
:10B540007801222309F454C060918402709185022D
:10B55000809186029091870297FF04C061587F4FC7
:10B560008F4F9F4FE7E09595879577956795EA957B
:10B57000D1F73327442755270E94F37797FF04C05C
:10B58000615E7F4F8F4F9F4F55E0959587957795DB
:10B5900067955A95D1F76093F9027093FA028093F8
:10B5A000FB029093FC026138AFEF7A07AFEF8A0796
:10B5B000AFEF9A072CF480E89FEFAFEFBFEF0AC020
:10B5C0006F3F71058105910569F064F080E091E0BD
:10B5D000A0E0B0E08093F9029093FA02A093FB02FE
:10B5E000B093FC028091F9029091FA02880E991EA4
:10B5F00080917601282F332780913108992787FD84
:10B600009095289FF001299FF00D389FF00D11248F
:10B610009F01F7FF02C021583F4F220F232F221F07
:10B62000330BFFEF21383F071CF420E83FEF06C043
:10B630002F3F310519F014F020E031E0820E931E07
:10B64000C401AA2797FDA095BA2FE0905002F09070
:10B6500051029701442737FD4095542FBC01CD017D
:10B660000E94F37797FF04C061507E4F8F4F9F4F2A
:10B6700029E095958795779567952A95D1F7C61A0C
:10B68000D70A80915E0290915F02892B09F060C019
:10B690001E141F040CF05CC0980117FF03C0309506
:10B6A00021953F4F2D33310540F480917C029091DC
:10B6B0007D028C159D0574F526C02C53304085E025
:10B6C000369527958A95E1F72031310510F02FE066
:10B6D00030E040917C0250917D0210161106E4F496
:10B6E00080E190E0821B930B489F9001499F300DB1
:10B6F000589F300D1124B4E036952795BA95E1F79F
:10B700002C153D0520F580917F0190918001C81690
:10B71000D906F4F06C011CC0205F3F4F80917F017F
:10B7200090918001829F8001839F100D929F100D48
:10B7300011249801A4E036952795AA95E1F74C15B8
:10B740005D0514F06A0104C0C216D30608F0690151
:10B75000C601AA2797FDA095BA2FFDE0880F991F73
:10B76000AA1FBB1FFA95D1F79501442737FD4095D5
:10B77000542FBC01CD010E9467782093FD023093C5
:10B78000FE024093FF0250930003C090FD02D09050
:10B79000FE0280912C0390912D039C01220F331FF8
:10B7A000280F391F2C0D3D1D37FF02C02D5F3F4F65
:10B7B000A901559547955595479550932D0340936D
:10B7C0002C038091C305282F3327220F331F220F0C
:10B7D000331F241735076CF48091A507282F3327D2
:10B7E000220F331F220F331F2055304042175307BB
:10B7F00024F030932D0320932C038091810780FF48
:10B8000014C080912C0390912D0329813A818217D5
:10B81000930724F030932D0320932C0340912C03A5
:10B8200050912D035A83498361C029813A812E1991
:10B830003F0937FF02C02D5F3F4F3595279535955E
:10B84000279560912C0370912D03620F731F7A83EB
:10B8500069834CC08091CB05882301F5609150022B
:10B860007091510277FF02C06D5F7F4F75956795AC
:10B870007595679540911E0150911F0180910001BF
:10B88000282F3327649FC001659F900D749F900DF2
:10B890001124B9010E943278CB0101C099279093FD
:10B8A000820180938101809181019091820187348E
:10B8B00091051CF486E490E005C08639910534F0CA
:10B8C00086E990E0909382018093810189819A8139
:10B8D00090932D0380932C0380913402806C80938D
:10B8E0003402809133028D7F809333028091340241
:10B8F00099279C012270307081FF2BC180912E030B
:10B9000090912F03A0913003B09131030097A105CE
:10B91000B10521F0809168028130B1F4E981FA81AA
:10B92000CF01AA2797FDA095BA2F1EE0880F991F77
:10B93000AA1FBB1F1A95D1F780932E0390932F0354
:10B94000A0933003B093310380916802813019F4E1
:10B9500082E080936802E980FA80C701AA2797FDF8
:10B96000A095BA2F9501442737FD4095542FBC016F
:10B97000CD010E94F377DC01CB018093FD0290930F
:10B98000FE02A093FF02B0930003B7FF04C08150F2
:10B99000904EAF4FBF4F7C018D01FDE0159507958F
:10B9A000F794E794FA95D1F7E092FD02F092FE0247
:10B9B0000093FF02109300036091350270913602EC
:10B9C0002FE0603A720750F580912E0390912F037B
:10B9D000A0913003B09131039C01AD01EAE056958E
:10B9E000479537952795EA95D1F7821B930BA40BC2
:10B9F000B50BA8019701F4E0220F331F441F551F18
:10BA0000FA95D1F7820F931FA41FB51F80932E03C1
:10BA100090932F03A0933003B093310360547F4180
:10BA200018F580912E0390912F03A0913003B091CF
:10BA300031039C01AD01ECE056954795379527956C
:10BA4000EA95D1F7821B930BA40BB50BA8019701C4
:10BA500072E0220F331F441F551F7A95D1F7820FD2
:10BA6000931FA41FB51F38C08091EB019091EC018A
:10BA70008091EB019091EC0197FF03C09095819527
:10BA80009F4F8436910584F5809164029091650200
:10BA90002091600230916102821B930B81509F4F75
:10BAA0008F5F914008F580912E0390912F03A09114
:10BAB0003003B09131039C01AD016EE0569547957E
:10BAC000379527956A95D1F7821B930BA40BB50B7D
:10BAD0008E0D9F1DA01FB11F80932E0390932F03E7
:10BAE000A0933003B093310380912E0390912F03E4
:10BAF000A0913003B09131035EE0B695A79597957C
:10BB000087955A95D1F790935102809350024091B6
:10BB1000C905442399F055279C01BA010E94327847
:10BB2000C901861B970B90937D0280937C02260FA0
:10BB3000371F3093800120937F011FC010927D0238
:10BB400010927C028FEF93E09093800180937F01AD
:10BB500014C01092680210922E0310922F031092BC
:10BB6000300310923103309351022093500205C0EC
:10BB700080913402806C8093340220916A07822F76
:10BB80009927880F991F880F991F889669817A8154
:10BB90008617970714F09A8389837091A5077D8B88
:10BBA000872F9927880F991F880F991F80559040DC
:10BBB000A981BA818A179B0714F49A83898380919B
:10BBC0002302882341F4809138088F3F21F480912B
:10BBD00044038823E9F08091350290913602029760
:10BBE000C097B0F4E981FA811E161F068CF481E03B
:10BBF00090E09093360280933502E22EFF24EE0C03
:10BC0000FF1CEE0CFF1C8701085D1F4F1A83098380
:10BC100029813A8130931F0520931E058091F502FA
:10BC20009091F602A091F702B091F80212E0880F0D
:10BC3000991FAA1FBB1F1A95D1F70091A607109153
:10BC4000A707081B190B213A31058CF0C90137FDF4
:10BC5000019695958795801791070CF48C01909526
:10BC600081959F4F081719076CF48C010BC00135A3
:10BC7000110514F000E510E03FEF003B130714F44A
:10BC800000EB1FEF4D89242F3327220F331F220F84
:10BC9000331FC90169817A81861B970B8017910731
:10BCA0000CF48C0189819A81821B930B0817190768
:10BCB0000CF48C01809165079091660760917A027F
:10BCC00070917B02861B970B909374078093730788
:10BCD000D090830720918C0230918D0240918E028A
:10BCE00050918F02DD2041F0661A770AC301AA271E
:10BCF00097FDA095BA2F04C0AA2797FDA095BA2F4B
:10BD0000280F391F4A1F5B1F20938C0230938D022E
:10BD100040938E0250938F0280918C0290918D02FD
:10BD2000A0918E02B0918F0281509A4FA040B040F6
:10BD300064F080E09AEFA0E0B0E080938C029093F2
:10BD40008D02A0938E02B0938F0280918C0290910D
:10BD50008D02A0918E02B0918F0280509640AF4F1D
:10BD6000BF4F64F480E096E0AFEFBFEF80938C02AA
:10BD700090938D02A0938E02B0938F02C090D8054D
:10BD8000209173073091740778E0E72EEC1498F057
:10BD90008C2D9927829FA001839F500D929F500D5B
:10BDA0001124CA0157FD07967C0163E0F594E794DE
:10BDB0006A95E1F712C08C2D86959927829FB00174
:10BDC000839F700D929F700D1124CB0177FD039618
:10BDD0007C01F594E794F594E794A0907C01B090F1
:10BDE0007D019501442737FD4095542F80918C02A9
:10BDF00090918D02A0918E02B0918F02BC01CD0175
:10BE00000E946778E20EF31E90906801692D7727F3
:10BE100088279927980117FF04C022273327201B62
:10BE2000310B37FF02C02F5F3F4F35952795A98112
:10BE3000BA812A0F3B1F442737FD4095542F0E949B
:10BE4000F37797FF04C0615C7F4F8F4F9F4F26E0D1
:10BE500095958795779567952A95D1F79B016E15EE
:10BE60007F050CF47B01309521953F4FE216F306D8
:10BE70000CF47901809155079091560760917802F2
:10BE800070917902861B970B909354078093530708
:10BE9000209188023091890240918A0250918B0250
:10BEA000DD2041F0461A570AC201AA2797FDA09546
:10BEB000BA2F04C0AA2797FDA095BA2F280F391FC3
:10BEC0004A1F5B1F209388023093890240938A02A5
:10BED00050938B028091880290918902A0918A02EE
:10BEE000B0918B0281509A4FA040B04064F080E046
:10BEF0009AEFA0E0B0E08093880290938902A0932B
:10BF00008A02B0938B028091880290918902A0915D
:10BF10008A02B0918B0280509640AF4FBF4F64F4BD
:10BF200080E096E0AFEFBFEF8093880290938902A4
:10BF3000A0938A02B0938B0220915307309154074B
:10BF400048E04C1598F08C2D9927829FB001839F73
:10BF5000700D929F700D1124CB0177FD07966C0137
:10BF6000B3E0D594C794BA95E1F712C0C6948C2D6E
:10BF70009927829FD001839FB00D929FB00D11240D
:10BF8000CD01B7FD03966C01D594C794D594C794A1
:10BF90009501442737FD4095542F80918802909158
:10BFA0008902A0918A02B0918B02BC01CD010E944E
:10BFB0006778C20ED31E692D7727882799279801A5
:10BFC00017FF04C022273327201B310B37FF02C085
:10BFD0002F5F3F4F35952795E981FA812E0F3F1F3F
:10BFE000442737FD4095542F0E94F37797FF04C0F4
:10BFF000615C7F4F8F4F9F4FE6E0959587957795D2
:10C000006795EA95D1F79B016C157D050CF46B01E2
:10C01000309521953F4FC216D3060CF469018091EB
:10C020006A07282E33245090190663E8862E66E0AE
:10C03000962E5AE3A52E56E0B52E4BE0442E34E85A
:10C04000632E37E0732ED5012C9112160CF029C106
:10C05000203429F4E981FA81FF8BEE8B1FC04981DE
:10C060005A81CA01AA2797FDA095BA2F332727FD29
:10C070003095432F532FBC01CD010E94F37797FFDA
:10C0800004C0615C7F4F8F4F9F4F26E09595879549
:10C09000779567952A95D1F77F8B6E8BF501218176
:10C0A000203439F42E893F892E0D3F1D3F8B2E8B76
:10C0B0002AC0203C39F44E895F894E195F095F8B95
:10C0C0004E8B21C0C701AA2797FDA095BA2F332711
:10C0D00027FD3095432F532FBC01CD010E94F377EC
:10C0E00097FF04C0615C7F4F8F4F9F4FB6E09595DF
:10C0F000879577956795BA95D1F7AE89BF89A60FD1
:10C10000B71FBF8BAE8BF5012281203439F42E8905
:10C110003F892C0D3D1D3F8B2E8B2AC0203C39F4CE
:10C120004E895F894C195D095F8B4E8B21C0C6011A
:10C13000AA2797FDA095BA2F332727FD3095432FC7
:10C14000532FBC01CD010E94F37797FF04C0615CBF
:10C150007F4F8F4F9F4FA6E0959587957795679571
:10C16000AA95D1F7AE89BF89A60FB71FBF8BAE8B3B
:10C17000F5012381203439F42E893F89200F311FA6
:10C180003F8B2E8B2AC0203C39F44E895F89401B9F
:10C19000510B5F8B4E8B21C0C801AA2797FDA0953C
:10C1A000BA2F332727FD3095432F532FBC01CD01E4
:10C1B0000E94F37797FF04C0615C7F4F8F4F9F4FC2
:10C1C000F6E09595879577956795FA95D1F7AE89BD
:10C1D000BF89A60FB71FBF8BAE8BF3018081918102
:10C1E0002E893F898217930764F4B901680F791F7C
:10C1F00077FF02C06F5F7F4F759567957F8B6E8B62
:10C200001DC0552049F44E895F89440F551F481BB6
:10C21000590B5F8B4E8B12C051E0551578F4252DCC
:10C2200033276E897F89861B970BB9010E9432786C
:10C23000AE89BF89A60FB71FBF8BAE8BC101880F18
:10C24000991F880F991FEE89FF898E179F0764F445
:10C25000FD898F2F9927880F991F880F991F2E8985
:10C260003F892817390714F09F8B8E8B8E899F8901
:10C2700097FD03969595879595958795F40181830C
:10C28000880F991F880F991F2E893F89281B390B0A
:10C29000C901880F8283EE89FF89D301ED93FC9356
:10C2A00003C0F401118212824A9422E030E0620E4F
:10C2B000731E44E050E0A40EB51E68E070E0860EE8
:10C2C000971E47FEC0CEE2E1C95E0C949E7884B111
:10C2D000806A84B93D9A82E58CBD1DBC459A81E097
:10C2E0008093B7078AEA8093C80783E88093C907D9
:10C2F0008AE08093CA071092CC071092CB07109265
:10C30000CE071092CD07109230081092EC070895D6
:10C310003091B707332309F085C00DB407FE82C002
:10C3200084E08093D901459A2EB5809147039927DF
:10C330008130910589F0823091051CF4892B21F020
:10C340003EC00297B9F03BC03093EB0720934803FF
:10C350002138A9F581E008C0253549F480914803CA
:10C36000820F8093480382E08093470328C0309374
:10C37000470325C08091EB07E82FFF27E35FF74FC6
:10C3800020838F5F8093EB07909148038032A0F069
:10C39000291769F480E2ADE0B8E0EDEEF7E00D902A
:10C3A00001928A95E1F781E08093EC0702C0309317
:10C3B000EC071092470303C0920F9093480320911B
:10C3C000C707223208F028C045980000000000008E
:10C3D000000000000000000000000000000000005D
:10C3E000000000000000000000000000000000004D
:10C3F00000000000000000000000E091C007F09184
:10C40000C107E20FF11D80818EBD8091E907908107
:10C41000890F8093E90703C081E08093B7072F5FFE
:10C420002093C7070895EF92FF920F931F93809177
:10C43000D1059927880F991F880F991F7C01002724
:10C44000F7FC0095102F8091C4029091C502A09135
:10C45000C602B091C702BC01CD01A80197010E949C
:10C4600067783093CC072093CB078091BC029091E2
:10C47000BD02A091BE02B091BF02BC01CD01A801D6
:10C4800097010E9467783093CE072093CD072091C3
:10C49000AD073091AE074091AF075091B007DA0178
:10C4A000C90163E0880F991FAA1FBB1F6A95D1F7C6
:10C4B000820F931FA41FB51F820F931FA41FB51FC8
:10C4C0002091430130914401409145015091460132
:10C4D000BC01CD010E9467783093D4072093D30725
:10C4E0008091D5029091D6022091F9013091FA0104
:10C4F000821B930B9093DA078093D907E091CB02CC
:10C50000F091CC0280917A0790917B07BF010E9445
:10C5100032789B01220F331F220F331F260F371F44
:10C52000260F371F37FF02C02D5F3F4F35952795E8
:10C53000359527953093D0072093CF078091A90791
:10C540009091AA07BF010E9432789B01220F331FEE
:10C55000220F331F260F371F260F371F37FF02C04A
:10C560002D5F3F4F35952795359527953093D20709
:10C570002093D1071092CC021092CB0210927B072D
:10C5800010927A071092AA071092A9078091CA0701
:10C5900099278D30910509F48EC08E3091055CF499
:10C5A0008B30910509F4B6C08C3091050CF037C181
:10C5B0000A9761F0E7C18F30910509F4B3C18F305C
:10C5C00091050CF482C14097A9F1DCC18091490228
:10C5D0008093DD07809148028093DE0780914702B7
:10C5E0008093DF07809146028093E00780914502A7
:10C5F0008093E107809144028093E2078091430297
:10C600008093E307809142028093E4078091340293
:10C610008093E50780913402837F809334020E94E7
:10C62000492C8093E60780911A068093E707809152
:10C630003302A6C180913208909133089093DE07AF
:10C640008093DD0780913608909137089093E0073A
:10C650008093DF0780911E0190911F018093E10775
:10C66000809100018093E207809142018093E3076B
:10C6700080919D078093E407809181078093E5076F
:10C68000909149039093E607E92FFF27A3E0EE0F6F
:10C69000FF1FAA95E1F7ED57F94F87818093E707D0
:10C6A00085818093E807892F8F5F6CE00E94127864
:10C6B0009093490367C1809105068093DD078091BF
:10C6C00006068093DE07809107068093DF0780913E
:10C6D00008068093E007809109068093E107809126
:10C6E0000D068093E20780910E068093E307809108
:10C6F0000F068093E407809112068093E5078091EE
:10C7000010068093E607809111068093E7078091D9
:10C71000130636C1F8948091B805E82FFF27EE0F75
:10C72000FF1FEC51F94F0190F081E02DE038F10549
:10C730001CF0EFE7F0E006C02FEFE138F20714F449
:10C74000E1E8FFEFE093DD078091B905E82FFF27CF
:10C75000EE0FFF1FEC51F94F0190F081E02DE03812
:10C76000F1051CF0EFE7F0E006C06FEFE138F607E7
:10C7700014F4E1E8FFEFE093DE078091B705E82FBE
:10C78000FF27EE0FFF1FEC51F94F0190F081E02DD4
:10C79000E038F1051CF0EFE7F0E006C08FEFE1387C
:10C7A000F80714F4E1E8FFEFE093DF078091B605A6
:10C7B000E82FFF27EE0FFF1FEC51F94F0190F0819A
:10C7C000E02DE038F1051CF0EFE7F0E006C02FEFB8
:10C7D000E138F20714F4E1E8FFEF7894E093E00722
:10C7E00080916B028093E10780916C028093E20755
:10C7F00080916D028093E30780916E028093E4073D
:10C8000080916F028093E507809170028093E60724
:10C81000809171028093E70780917202B1C080918C
:10C82000A903863018F01092A90385E08093DD07F4
:10C83000809114068093DE078091640290916502D6
:10C84000A0916602B0916702BC01CD0125E030E005
:10C8500040E050E00E9467783093E0072093DF07C4
:10C860008091600290916102A0916202B091630296
:10C87000BC01CD0125E030E040E050E00E94677847
:10C880003093E2072093E10780910A068093E30743
:10C8900080910B068093E40780910C068093E50756
:10C8A00080916A028093E6078091E4069091E50604
:10C8B0008093E70780911E0590911F0597FD0396D1
:10C8C00095958795959587955BC01092DD0786E5D0
:10C8D0008093DE0782E08093DF078BE18093E0079F
:10C8E000809102018093E10780918E038093E2079B
:10C8F00080918F038093E30710928E038071809361
:10C900008F03809190038093E4078091910380933B
:10C91000E507809192038093E60780911606809345
:10C92000E70730C08091EA058093DD0780911E06FD
:10C930008093DE0780916E018093DF078091E3058D
:10C940008093E0078091E4058093E1078091E505FD
:10C950008093E20780916D018093E3078091E70562
:10C960008093E4078091E8058093E5078091E905CD
:10C970008093E607809138088093E7078091480507
:10C980008093E8078091EC07882309F43EC18AEF81
:10C9900080939C0181E080938E014091EE0750913D
:10C9A000EF07CA0181509E4F8F5F9340B0F42091F2
:10C9B000F0073091F107C90181509E4F8F5F93407E
:10C9C00060F48091C20585FF08C0509338034093FE
:10C9D000370330933603209335038091F407909109
:10C9E000F50721E08936920724F490939001809313
:10C9F0008F012091FE073091FF078091DA0190911D
:10CA0000DB018217930720F43093DB012093DA01D6
:10CA10008091ED0799278836910509F468C0893619
:10CA2000910524F48736910551F0F7C089369105B8
:10CA300009F48EC08B36910509F4DAC0EEC08091FE
:10CA4000000880932D088091010880932F08809121
:10CA5000020880932E088091030880938D018091B5
:10CA60000408809331088091050880939D0180918E
:10CA700006088093460380910708809334038091D1
:10CA800041028823F9F0209108083091090837FD08
:10CA900019C030938302209382029091EC05992370
:10CAA00089F08FE0989FC0011124281B390BC90120
:10CAB00088599E4F68E671E00E9432789093830215
:10CAC0008093820220913F033091400380910A08B5
:10CAD00090910B08280F391F37FF02C02F5F3F4F7F
:10CAE000359527953093400320933F0396C080915E
:10CAF00000088093C207809101088093C30780914A
:10CB000002088093C407809103088093C507809131
:10CB100004088093C60780910E0590910508892B23
:10CB200080930E0590910F059370809106088C708C
:10CB3000982B90930F058091070880934403809170
:10CB4000080880939201809109088093300865C09D
:10CB5000809100088093B807809101088093B907FD
:10CB6000809102088093BA07809103088093BB07E5
:10CB700080910408909105089093BD078093BC07AD
:10CB800080910608909107089093BF078093BE0795
:10CB900080910808992787FD9095909317078093B7
:10CBA0001607809109088093590280910A08909194
:10CBB0000B089C01442737FD4095542FDA01C90129
:10CBC00063E0880F991FAA1FBB1F6A95D1F7820FD8
:10CBD000931FA41FB51F820F931FA41FB51F80931F
:10CBE0005A0290935B02A0935C02B0935D0215C061
:10CBF0008091000880934303809101088093420351
:10CC0000809102088093410308C01092380310926B
:10CC1000370310923603109235031F910F91FF9046
:10CC2000EF9008958091B707882309F43BC0459899
:10CC300088EC97E09093C1078093C00790914503DB
:10CC4000E92FFF27ED56FE4F9F5F909345038081AC
:10CC50008093CA07993010F0109245031092B707DD
:10CC60000E94136281E08093C7070000000000006B
:10CC700000000000000000000000000000000000B4
:10CC800000000000000000000000000000000000A4
:10CC9000000000000000000000008091C8078093A1
:10CCA000E9078EBD089587B18C6087B94298439893
:10CCB00010924B0380E880939F0110924A03809367
:10CCC0009E010895809150038150809350038F3FBF
:10CCD00009F0FAC089E080935003809134029927CB
:10CCE00080739070892B21F480918F0380FF1DC089
:10CCF00080910306882351F080915303882319F40F
:10CD000084E080934B0381E0809353038091040679
:10CD10008823B9F080915403882319F484E0809328
:10CD20004A0381E0809354030CC010925303109285
:10CD300054038091FF0580935103809101068093F5
:10CD4000520380915303882309F040C080911D064F
:10CD5000282F332724FF07C080916902882319F404
:10CD600025FD4DC04EC090910006983F50F0809137
:10CD70007C078D3D30F08091510388230CF43FC037
:10CD800040C0983F48F080917C07853029F480911D
:10CD900051038823B4F133C080914B0381508093B9
:10CDA0004B038F3F79F580917C07869580934B03E9
:10CDB00080919F01813011F480E801C086958093B5
:10CDC0009F0180919F019091510317C080914B0367
:10CDD000815080934B038F3FA9F489E080934B03EC
:10CDE00080919F01813011F480E801C08695809385
:10CDF0009F0180919F0190910306892311F0429A2F
:10CE000001C0429880915403882309F041C0909159
:10CE10001D0697FF07C080916902882319F496FDCB
:10CE200050C034C090910206983F50F08091A40702
:10CE30008D3D30F08091520388230CF442C026C00F
:10CE4000983F48F08091A407853029F480915203DF
:10CE50008823E4F036C080914A03815080934A03CE
:10CE60008F3F91F58091A407869580934A03809126
:10CE70009E01813011F480E801C0869580939E0167
:10CE800080919E01909152038923D9F4439808958B
:10CE900080914A03815080934A038F3FA9F489E02F
:10CEA00080934A0380919E01813011F480E801C093
:10CEB000869580939E0180919E019091040689231E
:10CEC00011F0439A0895439808954FB724E130E054
:10CED000F8948091C9008F778093C9008091C90030
:10CEE0008F7B8093C9008091C9008F7D8093C9009A
:10CEF0005A9A52985B9A539A832F99278093CD0020
:10CF00002093CC008091C80082608093C80080E1AB
:10CF10008093C9008091CA008F778093CA00809166
:10CF2000CA008F7B8093CA008091CA008F7D809356
:10CF3000CA008091CA008F7E8093CA008091CA0087
:10CF4000877F8093CA008091C9008B7F8093C9003E
:10CF50008091CA0084608093CA008091CA00826078
:10CF60008093CA008091C80087FF03C08091CE00E3
:10CF7000F9CF8091C90080688093C9004FBF0895A0
:10CF8000EF92FF920F931F93CF93DF93482F00E010
:10CF900010E08091A001813061F41092A00184E43E
:10CFA0008093550310925703109256031092580322
:10CFB0002BC180915503882319F421E030E001C092
:10CFC000980190915603992371F4232B11F081E07D
:10CFD00010C084E4809355039093570390935603B5
:10CFE00090935803FAC0913069F4232B09F0EBC0F9
:10CFF00082E080935603809157038F5F809357039D
:10D0000083E0E9C09230D1F4232B09F0DCC083E047
:10D01000809355034093580390915703923039F40D
:10D020001092590347FF03C081E08093590383E0C6
:10D03000809356039F5F90935703CFC0933009F0BE
:10D04000C2C0232B09F0BFC09093550382E08093A8
:10D050005603809157038F5F8093570320915803A5
:10D06000822F9927782F6627842F9927682B792B71
:10D070008091DC05813049F47370CB01805092407F
:10D0800063E070E00E94327817C0823061F47770FC
:10D09000CB018050944066E070E00E943278269583
:10D0A000269526950BC0737068567140CB0177FDAD
:10D0B0000196BC017595679526952695022F112737
:10D0C0000F7010700F5F1F4F0D30110508F074C006
:10D0D0007801E00EF11EF701EC51F94F808191814A
:10D0E0009B01281B390BC90137FF03C0909581951F
:10D0F0009F4F069794F480916A02883C30F48091A7
:10D100006A02865F80936A0208C088EC80936A0294
:10D1100080916F008F7D80936F00F701EC51F94F84
:10D12000808191819C01220F331F280F391F260F08
:10D13000371F37FF02C02D5F3F4FE901D595C795D7
:10D14000D595C795CB0101968C179D0714F42197AF
:10D1500006C061507040C617D7070CF42196809125
:10D160006A02843BD0F0F701EC51F94F8081918144
:10D17000FE01E81BF90BCF0163E070E00E943278FA
:10D18000CB01880F991F860F971F28E137E0E20E29
:10D19000F31EF7019183808307C028E137E0E20E98
:10D1A000F31EF70111821082000F111F0C51194F4D
:10D1B000F801D183C08311C00231110570F081E004
:10D1C0008093A0010AC081E08093A00110925703D0
:10D1D0001092590384E48093550380915703803162
:10D1E00098F080915903882331F48091A00188231D
:10D1F00011F4809341011092570310925903109239
:10D20000560384E480935503E6E0CDB7DEB70C9473
:10D21000AA78CF93FC0197FF05C0CFEFF095E19579
:10D22000FF4F01C0C1E028E631E0CF01B9010E9403
:10D230003278FC018B35910554F08B5590408A353E
:10D24000910538F484EB90E08E1B9F0BFC0141E0CC
:10D250000DC0CF01855B90408A35910518F4E45BE1
:10D26000F04003C02E1B3F0BF9014FEFEE0FFF1FE5
:10D27000E25DF64F259134918C2F992787FD90958B
:10D28000289FB001299F700D389F700D1124842FA5
:10D29000992787FD9095689FA001699F500D789F01
:10D2A000500D1124CA01CF9108952AE530E0281BC2
:10D2B000390BC9010E9409690895CF93DF9380E07B
:10D2C0000E94076F80911E0190911F016AE070E03B
:10D2D0000E9432789F938F9380911E0190911F013D
:10D2E0006AE070E00E9432787F936F9382E09AE068
:10D2F0009F938F93CAEFDEE6DF93CF93E0917503A0
:10D30000F091760309952DB73EB7285F3F4F2DBFAB
:10D3100080919C01882361F186E00E94076F8091D3
:10D32000920199279F938F938091BC079091BD079D
:10D330006AE070E00E941E787F936F938FED90E01B
:10D340009F938F9380915A0790915B079F938F9340
:10D350008BE09AE09F938F93DF93CF93E0917503D7
:10D36000F091760309958DB79EB70C968DBF12C0CC
:10D3700086E00E94076F89E19AE09F938F93DF9385
:10D38000CF93E0917503F091760309950F900F907C
:10D390000F900F90809144038823F9F086E00E945B
:10D3A000076F8091440399279F938F9380E29AE0BF
:10D3B0009F938F93DF93CF93E0917503F091760362
:10D3C00009952DB73EB72A5F3F4F2DBF8091690267
:10D3D000882319F08FE48093A60180E10E94076FF3
:10D3E0008091A8019091A9016CE370E00E941E78E1
:10D3F0009F938F938091A8019091A9016CE370E0B5
:10D400000E941E787F936F93809136089091370821
:10D410009F938F938CE29AE09F938F93CAEFDEE6FF
:10D42000DF93CF93E0917503F09176030995809196
:10D430009D072DB73EB7265F3F4F2DBF80FF29C008
:10D440008AE10E94076F8091420199279F938F93F1
:10D450008091640290916502A0916602B09167028A
:10D46000BC01CD0124E630E040E050E00E94677846
:10D470003F932F9389E39AE09F938F93DF93CF930A
:10D48000E0917503F091760309958DB79EB70896E4
:10D490008DBFDF91CF910895CF93DF9380E00E94FD
:10D4A000076F8091A206992787FD90959F938F9390
:10D4B00080919A06992787FD90959F938F938091ED
:10D4C0009206992787FD90959F938F9380918A0666
:10D4D000992787FD90959F938F9380E49AE09F937F
:10D4E0008F93CAEFDEE6DF93CF93E0917503F0915F
:10D4F0007603099580E10E94076F2DB73EB7245F40
:10D500003F4F2DBF8091C206992787FD90959F932D
:10D510008F938091BA06992787FD90959F938F935B
:10D520008091B206992787FD90959F938F93809164
:10D53000AA06992787FD90959F938F9380E59AE09F
:10D540009F938F93DF93CF93E0917503F0917603D0
:10D5500009958091B4052DB73EB7245F3F4F2DBF8D
:10D56000853098F480E10E94076F80E69AE09F93EF
:10D570008F93DF93CF93E0917503F0917603099534
:10D580000F900F900F900F9018C08730B0F488E183
:10D590000E94076F8FED90E09F938F9381E79AE051
:10D5A0009F938F93DF93CF93E0917503F091760370
:10D5B00009958DB79EB706968DBFDF91CF910895DF
:10D5C0000F931F9380E00E94076F2AE030E0809164
:10D5D000320890913308B9010E941E789F938F936F
:10D5E0008091320890913308B9010E941E787F9390
:10D5F0006F9380911E0190911F01B9010E943278B2
:10D600009F938F9380911E0190911F01B9010E94F9
:10D6100032787F936F938AE79AE09F938F930AEF14
:10D620001EE61F930F93E0917503F0917603099521
:10D6300080E10E94076F8DB79EB70C968DBF8091D9
:10D640003608909137089F938F938091340890917A
:10D6500035089F938F938CE89AE09F938F931F9345
:10D660000F93E0917503F091760309958DB79EB7FE
:10D6700008968DBF1F910F910895EF92FF920F931F
:10D680001F9380E00E94076F8FEDE82EF12CFF9230
:10D69000EF9280918F01909190019F938F93809151
:10D6A000430399279F938F9388E99AE09F938F93E1
:10D6B0000AEF1EE61F930F93E0917503F091760336
:10D6C000099580E10E94076F8DB79EB70A968DBFBE
:10D6D0008091410399279F938F93FF92EF928091BE
:10D6E000420399279F938F938BEA9AE09F938F939E
:10D6F0001F930F93E0917503F091760309958DB711
:10D700009EB70A968DBF1F910F91FF90EF900895DD
:10D710000F931F93CF93DF9380919C01CAEFDEE6B6
:10D72000882309F47DC080E00E94076F8091B907CB
:10D7300099279F938F938091BB0799279F938F93EE
:10D740008EEB9AE09F938F938E01DF93CF93E091BE
:10D750007503F091760309958DB79EB708968DBF36
:10D760008091BA07833031F48CE00E94076F8DEC12
:10D770009AE005C08CE00E94076F82ED9AE09F93CB
:10D780008F93DF93CF93E0917503F0917603099522
:10D790000F900F900F900F908091B80781FF12C0EB
:10D7A0008CE00E94076F87ED9AE09F938F931F9301
:10D7B0000F93E0917503F091760309950F900F9008
:10D7C0000F900F9080E10E94076F8091920199273E
:10D7D0009F938F938FED90E09F938F938091BE07DF
:10D7E0009091BF079F938F938091BC079091BD0745
:10D7F0006AE070E00E941E787F936F938CED9AE050
:10D800009F938F938AEF9EE69F938F93E09175038A
:10D81000F091760309958DB79EB70C968DBF12C017
:10D8200082E00E94076F8FEE9AE09F938F93DF93C1
:10D83000CF93E0917503F091760309950F900F90C7
:10D840000F900F90DF91CF911F910F910895CF937B
:10D85000C82F20915A0320935B0399278F3291059B
:10D86000E1F0803391051CF44F9779F027C08F3495
:10D870009105D9F08F38910509F586E0289FF001D0
:10D880001124EC51F64F849117C086E0289FF001D7
:10D890001124EB51F64F84910FC086E0289FF001D0
:10D8A0001124EA51F64F849107C086E0289FF001C9
:10D8B0001124E951F64F849180935A0390915A03B1
:10D8C00080915B039813C0E00E940D6F90915A0302
:10D8D00086E0989FF0011124E851F64F259134918C
:10D8E0008C2FF901099580E090E0CF910895109276
:10D8F00033081092320810923708109236081092AE
:10D90000350810923408109238088AE090E00E949E
:10D91000A51690935D0380935C030895CF93DF93E6
:10D9200080915C0390915D030E94AE16882309F4F8
:10D93000AFC080915C0390915D030A9690935D0364
:10D9400080935C03E0E0F0E09F0190E05FEFA3E8EC
:10D95000B6E04BE0ED018B8187FF0BC09F5F8D81AF
:10D96000E80FF11D8981280F311D8E81851708F47C
:10D97000582F4150189647FFEDCF50933808232B6E
:10D9800041F520916203309163034091640350910B
:10D990006503BB27A52F942F832F9093610380935A
:10D9A0006003AA27BB27281B390B4A0B5B0BCF014F
:10D9B000AA27BB27280F391F4A1F5B1F209362032A
:10D9C000309363034093640350936503E5E0F0E014
:10D9D00013C020916003309161032E173F0718F4A4
:10D9E000E21BF30B02C0E0E0F0E0892F9927880FDB
:10D9F000991FE80FF91F3596F0933308E09332082A
:10DA0000EF3FF10578F480911E0190911F018E9FE8
:10DA100090018F9F300D9E9F300D1124C90164E647
:10DA200070E013C0CF0196958795969587952091C4
:10DA30001E0130911F01289FA001299F500D389F82
:10DA4000500D1124CA0169E170E00E941E787093A4
:10DA500035086093340820915E0330915F032E0FE8
:10DA60003F1F30935F0320935E035EE02131350753
:10DA700078F0809136089091370801969093370896
:10DA80008093360820513E4030935F0320935E031D
:10DA9000DF91CF9108954FB720E430E0F894809162
:10DAA000C9008F778093C9008091C9008F7B8093D4
:10DAB000C9008091C9008F7D8093C9005A9A5298FD
:10DAC0005B9A539A832F99278093CD002093CC00A3
:10DAD0008091C80082608093C80088E18093C9006B
:10DAE0008091CA008F778093CA008091CA008F7B93
:10DAF0008093CA008091CA008F7D8093CA00809174
:10DB0000CA008F7E8093CA008091CA00877F80936D
:10DB1000CA008091C9008B7F8093C9008091CA00A0
:10DB200084608093CA008091CA0082608093CA009A
:10DB30008091C80087FF03C08091CE00F9CF80910B
:10DB4000C90080688093C9004FBF08950F931F9349
:10DB5000CF93DF93482F4F5F893108F08BC08091BE
:10DB6000E306841720F44F5F4093E3064150CB0156
:10DB700083539B4268E170E00E943278A42FBB2758
:10DB8000FD01EA0FFB1FEC51F94F808191819B0150
:10DB9000281B390BC90137FF03C0909581959F4F12
:10DBA000069794F480916A02883C30F480916A026E
:10DBB000865F80936A0208C088EC80936A02809135
:10DBC0006F008F7D80936F00FD01EA0FFB1FEC510A
:10DBD000F94F808191819C01220F331F280F391F3B
:10DBE000260F371F37FF02C02D5F3F4FE901D59544
:10DBF000C795D595C795CB0101968C179D0714F451
:10DC0000219706C061507040C617D7070CF42196C3
:10DC100080916A02843BD8F08D010A0F1B1FF80126
:10DC2000EC51F94F80819181FE01E81BF90BCF0186
:10DC300063E070E00E943278CB01880F991F860F55
:10DC4000971F085E184FF8019183808307C0AA0FC1
:10DC5000BB1FA85EB84F11961C921E92E42FFF279F
:10DC6000EE0FFF1FEC51F94FD183C083443011F404
:10DC700010924101DF91CF911F910F910895CF93A1
:10DC8000DF9320913908822F9927807F90704097E9
:10DC900009F06CC02F3109F046C080913A0880939A
:10DCA0006A0320913C0820936C0380913D08809387
:10DCB0006B03822F99279093E5068093E406222335
:10DCC00009F054C08091B605282F3327220F331F47
:10DCD000F901E85EF84F118210828091B705A82FF4
:10DCE000BB27AA0FBB1FFD01E85EF84F118210820F
:10DCF0008091B905E82FFF27EE0FFF1FCF01885E47
:10DD0000984FEC01198218822C51394FE901198280
:10DD10001882AC51B94F11961C921E92EC51F94FDA
:10DD20001182108223C0C22FCF70CA30F8F48091C4
:10DD30003A088093630880913B0880936208809141
:10DD40003C088093650880913D0880936408609149
:10DD50006208709163088C2F0E94A66D6091640820
:10DD6000709165088C2F8F5F0E94A66DDF91CF9117
:10DD70000895CF93C82F8F3F49F480916D038F3F53
:10DD800029F410926F0310926E0332C020916F033A
:10DD9000222339F4CF3111F485E001C084E080936F
:10DDA00070038091700390916E038217A0F4892F05
:10DDB000809580936E038F3F19F48EEF80936E03EE
:10DDC00080916E03C81711F40E943F6E10926F038A
:10DDD00010926E030BC0E22FFF27E75CF74FC08362
:10DDE0002F5F20936F039C0F90936E03C0936D037E
:10DDF000CF91089590916903933240F4E92FFF2762
:10DE0000E15CF74F80839F5F9093690308958332AD
:10DE100018F48D5F80936903089590E2E2E4F8E0DE
:10DE20008FE19193815087FFFCCF0895CF93CFB7B7
:10DE300023E031E0F8948091C9008F778093C90086
:10DE40008091C9008F7B8093C9008091C9008F7D2C
:10DE50008093C9005A9A52985B9A539A832F9927B4
:10DE60008093CD002093CC008091C8008260809385
:10DE7000C80088E18093C9008091CA008F778093A1
:10DE8000CA008091CA008F7B8093CA008091CA002B
:10DE900080628093CA008091CA0080618093CA002A
:10DEA0008091CA0088608093CA008091C900846014
:10DEB0008093C9008091CA0084608093CA008091D9
:10DEC000CA0082608093CA008091C80087FF03C0A7
:10DED0008091CE00F9CF8091C90080688093C900FD
:10DEE0008091C90080648093C9000E940D6FCFBFEC
:10DEF000CF910895282F99278F709070892B31F436
:10DF0000209580916803822B809368030895809107
:10DF1000A301882309F44BC08091340285FD04C01D
:10DF20008091A601882381F082E980933F0883E2F3
:10DF3000809340088091A601882309F485E58093A9
:10DF400041081092A60102C080933F088091A4016D
:10DF50008F3071F4809168030E94276C882341F010
:10DF600081E980933F088093400881E380934108D2
:10DF70001092A3018091C80085FFFCCF8091C90059
:10DF80008F7E8093C9008091C9008E7F8093C900E5
:10DF900080913F08882311F48EEF01C08EE78093B3
:10DFA000CE00809168038093A401109268030895C5
:10DFB0001F920F920FB60F9211248F939F93EF939E
:10DFC000FF939091A301992309F040C080917103C0
:10DFD000882361F480913F08882311F483E003C013
:10DFE000813999F481E0809371030FC0833099F4F3
:10DFF00080913F08882349F090933F088091C900A1
:10E000008E7F8093C9008EEF1EC08091C900816011
:10E010008093C9000EC0833261F48091C9008E7F65
:10E020008093C9008FEF8093CE0081E08093A3019D
:10E0300014C080917103E82FFF27E15CF74F8F5FD9
:10E040008093710380818093CE0007C0109271038A
:10E050008091C90080618093C900FF91EF919F91E9
:10E060008F910F900FBE0F901F901895EF92FF9217
:10E070000F931F93CF93DF937C018B01EA01452B14
:10E0800039F0F80181918F01F70109952197C9F7BE
:10E09000E6E0CDB7DEB70C94AA78EF92FF920F932B
:10E0A0001F93CF93DF937C018B01EA01452B41F055
:10E0B000F8010F5F1F4F8491F70109952197C1F770
:10E0C000E6E0CDB7DEB70C94AA780F931F93CF93F9
:10E0D0008C01C62F161634F480E2F8010995C15060
:10E0E0001C16D4F3CF911F910F9108950F931F9396
:10E0F000CF938C01C62F161634F480E3F8010995EE
:10E10000C1501C16D4F3CF911F910F910895A5E330
:10E11000B0E0EDE8F0E70C9482782E96EEADFFAD1E
:10E120002E9788249924540180916703882321F431
:10E130002C961FAE1EAE2C975EE4452E512C4C0E35
:10E140005D1E6F01B60105C0153239F00894C11C7F
:10E15000D11CF60114911123B9F7A601461B570BE8
:10E1600031F02C968EAD9FAD2C970E944D701123EF
:10E1700009F46AC20894C11CD11CFF24FDA6FCA6A8
:10E180004FEFE42EF9A6F6010894C11CD11C14919E
:10E19000153721F0812F80628837B1F4F0FE0AC074
:10E1A000F20124E030E0420E531E80809180A28074
:10E1B000B3800AC0F20142E050E0440E551E808157
:10E1C00091814C01AA24BB24103221F489A5882313
:10E1D000D1F61DC0133219F458E0F52AD4CF1A3203
:10E1E00011F01D3291F41A3259F4F20182E090E0FC
:10E1F000480E591EE081ECA7EE232CF6E195ECA722
:10E2000090E1F92AAFEDFA22BECF1B3211F419A723
:10E21000BACF1E32C1F5F6010894C11CD11C14916D
:10E220001A3279F4F20122E030E0420E531E4081AE
:10E2300051813FEF4F3F530714F44FEF5FEFE42E50
:10E24000A2CF40E050E0812F80538A30A0F4CA0171
:10E2500033E0880F991F3A95E1F7840F951F480F17
:10E26000591F410F511D40535040F6010894C11CE5
:10E27000D11C1491E8CF8FEF4F3F580714F44FEFA4
:10E280005FEFE42E85CF103329F4F4FC7CCF90E2CD
:10E29000F92A79CF812F81538930D8F440E050E0BA
:10E2A000CA0123E0880F991F2A95E1F7840F951F73
:10E2B000480F591F410F511D40535040F60108941B
:10E2C000C11CD11C1491812F80538A3048F34CA774
:10E2D0005FCF183619F4A4E0FA2A55CF1C3619F48A
:10E2E000B1E0FB2A50CF133661F43E010894611C63
:10E2F000711CF20122E030E0420E531E80818983BE
:10E300003CC1143421F0143611F0193651F514348F
:10E3100011F431E0F32AF0FE0AC0F20144E050E0CB
:10E32000440E551E80809180A280B3800CC0F20103
:10E3300082E090E0480E591E808191814C01AA2410
:10E3400097FCA094BA2CB7FE0AC0B094A094909405
:10E350008094811C911CA11CB11C8DE289A70AE04C
:10E360006FC01F3411F01F3631F41F3411F491E0E7
:10E37000F92A08E064C0103779F4F201A2E0B0E0B5
:10E380004A0E5B1E808191814C01AA24BB2400E1CE
:10E39000B0E4FB2A18E753C01337C1F5F20122E0BD
:10E3A00030E0420E531E608071806114710489F464
:10E3B0003E010894611C711C88E289838EE6F3019A
:10E3C000818385E78B838CE68C838D8389E28E83C2
:10E3D0001F82E7FC13C08E2D992787FD9095AC0115
:10E3E00060E070E0C3010E944F76009729F0382E5C
:10E3F0003618E3140CF0C3C03E2CC1C0F3010190E9
:10E400000020E9F731973E2E3618B9C0153511F0C6
:10E41000153731F4153511F4F1E0FF2A0AE00FC089
:10E42000183519F0183709F0A0C000E1F3FE07C055
:10E4300081149104A104B10411F020E4F22A19A678
:10E44000EDA6E7FC02C03FEDF32289E2682E712CB5
:10E450006C0E7D1E81149104A104B10421F44DA51C
:10E46000442309F47BC0802F9927AA27BB278EA7B6
:10E470009FA7A8ABB9AB202E332490E0891690E07B
:10E48000990691E0A90690E0B90648F0C501B401EB
:10E490002EA53FA548A959A90E94457817C0AFEFFE
:10E4A0008A169104A104B10449F040F0C401B101FD
:10E4B0000E941E789B014427552708C0882D602F95
:10E4C0000E941278282F3327442755272AAB3BABCD
:10E4D0004CAB5DAB0A3059F48AA9880F880F880FBE
:10E4E0009AA9990F890F382D381B832F10C000313E
:10E4F00039F48AA98295807F482D481B842F07C054
:10E500008AA9880F880F880F582D581B852F90E0F7
:10E510002EA53FA548A959A982169306A406B506BB
:10E5200008F091E08AA89BA8ACA8BDA88A3010F496
:10E53000805D04C0895A183509F48F7DD3018E930C
:10E540003D01992309F099CF083041F4F3FE06C04C
:10E55000803321F080E3FD0182933F01CE010196DB
:10E56000382E3618F8E23F0E0BC0112309F46CC0A8
:10E570003E010894611C711C1983B1E03B2E19A661
:10E58000032D2DA4231827FC222489A5882311F00C
:10E590000F5F02C0F6FC0E5F020DEF2CFF24C701D7
:10E5A00080739070892B49F48CA5801B682F2C9662
:10E5B0008EAD9FAD2C970E94657089A5882331F0A0
:10E5C00041E050E0BE01675D7F4F0AC0E6FE0EC02D
:10E5D00080E38AA71BA742E050E0BE01665D7F4F43
:10E5E0002C968EAD9FAD2C970E943670C70180731C
:10E5F0009070809749F48CA5801B682F2C968EAD67
:10E600009FAD2C970E947670622D2C968EAD9FAD9B
:10E610002C970E947670832D992787FD9095AC01E9
:10E62000B3012C968EAD9FAD2C970E943670E4FE00
:10E6300089CD2CA5201B2CA7622F2C968EAD9FADCB
:10E640002C970E9465707ECDE2E1CB5C0C949E78A5
:10E650002FB740E0F894E0E0F0E081E280935700CB
:10E660009491E2E0F0E0809357003491E4E0F0E030
:10E670008093570084912FBF9E3199F4363941F42D
:10E68000893011F441E00DC08A3059F442E009C0EC
:10E69000373939F4863011F443E003C0853009F48A
:10E6A00044E0842F992708959FB7F8948091C9007A
:10E6B000877F8093C9008091C9008F7E8093C900B5
:10E6C0008091C9008F778093C9008091C9008F7BAA
:10E6D0008093C9008091C9008F7D8093C9005298B2
:10E6E0005A9A53985B9A9FBF08951F93CF93DF93D5
:10E6F000182F80916703882309F4A9C08091A20193
:10E70000181709F4A4C080916603882321F40E949D
:10E7100028738093660382ED91E09093400180938B
:10E720003F0186EF9BE09F938F93C6E9D2E1DF9391
:10E73000CF93E0917503F091760309950F900F90B8
:10E740000F900F90812F99278330910539F18430F4
:10E7500091054CF48130910591F082309105DCF403
:10E76000892B51F036C085309105F1F08530910547
:10E77000C4F00697E1F02DC086EE9BE002C084ED68
:10E780009BE09F938F93DF93CF93E0917503F0917C
:10E79000760309952AC08BEB9BE0F3CF88E99BE0D9
:10E7A000F0CF8AE89BE0EDCF82E89BE0EACF84E7F8
:10E7B0009BE09F938F93DF93CF93E0917503F0914C
:10E7C0007603099588ED91E09093400180933F0195
:10E7D0000CC083E09CE09F938F93DF93CF93E091F5
:10E7E0007503F0917603099510E00F900F900F904C
:10E7F0000F9080916603843011F0823099F40E946A
:10E800005473812F8150833018F40E9465671DC0B6
:10E81000143019F40E94166F18C01530B1F40E941C
:10E820004B6D13C0112389F089E19CE09F938F9376
:10E8300086E992E19F938F93E0917503F0917603BF
:10E8400009950F900F900F900F901093A201DF91F8
:10E85000CF911F9108950F931F9381E080936703D9
:10E860004091A101E4E2FBE020E030E05FE484912C
:10E8700099272F5F3F4F829FB001839F700D929F1A
:10E88000700D112446275150319657FFF0CF409319
:10E89000A101ECEFFAE020E030E057E28491992703
:10E8A0002F5F3F4F829FB001839F700D929F700D2D
:10E8B000112446275150319657FFF0CF4093A101C4
:10E8C00080916603882321F40E9428738093660355
:10E8D0008091A101833459F088E190E029E20FB6DC
:10E8E000F894A895809360000FBE2093600087E89D
:10E8F00090E7909376038093750384E39CE09F9365
:10E900008F9306E912E11F930F93E0917503F09145
:10E91000760309950F900F900F900F9083E690E08B
:10E920009F938F9386E590E09F938F931F921F9202
:10E93000809102016AE00E941278892F99279F93A3
:10E940008F93809102010E94127899279F938F9351
:10E950008AE59CE09F938F931F930F93E09175033B
:10E96000F0917603099584E29BE09F938F931F9328
:10E970000F93E0917503F091760309958CEF9AE07F
:10E980009F938F931F930F93E0917503F0917603FC
:10E9900009958DB79EB746968DBF8EE89CE09F93F4
:10E9A0008F931F930F93E0917503F0917603099570
:10E9B00082EC8093810080916F00806280936F0071
:10E9C0000F900F900F900F901F910F9108958091CD
:10E9D0001B068F3138F08091B80787FD03C08EE1A8
:10E9E00080931B068091CB05882331F080558536B6
:10E9F00018F08FE78093CB050895CF93809167033C
:10EA0000882309F46EC08091720381508093720351
:10EA1000882309F04FC089E18093720380911B061F
:10EA2000803238F08091B80787FD03C08FE1809372
:10EA30001B0680916A02823800F580913502909120
:10EA40003602885E934020F4109274031092730390
:10EA50008091730390917403009739F1019790931B
:10EA6000740380937303419728F18091B80784FF62
:10EA700021C08091330284601BC080916A02853B73
:10EA8000C8F090911B0684E1989FC0011124409624
:10EA900020917303309174032817390730F42F5FE6
:10EAA0003F4F3093740320937303809133028B7F25
:10EAB00080933302C091A501CC2321F0C150C093B3
:10EAC000A5010FC086E98093A5018091A201843041
:10EAD00011F40E94876F8091A101833411F0C093DB
:10EAE0006703CF9108951F920F920FB60F921124D2
:10EAF0002F933F934F935F936F937F938F939F9346
:10EB0000AF93BF93EF93FF932091CE008091B0011C
:10EB10008823B1F02093C6008091B001823029F59E
:10EB20002F3F19F58FEF94E3ACE0B0E0C297A10955
:10EB3000B109B7FFFBCF8091B8038093CE0015C019
:10EB40009091A201892F8150833020F4822F0E945E
:10EB5000C0670BC0943021F4822F0E947A6F05C0E9
:10EB6000953019F4822F0E94B96EFF91EF91BF91F9
:10EB7000AF919F918F917F916F915F914F913F9155
:10EB80002F910F900FBE0F901F90189500242227F1
:10EB90003327442751E0BB27EE27FF27A0E1660F6C
:10EBA000771F881F991F001C221F331F441F660FE9
:10EBB000771F881F991F001C221F331F441F2AF430
:10EBC000050E2B1F3E1F4F1F04C0051A2B0B3E0BBB
:10EBD0004F0B550FBB1FEE1F587F556047FD52501E
:10EBE000AA95E9F6E695B7955795E695B7955795A1
:10EBF000852F9B2F08952227332741E0552768E072
:10EC0000880F991F221F331F880F991F221F331F40
:10EC10001AF4240F351F02C0241B350B440F551F57
:10EC2000487F456037FD42506A9551F756954795A4
:10EC300056954795842F0895AA2797FF04C080957D
:10EC400090958A1F9A1F77FF04C0609570956A1F80
:10EC50007A1F669F9001779FA001679F300D411D2D
:10EC60005A1F300D411D5A1F889FF001999F2E0F8A
:10EC70003F1F401D511D899F300D411D5A1F300DF2
:10EC8000411D5A1FCA01B901112480CFFB01DC01CB
:10EC900002C005900D9241505040D8F70895FC01F4
:10ECA0004150504030F001900616D1F73197CF0116
:10ECB0000895882799270895A0E0B0E0E2E6F6E7F6
:10ECC0000C948A786C017B01EA01590121978FEF3E
:10ECD000CF3FD80789F086010894C11CD11CC70119
:10ECE0000894E11CF11CF5010995F8018083219736
:10ECF000FFEFCF3FDF0779F7EAE0CDB7DEB70C943F
:10ED0000A678CF92DF92EF92FF920F931F937C0130
:10ED10006B01FB010995082FC7010196F6010995C2
:10ED2000182FC8011F910F91FF90EF90DF90CF90A7
:10ED30000895A0E0B0E0EFE9F6E70C948C788C0140
:10ED40007B01EA01690121978FEFCF3FD80771F06E
:10ED5000F70121917F01C8010F5F1F4F622FF6015C
:10ED600009952197FFEFCF3FDF0791F7E8E0CDB797
:10ED7000DEB70C94A878CF92DF92EF92FF920F93B8
:10ED80001F936C018B017A01FA010995812F992754
:10ED9000682FC6010196F70109951F910F91FF9009
:10EDA000EF90DF90CF9008955058BB27AA270ED040
:10EDB000E0C0D1D030F0D6D020F031F49F3F11F434
:10EDC0001EF4C6C00EF4E095E7FBBCC0E92FE2D00C
:10EDD00080F3BA17620773078407950718F071F478
:10EDE0009EF5FAC00EF4E0950B2EBA2FA02D0B0164
:10EDF000B90190010C01CA01A0011124FF27591B80
:10EE000099F0593F50F4503E68F11A16F040A22F85
:10EE1000232F342F4427585FF3CF469537952795F6
:10EE2000A795F0405395C9F77EF41F16BA0B620BF5
:10EE3000730B840BBAF09150A1F0FF0FBB1F661F3C
:10EE4000771F881FC2F70EC0BA0F621F731F841F7F
:10EE500048F4879577956795B795F7959E3F08F0A5
:10EE6000B3CF9395880F08F09927EE0F9795879564
:10EE7000089598D088F09F5790F0B92F9927B751EF
:10EE8000A0F0D1F0660F771F881F991F1AF0BA956E
:10EE9000C9F712C0B13081F09FD0B1E008959CC095
:10EEA000672F782F8827B85F39F0B93FCCF3869564
:10EEB00077956795B395D9F73EF4909580957095C1
:10EEC00061957F4F8F4F9F4F0895E89409C097FB3E
:10EED0003EF490958095709561957F4F8F4F9F4F31
:10EEE0009923A9F0F92F96E9BB279395F695879575
:10EEF00077956795B795F111F8CFFAF4BB0F11F438
:10EF000060FF1BC06F5F7F4F8F4F9F4F16C08823DE
:10EF100011F096E911C0772321F09EE8872F762F14
:10EF200005C0662371F096E8862F70E060E02AF055
:10EF30009A95660F771F881FDAF7880F9695879541
:10EF400097F9089597F99F6780E870E060E0089569
:10EF50009FEF80EC089500240A94161617061806F1
:10EF60000906089500240A941216130614060506CD
:10EF70000895092E0394000C11F4882352F0BB0F5E
:10EF800040F4BF2B11F460FF04C06F5F7F4F8F4FC1
:10EF90009F4F089557FD9058440F551F59F05F3FFC
:10EFA00071F04795880F97FB991F61F09F3F79F0AB
:10EFB00087950895121613061406551FF2CF46952D
:10EFC000F1DF08C0161617061806991FF1CF8695AF
:10EFD0007105610508940895E894BB276627772793
:10EFE000CB0197F90895629FD001739FF001829F32
:10EFF000E00DF11D649FE00DF11D929FF00D839FC8
:10F00000F00D749FF00D659FF00D9927729FB00D64
:10F01000E11DF91F639FB00DE11DF91FBD01CF0177
:10F0200011240895991B79E004C0991F961708F0E0
:10F03000961B881F7A95C9F780950895AA1BBB1B5C
:10F0400051E107C0AA1FBB1FA617B70710F0A61BE8
:10F05000B70B881F991F5A95A9F780959095BC0109
:10F06000CD01089597FB092E07260AD077FD04D01D
:10F07000E5DF06D000201AF4709561957F4F089562
:10F08000F6F7909581959F4F0895A1E21A2EAA1B3D
:10F09000BB1BFD010DC0AA1FBB1FEE1FFF1FA21748
:10F0A000B307E407F50720F0A21BB30BE40BF50B45
:10F0B000661F771F881F991F1A9469F760957095CE
:10F0C000809590959B01AC01BD01CF01089597FB00
:10F0D000092E05260ED057FD04D0D7DF0AD0001C1C
:10F0E00038F450954095309521953F4F4F4F5F4FE5
:10F0F0000895F6F790958095709561957F4F8F4FA5
:10F100009F4F08952F923F924F925F926F927F92FE
:10F110008F929F92AF92BF92CF92DF92EF92FF9227
:10F120000F931F93CF93DF93CDB7DEB7CA1BDB0BD3
:10F130000FB6F894DEBF0FBECDBF09942A88398878
:10F1400048885F846E847D848C849B84AA84B9847F
:10F15000C884DF80EE80FD800C811B81AA81B9818B
:10F16000CE0FD11D0FB6F894DEBF0FBECDBFED019F
:10F170000895EE0FFF1F0590F491E02D0994FFCF45
:10F180005E010A010164FF01FFFFC01FC01F0101F2
:10F1900001737373FF03007D0000C409C409640098
:10F1A000104661737400004E6F726D616C00004513
:10F1B000617379000051756164726F00006400D260
:10F1C0000101200B050000ECFF00020406070808FF
:10F1D000080706040200FEFCFAF9F8F8F8F9FAFC50
:10F1E000FE000204060708086440415A4664640AA7
:10F1F00002969696960840403A10FB30380132FF4E
:10F2000003780090D0030090D0030032002064FF08
:10F21000FF64200B0A0D0B0C0E0B0F10FA200101DE
:06F220000170FF010F6404
:00000001FF
